:100000000C94EE1C0C941F1D0C941F1D0C941F1DB2
:100010000C941F1D0C941F1D0C941F1D0C941F1D70
:100020000C941F1D0C941F1D0C941F1D0C941F1D60
:100030000C941F1D0D94F2080C941F1D0C941F1D91
:100040000C941F1D0C9442DB0C941F1D0C941F1D5F
:100050000C941F1D0C94EEDC0C94E5DB0D94B203A4
:100060000C941F1D0C9446DD0C9470DD0C941F1D28
:100070000C941F1D0C941F1D0C941F1D0C941F1D10
:100080000C941F1D0C941F1D0C941F1D0C941F1D00
:100090000C941F1D0C941F1D0C941F1D0D94C0016A
:1000A0000C941F1D0C941F1D0C941F1D0C941F1DE0
:1000B0000C941F1D0C941F1D0C941F1D0C941F1DD0
:1000C0000C941F1D0C941F1D0C941F1D0C941F1DC0
:1000D0000C941F1D0C941F1D0C941F1D0C941F1DB0
:1000E0000C941F1DD295EA95EA95EA95EA95EA9552
:1000F000EA95EA95EA95EA95EA95EA95EA95EA9508
:10010000EA95EA95EA95EA95EA95EA95EA95EA95F7
:10011000EA95EA95EA95EA95C19573957D95F794E8
:10012000EA95A395AD95EA95EA950895E594EA9543
:100130009995EA95B7958F958795EA95EA95EA9509
:1001400055955F956995EA95EA95EA95EA95EA9558
:10015000EA95EA95EA95EA95C19573957D95F794A8
:10016000EA95A395AD95EA95EA950895E594EA9503
:100170009995EA95B7958F958795EA95EA95EA95C9
:1001800055955F956995FAB28BB31EB46FB50AC4E5
:100190000AC40AC40AC40AC40AC40AC40AC40AC4EF
:1001A000B7B4F3B431B50AC40AC40AC40AC40AC451
:1001B0000AC40AC40AC40AC40AC40AC496B8F8B86D
:1001C00058B9B8B918BA78BAD8BA0AC454BF5CBB1F
:1001D000D2BB45BCB7BC29BD9BBD0DBE7ABEE7BE38
:1001E0000AC40AC40AC40AC40AC419B7E6B73CB7A9
:1001F0009CBF09C075C0E2C003C145C177C1A9C198
:1002000002C25DC2B6C20FC330C324C10AC40AC44D
:100210000AC40AC40AC40AC40AC40AC40AC40AC46E
:100220000AC40AC4B9B6E8B60AC40AC40AC40AC4ED
:100230000AC40AC40AC40AC4B2C30AC4B5B70AC409
:100240000AC40AC45AC388C30AC40AC40AC40AC472
:10025000EDB20AC40AC4B2B555B699B63EB8BC01EF
:100260008401BE019801B201C8017A01A201940182
:1002700092019001B6018601C401C801AA01A6013C
:100280009A019C01C601B401C001880196019E013A
:100290008201AE01A401BA0176017E018E019601B0
:1002A000A001AC01C20107634236B79BD8A71A3937
:1002B000685618AEBAAB558C1D3CB7CC5763BD6DB4
:1002C000EDFD753EF6177231BF000000803F05A8B6
:1002D0004CCDB2D44EB93836A9020C50B9918688AB
:1002E000083CA6AAAA2ABE000000803F0D94F40490
:1002F0000D9440000D943A030D941E000D94F804E3
:100300000D9431000D94E0040D9417030D947703C0
:100310000D94D1040D9441000D94A6050D94FC0498
:100320000D945E030D9454030D944A030D940F0530
:100330000D9426030D949F030D94D5040D94DC04B5
:100340000D9402050D9442030D94EA040D94950357
:100350000D9416000D948B030D9406050D94E60480
:100360000D946D000D9430030D94C7040D94680333
:100370000D94E1000D94EE040D9412030D941C03F2
:100380000D94CB040D940A050D9481030D94D804AB
:100390000D94A903436F6C6420657874727573695A
:1003A0006F6E20646973616C6C6F77656400436F76
:1003B0006C6420657874727573696F6E20616C6C03
:1003C0006F776564004175746F72657472616374F0
:1003D0003A0053657474696E67206D6F746F722094
:1003E00063757272656E742E2E2E00536574204DE7
:1003F0006963726F7374657070696E6700547269B7
:1004000067676572696E67207761746368646F6798
:100410002E204966206163746976617465642C20BE
:10042000746865207072696E7465722077696C6C8F
:100430002072657365742E0053657474696E67204D
:100440005468726573686F6C6420546F3A00494E4B
:10045000542050494E3A20004D323531200020744E
:100460006F200053657420766F6C756D65747269CA
:100470006320657874727573696F6E20666F722081
:100480006578747275646572200044697361626C8A
:10049000656420766F6C756D65747269632065782C
:1004A00074727573696F6E20666F722065787472EE
:1004B0007564657220004D313134200048656174E7
:1004C000696E67204265640048656174696E6720E3
:1004D00045787472756465720050696E2063616E50
:1004E000206E6F7420626520736574206279204DE0
:1004F00034322C206D617920696E20696E76616CD2
:100500006964206F7220696E207573652E20004922
:100510006C6C6567616C20532076616C7565206634
:100520006F72204D3432005A2028432920746F778F
:10053000657220666C6F6F722073657420746F3AF9
:100540002000592028422920746F77657220666C3C
:100550006F6F722073657420746F3A2000582028E2
:10056000412920746F77657220666C6F6F722073FB
:10057000657420746F3A2000526F64205261646980
:1005800075732073657420746F3A200047313334DB
:100590002000506F7346726F6D53746570733A002C
:1005A000436F6D7044656C74613A0043616C6962BD
:1005B000726174696F6E206D6F76656D656E742003
:1005C0006973206C696D6974656420746F203130C3
:1005D0006D6D2E004669727374206D6F76652074A0
:1005E0006F20746F75636820617420782C793D30BA
:1005F0002C3020746F206175746F2D7365742072B8
:1006000061646975732E0043616C6962726174691B
:100610006F6E206D6F76656D656E74206973206CEA
:10062000696D6974656420746F2031306D6D2E00C2
:1006300043616E6E6F7420736574207261646975B6
:100640007320616E6420666C6F6F7220617420731A
:10065000616D652074696D652E0043616C6962721D
:100660006174696F6E20636F6465206973206C69C3
:100670006D6974656420746F20626F74746F6D208F
:10068000313025206F66205A2068656967687400DC
:1006900052656C617469766520706F736974696FF7
:1006A0006E696E67004162736F6C75746520706F60
:1006B000736974696F6E696E670047363920005A36
:1006C0003A2000593A2000583A20004F46465345F8
:1006D0005453204F464620425920544F4F204D55E9
:1006E0004348205F20545259494E472041474149D1
:1006F0004E3A200053657474696E672050726F62C1
:10070000652053656E736974697669747920546FD6
:100710003A005A2070726F6265206661696C656488
:10072000206F6E2073656E73697469766974793AA7
:10073000200053657474696E672050726F62652083
:1007400053656E736974697669747920546F3A00E1
:100750005A2070726F6265206661696C6564206FF3
:100760006E2073656E73697469766974793A2000D6
:1007700053657474696E672050726F6265205365AB
:100780006E736974697669747920546F3A005A20DF
:1007900070726F6265206661696C6564206F6E209F
:1007A00073656E73697469766974793A2000686557
:1007B0006865004E6577205261646975733A200060
:1007C0004F6C64205261646975733A200043616C18
:1007D00063756C6174656420526164697573206926
:1007E0007320626164203A0053657474696E6720F7
:1007F00050726F62652053656E73697469766974AF
:100800007920546F3A005A2070726F6265206661D9
:10081000696C6564206F6E2073656E7369746976A8
:100820006974793A200053657474696E6720507258
:100830006F62652053656E73697469766974792097
:10084000546F3A005A2070726F6265206661696C5D
:100850006564206F6E2073656E7369746976697460
:10086000793A2000473332200050524F42452D5AEA
:100870004F46465345543A0047333000536574742D
:10088000696E672050726F62652053656E7369747C
:10089000697669747920546F3A0050726F6265739B
:1008A00020646F206E6F74206D617463682E204F1A
:1008B0006666206279200047333020004D313137A1
:1008C0002043414C4942524154494F4E20434F4DE1
:1008D000504C4554450068656865004E6577204872
:1008E0006F72697A6F6E74616C205261646975739E
:1008F0003A20004F6C6420486F72697A6F6E7461A1
:100900006C205261646975733A200043616C6375B1
:100910006C61746564205261646975732069732029
:100920006261643A20004D3131372043414C4942E5
:10093000524154494F4E204641494C454400436181
:100940006C6962726174696F6E204661696C65647E
:100950000053657474696E672050726F626520532E
:10096000656E736974697669747920546F3A005AB8
:100970002070726F626520284852202D205A207402
:100980006F77657229206661696C6564206F6E20DF
:1009900073656E73697469766974793A20004E657F
:1009A00077205A204865696768743A004F6C642064
:1009B0005A204865696768743A004D3131372043E1
:1009C000414C4942524154494F4E204641494C45C1
:1009D000440043616C6962726174696F6E204661A4
:1009E000696C65640053657474696E672050726F3A
:1009F00062652053656E73697469766974792054F1
:100A00006F3A005A2070726F626520284852202D7C
:100A10002043656E74657220506F696E742920667C
:100A200061696C6564206F6E2073656E73697469AB
:100A3000766974793A200047363920005A3A200006
:100A4000593A2000583A20004D31313720456E6424
:100A500073746F70204F6666736574204572726F91
:100A600072004F464653455453204F464620425944
:100A700020544F4F204D5543482E2041626F7274D1
:100A8000696E672E2053656E73697469766974792F
:100A90003A20004D3131372043414C4942524154B4
:100AA000494F4E204641494C45440043616C6962C0
:100AB000726174696F6E204661696C65640053658C
:100AC0007474696E672050726F62652053656E732F
:100AD0006974697669747920546F3A005A2070728B
:100AE0006F626520285A20546F77657229206661ED
:100AF000696C6564206F6E2073656E7369746976C6
:100B00006974793A20004D3131372043414C4942D4
:100B1000524154494F4E204641494C45440043619F
:100B20006C6962726174696F6E204661696C65649C
:100B30000053657474696E672050726F626520534C
:100B4000656E736974697669747920546F3A005AD6
:100B50002070726F626520285920546F7765722962
:100B6000206661696C6564206F6E2073656E7369C1
:100B70007469766974793A20004D313137204341E8
:100B80004C4942524154494F4E204641494C4544FC
:100B90000043616C6962726174696F6E20466169BD
:100BA0006C65640053657474696E672050726F627F
:100BB000652053656E736974697669747920546F22
:100BC0003A005A2070726F626520285820546F775F
:100BD000657229206661696C6564206F6E2073659B
:100BE0006E73697469766974793A2000456E64732E
:100BF000746F70287329206E6F7420776F726B6921
:100C00006E672070726F7065726C79005A2000599F
:100C100020005820004572726F723A20004D313129
:100C20003720454E4453544F50204552524F5200A6
:100C30004D3130342053300A4D3134302053300A96
:100C40004D313037004D3131372049324320457224
:100C5000726F722E2041626F7274696E6700493242
:100C600043204572726F72202D2043616C6962725D
:100C70006174696F6E2041626F7274656400456EC5
:100C80006473746F70287329206E6F7420776F728D
:100C90006B696E672070726F7065726C79005A2094
:100CA000005920005820004572726F723A20004DA2
:100CB00031313720454E4453544F50204552524F06
:100CC00052006578656375746547436F6465202FCE
:100CD00020717565756544656C74614D6F7665202E
:100CE00072657475726E73206572726F72006969D5
:100CF0007332646820616363656C65726F6D6574DF
:100D0000657220696E697469616C697A696E672EB3
:100D10002E2E00616363656C65726F6D657465721C
:100D2000206932632072656376206661696C656450
:100D30002E00616363656C65726F6D65746572200A
:100D4000777269746520693263206661696C6564D5
:100D50002E00616363656C65726F6D6574657220EA
:100D600073656E6420693263206661696C65642E08
:100D70000000000100250030001D000C00180024B8
:100D80000031001C000B00170023002F001B000A7D
:100D9000001E000D00FFFF0900030022002B001AB7
:100DA0000041004200000002003500206465672E0B
:100DB000204300206D656173757265642000457283
:100DC000726F723A436F756C64206E6F7420686F37
:100DD0006C642074656D7065726174757265200055
:100DE000206D730020616674657220004572726F19
:100DF000723A54656D702E20726169736564207457
:100E00006F20736C6F772E2052697365203D200030
:100E10004739310A4731452D313830463630303088
:100E20000A473930004D3131372045787472756486
:100E3000657220300A54300A4D38342050340A4745
:100E400039310A47314531373246363030300A477A
:100E5000314535463530300A473930001C151C14F1
:100E60000000002243141F1F70121C12AC115C11F1
:100E7000000000000000D410C80F780FFC0E800E98
:100E80000400081D900058091C01B007A801C806FD
:100E900034023006C002C0054C036805D8031805AB
:100EA0006404D004F00498047C056004080630044F
:100EB000940600042007D003AC07A8033808800379
:100EC000C408580350093003DC090803680AD80233
:100ED000F40AB002800B88020C0C6002980C3002FD
:100EE000240DF801B00DC0013C0E8001C80E300188
:100EF000540FB800B40F2800E00F00000400401D9C
:100F0000900060091C01B007A801D0063402380621
:100F1000C002C8054C036805D80318056404D8044A
:100F2000F00498047C05600408063004940600046C
:100F30002007D003AC07A80338088003C40858036F
:100F400050093003DC090803680AE002F40AB80219
:100F5000800B88020C0C6002980C3002240DF80102
:100F6000B00DC0013C0E8001C80E3001540FB80016
:100F7000B40F2800E00F000004000016D800C006DF
:100F8000AC0178058002C004540348042804E80337
:100F9000FC049803D0055003A40618037807D80270
:100FA0004C08A80220097002F4093802C80A080295
:100FB0009C0BD001700C9001440D5001180EF800EC
:100FC000EC0E8800C00F00000400681D4C00500BA0
:100FD00094005809DC0050082401A8076C01280778
:100FE000B401C006FC017006440228068C02F0051C
:100FF000D402B8051C03880564035805AC0330050A
:10100000F40310053C04E8048404C804CC04A804D8
:10101000140590045C057004A4055804EC0538041C
:10102000340620047C060804C406F0030C07D80329
:101030005407C8039C07B003E40798032C088003F7
:1010400074087003BC085803040948034C093003B2
:1010500094091803DC090803240AF0026C0AE00270
:10106000B40AC802FC0AB002440BA0028C0B88022E
:10107000D40B70021C0C5802640C4002AC0C280209
:10108000F40C10023C0DF001840DD801CC0DB80118
:10109000140E98015C0E7001A40E4801EC0E1801AC
:1010A000340FD8007C0F8800C40F0800FC0F00002C
:1010B0000000000000000000000000000000000030
:1010C0000000000000000000000000000000000020
:1010D000000000000000401F450060094F0010099B
:1010E0005C00C0086B0070087D0020089200D007EB
:1010F000AC008007CC003007DE00E006230190063C
:101100005E014006A601F005FF01A0056D02500535
:10111000F30200059603B0045A046004400510046D
:101120004806C0036E077003A8082003EB09D0022D
:10113000230B8002410C3002390DE001040E9001B6
:10114000A20E4001170FF000690FA000A20F50007F
:10115000C60F0000DD0FB0FFEB0F60FF0400700D45
:10116000D8004804AC0158038002D802540380021E
:1011700028043802FC040002D005C801A406980126
:10118000780770014C08480120091801F409F000A3
:10119000C80AC8009C0BA000700C7000440D3800F9
:1011A000180E0000EC0EA8FFC00FE8FE0400001BA4
:1011B00054006009640010097400C00884007008BD
:1011C0009C002008B800D007D80080070001300735
:1011D0002C01E00668019006AC0140060002F00513
:1011E0006802A005E0025005740300052404B00461
:1011F000F0046004DC051004E406C0030408700376
:1012000030092003780B8002600DE001A80E400138
:10121000680FA000C00F0000E80F60FF0400801AF4
:10122000D8009808AC012007800250065403C80576
:1012300028045805FC040005D005B004A406680481
:10124000780728044C08E8032009B003F409700368
:10125000C80A38039C0BF802700CB002440D6802F7
:10126000180E0802EC0E8801C00F8800F00F000075
:101270000000A00F5C006009690010097900C00837
:101280008C007008A2002008BD00D007DE00800797
:10129000050130073401E0066D019006B2014006F9
:1012A0000702F0056D02A005E80250057B0300056A
:1012B0002B04B004F8046004EB06C00335092003D6
:1012C0007F0B8002650DE001B00E40011D0FF000A4
:1012D000480FC8006C0FA000ED0F60FFFE0F48FE26
:1012E000000200002110422063308440A550C660F7
:1012F000E770088129914AA16BB18CC1ADD1CEE1D3
:10130000EFF13112100273325222B5529442F77249
:10131000D662399318837BB35AA3BDD39CC3FFF322
:10132000DEE36224433420040114E664C774A44459
:1013300085546AA54BB528850995EEE5CFF5ACC572
:101340008DD55336722611163006D776F666955629
:10135000B4465BB77AA719973887DFF7FEE79DD7C2
:10136000BCC7C448E5588668A778400861180228B9
:101370002338CCC9EDD98EE9AFF9488969990AA912
:101380002BB9F55AD44AB77A966A711A500A333A89
:10139000122AFDDBDCCBBFFB9EEB799B588B3BBB62
:1013A0001AABA66C877CE44CC55C222C033C600C19
:1013B000411CAEED8FFDECCDCDDD2AAD0BBD688DB2
:1013C000499D977EB66ED55EF44E133E322E511E69
:1013D000700E9FFFBEEFDDDFFCCF1BBF3AAF599F02
:1013E000788F8891A981CAB1EBA10CD12DC14EF1A2
:1013F0006FE18010A100C230E32004502540467008
:101400006760B9839893FBA3DAB33DC31CD37FE332
:101410005EF3B1029012F322D23235421452776257
:101420005672EAB5CBA5A89589856EF54FE52CD502
:101430000DC5E234C324A0148104667447642454A7
:101440000544DBA7FAB79987B8975FE77EF71DC712
:101450003CD7D326F2369106B016576676761546F7
:1014600034564CD96DC90EF92FE9C899E9898AB962
:10147000ABA94458654806782768C018E108823847
:10148000A3287DCB5CDB3FEB1EFBF98BD89BBBAB72
:101490009ABB754A545A376A167AF10AD01AB32A97
:1014A000923A2EFD0FED6CDD4DCDAABD8BADE89DC2
:1014B000C98D267C076C645C454CA23C832CE01CE7
:1014C000C10C1FEF3EFF5DCF7CDF9BAFBABFD98F52
:1014D000F89F176E367E554E745E932EB23ED10E37
:1014E000F01E7C3C3E5E2B3D3F2F5B5D3B2C2A2259
:1014F0005C004D617854656D703A004469616D65BA
:101500007465723A00416363656C65726174696FFA
:101510006E3A004D617853706565643A004A6572B1
:101520006B3A004D617842656454656D703A0050C5
:1015300072696E746572547970653A44656C746151
:10154000005A54726176656C416363656C3A005968
:1015500054726176656C416363656C3A00585472ED
:101560006176656C416363656C3A005A5072696ECE
:1015700074416363656C3A00595072696E744163DB
:1015800063656C3A00585072696E74416363656CB0
:101590003A005A53697A653A005953697A653A00B4
:1015A0005853697A653A005A4D61783A00594D614D
:1015B000783A00584D61783A005A4D696E3A0059B0
:1015C0004D696E3A00584D696E3A004A65726B5823
:1015D000593A005072696E746C696E654361636854
:1015E000653A00454550524F4D3A004175746F6C55
:1015F0006576656C3A005A50726F62653A004361D5
:1016000073654C69676874733A00537570706F72D4
:10161000744C6F63616C46696C616D656E74636870
:10162000616E67653A00537570706F727447313040
:101630004731313A005A486F6D654469723A005932
:10164000486F6D654469723A0058486F6D6544692A
:10165000723A00536F667477617265506F77657286
:101660005377697463683A004C43443A0046616EAC
:101670003A005344436172643A004865617465649A
:101680004265643A004D6978696E67457874727591
:101690006465723A004E756D457874727564657252
:1016A0003A00496E7075744275666665723A00421A
:1016B000617564726174653A004E6F206361736591
:1016C000206C6967687473004D31313420006465A3
:1016D0006C6179203130306D732E00686F6D65411B
:1016E0007869732000686F6D6541786973202F20D9
:1016F000717565756544656C74614D6F76652072B2
:10170000657475726E73206572726F7200486F6DCA
:10171000652044656C7461005072696E7465723A3C
:101720003A736574757020006D6F7665546F5265FD
:10173000616C202F20717565756544656C74614D11
:101740006F76652072657475726E73206572726F44
:1017500072006D6F7665546F202F20717565756509
:1017600044656C74614D6F76652072657475726E38
:1017700073206572726F72005374657070657220A9
:1017800044697361626C6564004B696C6C656400EC
:101790006973506F736974696F6E416C6C6F7765B4
:1017A0006420005344206572726F72206669786508
:1017B00064005344206572726F7220646964206E05
:1017C0006F74207265636F766572210053442052F6
:1017D000656164204572726F720055706C6F616450
:1017E000696E672E2E2E00005344207072696E744D
:1017F0002073746F707065642062792075736572F0
:101800002E005344206361726420696E73657274A4
:101810006564005344204361726420696E7365728D
:1018200074656400534420436172642072656D6F77
:1018300076656400534420636172642072656D6F45
:1018400076656400457874722E00436F6E66696732
:101850003A004F6E65206865617465722073656536
:101860006D73206465636F75706C65642066726F5C
:101870006D20746865726D6973746F72202D2064B9
:10188000697361626C696E6720616C6C20666F724F
:101890002073616665747921004865617465722002
:1018A0006465636F75706C6564004372656174692B
:1018B0006F6E206661696C6564004469726563746B
:1018C0006F727920637265617465640044656C654C
:1018D00074696F6E206661696C65640046696C6549
:1018E0002064656C6574656400446F6E6520736187
:1018F00076696E672066696C652E00577269746937
:101900006E6720746F2066696C653A20006F7065A1
:101910006E206661696C65642C2046696C653A20AE
:10192000004E6F74205344207072696E74696E6744
:10193000005344207072696E74696E672062797416
:1019400065200066696C652E6F70656E2066616942
:101950006C65640046696C652073656C65637465CD
:1019600064002053697A653A0046696C65206F709F
:10197000656E65643A00456E642066696C65206C2E
:1019800069737400426567696E2066696C65206CD6
:10199000697374006572726F722077726974696E10
:1019A0006720746F2066696C6500534420696E6916
:1019B00074206661696C00616476616E6365204CB9
:1019C000205B303D6F66665D006578747275646596
:1019D0007220636F6F6C6572207370656564205B45
:1019E000302D3235355D0064697374616E63652036
:1019F000746F2072657472616374207768656E20FD
:101A000068656174696E67205B6D6D5D0074656DFE
:101A1000702E20666F722072657472616374696FD4
:101A20006E207768656E2068656174696E67205BFB
:101A3000435D0074656D702E2073746162696C691A
:101A40007A652074696D65205B735D00592D6F6642
:101A500066736574205B73746570735D00582D6FD9
:101A60006666736574205B73746570735D005049BE
:101A700044206D61782076616C7565205B302D3275
:101A800035355D0050494420442D6761696E005032
:101A9000494420492D6761696E0050494420502D0A
:101AA0006761696E2F646561642D74696D650050AE
:101AB0004944206472697665206D696E005049441E
:101AC000206472697665206D6178006865617420B4
:101AD0006D616E61676572205B302D335D006163FF
:101AE00063656C65726174696F6E205B6D6D2F73D9
:101AF0005E325D0073746172742066656564726144
:101B00007465205B6D6D2F735D006D61782E2066AE
:101B100065656472617465205B6D6D2F735D007324
:101B20007465707320706572206D6D00426564206D
:101B3000504944206D61782076616C7565205B307A
:101B40002D3235355D004265642050494420442DD6
:101B50006761696E004265642050494420492D67E1
:101B600061696E004265642050494420502D6761D0
:101B7000696E00426564205049442064726976654C
:101B8000206D696E0042656420504944206472698A
:101B90007665206D61780042656420486561742037
:101BA0004D616E61676572205B302D335D00436F60
:101BB00072722E20646961676F6E616C2043205BD6
:101BC0006D6D5D00436F72722E20646961676F6E88
:101BD000616C2042205B6D6D5D00436F72722E2040
:101BE000646961676F6E616C2041205B6D6D5D00A3
:101BF0004D6178207072696E7461626C65207261EB
:101C000064697573205B6D6D5D00546F776572203C
:101C10005A20656E6473746F70206F6666736574A6
:101C2000205B73746570735D00546F776572205923
:101C300020656E6473746F70206F666673657420C0
:101C40005B73746570735D00546F77657220582004
:101C5000656E6473746F70206F6666736574205B65
:101C600073746570735D005365676D656E74732F73
:101C70007320666F722074726176656C00536567BD
:101C80006D656E74732F7320666F72207072696E4B
:101C900074696E6700486F72697A6F6E74616C2048
:101CA000726F642072616469757320617420302CD6
:101CB00030205B6D6D5D00446961676F6E616C2003
:101CC000726F64206C656E677468205B6D6D5D007B
:101CD000486F6D696E672066656564726174652022
:101CE0005B6D6D2F735D004D61782E2066656564B8
:101CF00072617465205B6D6D2F735D005374657048
:101D00007320706572206D6D0054726176656C2071
:101D1000616363656C65726174696F6E205B6D6D84
:101D20002F735E325D00416363656C657261746937
:101D30006F6E205B6D6D2F735E325D004D61782E8E
:101D4000206A65726B205B6D6D2F735D005A206D8C
:101D50006178206C656E677468205B6D6D5D0059FD
:101D6000206D6178206C656E677468205B6D6D5DB9
:101D70000058206D6178206C656E677468205B6D1B
:101D80006D5D005A20686F6D6520706F73205B6D0C
:101D90006D5D005920686F6D6520706F73205B6DFD
:101DA0006D5D005820686F6D6520706F73205B6DEE
:101DB0006D5D0053746F7020737465707065722070
:101DC000616674657220696E61637469766974799D
:101DD000205B6D732C303D6F66665D004D61782E23
:101DE00020696E6163746976652074696D65205B36
:101DF0006D732C303D6F66665D005072696E746560
:101E00007220616374697665205B735D0046696C5E
:101E1000616D656E74207072696E746564205B6DAF
:101E20005D00416476616E63656420557365720080
:101E30004261756472617465004550523A33200006
:101E40004550523A3220004550523A312000455018
:101E5000523A30200050726F746F636F6C20766559
:101E60007273696F6E206368616E6765642C20759C
:101E70007067726164696E6700436F6E666967754B
:101E8000726174696F6E20726573657420746F205F
:101E900064656661756C74732E00436F6E66696766
:101EA00075726174696F6E206C6F61646564206621
:101EB000726F6D20454550524F4D2E00436F6E6638
:101EC000696775726174696F6E2073746F7265648F
:101ED00020746F20454550524F4D2E004175746F50
:101EE0006C6576656C206163746976652028312F96
:101EF0003029005A2D70726F6265205933005A2DB7
:101F000070726F6265205833005A2D70726F62656F
:101F1000205932005A2D70726F6265205832005A73
:101F20002D70726F6265205931005A2D70726F6288
:101F300065205831005A2D70726F626520782D79B6
:101F40002D7370656564205B6D6D2F735D005A2D78
:101F500070726F6265207370656564205B6D6D2FB4
:101F6000735D005A2D70726F6265206F66667365CF
:101F7000742079205B6D6D5D005A2D70726F626503
:101F8000206F66667365742078205B6D6D5D004D13
:101F900061782E207A2D70726F6265202D20626527
:101FA0006420646973742E205B6D6D5D005A2D7022
:101FB000726F626520686569676874205B6D6D5D2E
:101FC0000077616974005072696E7465722068658B
:101FD000696768743A005A2D70726F626520666195
:101FE000696C6564005472616E73666F726D6174C2
:101FF000696F6E206D61747269783A004175746F13
:102000006C6576656C696E672064697361626C6586
:1020100064004175746F6C6576656C696E672065E8
:102020006E61626C6564004175746F6C6576656C99
:10203000206D617472697820726573657400004761
:1020400032382F6E47315A32352F6E005A2D70724A
:102050006F62652073746174653A005265736574CC
:10206000205A20686569676874005A2D70726F6223
:102070006520617665726167652068656967687467
:102080003A00205374657020566172696174696FFB
:102090006E2066726F6D2050726F626520746F20C3
:1020A0006265642044697374616E63653A005A2DF9
:1020B00070726F62653A005072696E746572207357
:1020C000657420696E746F206472792072756E2059
:1020D0006D6F646520756E74696C207265737461D0
:1020E000727421003A20776F726B696E67003A2034
:1020F00074656D702073656E736F722064656665BC
:102100006374006578747275646572200068656137
:1021100074656420626564004D54454D503A00502A
:102120004944204175746F74756E652066696E69E7
:1021300073686564202120506C6163652074686554
:10214000204B702C204B6920616E64204B6420630F
:102150006F6E7374616E747320696E20746865208D
:10216000436F6E66696775726174696F6E2E682061
:102170006F7220454550524F4D00504944204175E3
:10218000746F74756E65206661696C656421207476
:10219000696D656F757400504944204175746F74A2
:1021A000756E65206661696C6564212054656D708B
:1021B0006572617475726520746F20686967680064
:1021C000204B643A2000204B693A2000204B703AA3
:1021D000200020436C6173736963205049440020E0
:1021E00054753A2000204B753A2000206D61783AF2
:1021F0002000206D696E3A200020643A20002062A1
:102200006961733A2000504944204175746F7475B8
:102210006E652073746172740054617267657442F4
:1022200065643A0054617267657445787472004E53
:102230006F206D6F766520696E2064656C74612017
:102240007365676D656E742077697468203E203110
:10225000207365676D656E742E20546869732073F2
:10226000686F756C64206E65766572206861707049
:10227000656E20616E64206D6179206361757365A0
:1022800020612070726F626C656D210044656C7412
:10229000612052616469757320432830293A0044F3
:1022A000656C74612052616469757320422830291D
:1022B0003A0044656C746120526164697573204111
:1022C0002830293A00416C70686120432839302950
:1022D0003A00416C706861204228333330293A005B
:1022E000416C706861204128323130293A00546FC6
:1022F00077657220333A00546F77657220323A0066
:10230000546F77657220313A00496E76616C69646A
:102310002064656C746120636F6F7264696E6174B0
:1023200065202D206D6F76652069676E6F7265641C
:10233000006C696E656172204C3A00454550524F01
:102340004D2075706461746564002C207370656540
:10235000643D00206C696E656172207374657073F2
:102360003A004A65726B3A007A5F6D61783A00799B
:102370005F6D61783A00785F6D61783A004C2000BB
:10238000482000206973200020746F20005365747A
:10239000206F75747075743A20004D53312C4D5375
:1023A000322050696E730045313A0045303A005A88
:1023B0003A00593A0020002C00206D696E00206818
:1023C0006F7572732000206461797320006D2000A6
:1023D0005072696E74696E672074696D653A005059
:1023E00072696E7465642066696C616D656E743ABD
:1023F0000046616E73706565643A00482E20526134
:10240000646975733A00466C6F774D756C746970CA
:102410006C793A0053706565644D756C7469706CC5
:10242000793A00202F002F003A0020524157002017
:1024300042403A0020403A0020423A00543A0020FC
:10244000453A00205A3A0020593A0020583A00589C
:102450003A00467265652052414D3A00556E6B6EEA
:102460006F776E20636F6D6D616E643A00536F66B7
:102470007477617265205265736574005761746387
:1024800068646F672052657365740042726F776E7F
:10249000206F757420526573657400457874657299
:1024A0006E616C20526573657400506F776572556C
:1024B0007000737461727400424C4B2000736B693E
:1024C00070200020676F7420004572726F723A6549
:1024D00078706563746564206C696E652000534490
:1024E0002072656164206572726F72002052002054
:1024F0004A0020490020500020530020460020457B
:1025000000205A00205900205800446F6E6520704A
:1025100072696E74696E672066696C6500466F72D9
:102520006D6174206572726F720057726F6E6720F2
:10253000636865636B73756D004563686F3A00523D
:102540006573656E643A005761726E696E673A0032
:10255000496E666F3A004572726F723A00494E4694
:10256000004E414E006F6B004649524D5741524557
:102570005F4E414D453A52657065746965725F30D2
:102580002E39322E32204649524D574152455F4432
:102590004154453A3230313731313133204D4143A6
:1025A00048494E455F545950453A4F52494F4E2085
:1025B00044656C7461200052657175657374506177
:1025C0007573653A004D31313720494E53455254A9
:1025D0002053442043415244004D3131372053446D
:1025E0002043415244204552524F520055495F41C9
:1025F0004354494F4E5F5345545F4D4541535552E7
:1026000045445F4F524947494E20004E6F20534486
:1026100020436172640053687574204F66662041E0
:102620004C4C204865617473005072656865617434
:1026300020414253005072656865617420504C41DE
:102640000055495F414354494F4E5F484F4D455FE8
:102650005A200055495F414354494F4E5F484F4D02
:10266000455F59200055495F414354494F4E5F48EB
:102670004F4D455F58200055495F414354494F4EE7
:102680005F484F4D45414C4C200055495F414354F4
:10269000494F4E5F5A504F534954494F4E5F464140
:1026A00053545F4E4F54455354200055495F4143A6
:1026B00054494F4E5F5A504F534954494F4E5F4E05
:1026C0004F54455354200055495F414354494F4EA0
:1026D0005F45504F534954494F4E200055495F4183
:1026E0004354494F4E5F5A504F534954494F4E5FE0
:1026F00046415354200055495F414354494F4E5F72
:1027000059504F534954494F4E5F4641535420004E
:1027100055495F414354494F4E5F58504F534954B8
:10272000494F4E5F46415354200055495F41435441
:10273000494F4E5F5A504F534954494F4E20005510
:10274000495F414354494F4E5F59504F5349544993
:102750004F4E200055495F414354494F4E5F5850FA
:102760004F534954494F4E200042616E6742616E9B
:102770006700536C6F7742616E6700446561642047
:1027800054696D650050494400003A002064617945
:1027900073200050657263656E74205072696E74A8
:1027A00065643A00206465662000465720446174E1
:1027B00065203230313731313133004F52494F4E7D
:1027C0002044656C7461005365654D65434E43005C
:1027D0004F52494F4E2044656C7461005A34103496
:1027E000A6334933416374696F6E3A256C61000406
:1027F0000003004E6F00596573004E2F41004F6675
:1028000066004F6E000000003FCDCC4C3D0AD7A3C0
:102810003B6F12033A5265706574696572207620C9
:10282000302E39322E3200004014548025000040F2
:10283000380000004B00008070000000960000C0CF
:10284000DA000000E10000002C010008B2010000E5
:10285000C2010000F401000084030090D0030000D6
:10286000E803000008070020A1070000100E004048
:10287000420F0060E3160000000000110A0411047A
:102880000A1111001C1F11111F0000040A0A0A0E70
:102890001F1F0E001F1111111F0000001F1F1F1FFF
:1028A0001F0000040A040000000000040E15041CB0
:1028B0000000000200000600BA28D0302029A12D17
:1028C000F328F42D62290200000700CD28D030DB68
:1028D00028A12DF328F42D2C2D0729E22802A22E61
:1028E00000005072696E7465722053657474696E6D
:1028F000677300FA2802742F000041646A757374CC
:102900002054656D7073000E29023829000041645F
:1029100076616E6365642053657474696E677300D5
:10292000272902B92E00005072696E746572205317
:10293000657474696E67730002000009003F29D056
:10294000304D2A392A292A192A5129022AEA2962CC
:1029500029582902CF2C0000446562756767696EAB
:102960006700692902B12F000043616C69627261DE
:1029700074696F6E204D656E75000310270200812B
:10298000298C29852993290000000000A429000032
:102990000000006C6F6164656420662E2045455020
:1029A000524F4D00436F6E66696775726174696F4F
:1029B0006E000310270200B929C429BD29CB2900C4
:1029C00000000000DC29000000000073746F7265D5
:1029D0006420696E20454550524F4D00436F6E662E
:1029E000696775726174696F6E00F12903070400ED
:1029F000004C6F61642066726F6D20454550524FE8
:102A00004D00092A030604000053746F7265207498
:102A10006F20454550524F4D00202A025C2A00008D
:102A2000457874727564657200302A02632C000068
:102A3000466565647261746500402A028F2C00004F
:102A4000416363656C65726174696F6E00542A023C
:102A5000AF2B000047656E6572616C0002000010CC
:102A600000632AD0309B2B872B752B642B4F2B2098
:102A70002B382B092BF62AE22AD12AC02AAB2A9618
:102A80002A832A8A2A042F040000504944204D61D9
:102A9000783A255844009D2A0426040000447269AF
:102AA0007665204D61783A25584D00B22A042504F8
:102AB00000004472697665204D696E3A25586D00B4
:102AC000C72A042404000050494420443A2558648D
:102AD00000D82A042304000050494420493A2558CC
:102AE0006900E92A042204000044542F504944207C
:102AF000503A25587000FD2A042D040000436F6EE3
:102B000074726F6C3A25586800102B04460400005C
:102B1000416476616E6365206C696E3A25586C007D
:102B2000272B044D0400005761697420556E6974A9
:102B3000733A2558556D6D003F2B044C0400005727
:102B40006169742054656D702E25585402430056F7
:102B50002B042E040000537461622E54696D653A93
:102B6000255877006B2B042A040000416363656CD1
:102B70003A255841007C2B042B0400004D6178203D
:102B800046523A255846008E2B042C0400005374FC
:102B90006172742046523A25586600A22B0429041B
:102BA000000053746570732F4D4D3A255365000234
:102BB00000000400B62BD030EB2BD32BBE2BC52B43
:102BC00002FF2B00004D61782E20496E616374690D
:102BD000766500DA2B02312C000053746570706545
:102BE0007220496E61637469766500F22B041004EB
:102BF000000042617564726174653A256F63000379
:102C000058040200062C112C0A2C182C000000007D
:102C100000222C00000000005B735D20303D4F66F9
:102C200066004469732E2041667465723A256970A6
:102C3000000320040200382C432C3C2C4A2C0000BA
:102C4000000000542C00000000005B735D20303D4C
:102C50004F6666004469732E2041667465723A259A
:102C600069730002000003006A2CD030802C702CA5
:102C7000772C0413040000486F6D653A25665A00EE
:102C8000872C04160400004D61783A25667A00020C
:102C900000000400962CD030BE2CAE2C9E2CA52C0F
:102CA000040E0400004A65726B3A25616A00B52C77
:102CB000040D0400004D6F76653A25615A00C52C5D
:102CC000040A0400005072696E743A25617A0002A9
:102CD00000000500D62CD030192D062DF32CE02C49
:102CE000E72C03350400004472792072756E3A2592
:102CF000646400FA2C03340400004572726F72732E
:102D0000203A256465000D2D0333040000496E66EA
:102D10006F2020203A25646900202D033204000032
:102D20004563686F2020203A25646F00332D0240F0
:102D30002D000053442043617264204D656E750080
:102D40000200000600472DD030A12D8E2D782D6673
:102D50002D532D5A2D03F403010244656C657465EF
:102D60002066696C65006D2D02C02D020053746FE2
:102D700070205072696E74007F2D03F703040043C6
:102D80006F6E74696E7565205072696E7400952D52
:102D900003F60302045061757365205072696E7406
:102DA00000A82D03F503010253656C65637420537D
:102DB000442046696C65000100000100BE2DD03042
:102DC0000200000300C72DE22DD82DCD2DD42D03F8
:102DD0005424020059657300DF2D03E80300004E00
:102DE0006F00E92D010000000053746F70205072D5
:102DF000696E7400FB2D020C2E000041646A75732D
:102E0000742046616E2073706565640002000007DF
:102E100000132ED0308A2E762E612E4C2E372E2186
:102E20002E282E031E0400005365742046616E2078
:102E3000313030252525003E2E031D04000053654A
:102E4000742046616E20373525252500532E031C3E
:102E50000400005365742046616E20353025252519
:102E600000682E031B0400005365742046616E2029
:102E70003235252525007D2E031A0408005475726D
:102E80006E2046616E204F666600912E045204004B
:102E90000046616E2073706565643A25467325258A
:102EA00025000200000900A92ED030032FEA2E6170
:102EB0002F4E2F342FBC301C2F0200000900C02ED3
:102EC000D030032FEA2E612F4E2F342FBC30D22E5C
:102ED0001C2FD92E03B20F0000556E6C6F636B2050
:102EE00046756C6C204D656E7500F12E044804002B
:102EF00000466C6F772020526174653A256F662515
:102F00002525000A2F041F04000053706565642006
:102F1000526174653A256F6D25252500232F0342E4
:102F200004001044697361626C65205374657070AD
:102F3000657273003B2F03380400005368757420DA
:102F40004F666620414C4C20486561747300552FD4
:102F50000347040000507265686561742041425364
:102F600000682F03370400005072656865617420A3
:102F7000504C410002000004007B2FD030992F817B
:102F80002F882F043C0400004245442054656D7096
:102F90003A2020254562024300A02F043D04000092
:102FA0004E4F5A2054656D703A202025453002431B
:102FB000000200000600B82FD030EE2FC42FBC3026
:102FC0008630DA2FCB2F0421040000482E205261D6
:102FD00064697573203A256F6800E12F03AC0F0018
:102FE00000536574205A204F726967696E00F52F8F
:102FF000020630000046756C6C2043616C69627299
:103000006174696F6E0002000004000D30D030431F
:10301000302E3015301C3003B10F00004265676957
:103020006E2043616C6962726174696F6E00353045
:1030300003B50F00004245442041524520434C4512
:10304000414E004A3003B40F00004D414B45205320
:10305000555245204E4F5A5A4C452026000200003A
:1030600006006430D030BC30AA30983086307030E2
:10307000773002E9300000457874722E20706F734B
:103080006974696F6E008D30024A3200005A205018
:103090006F736974696F6E009F30029F3200005930
:1030A00020506F736974696F6E00B13002F43200A2
:1030B000005820506F736974696F6E00C33003FD50
:1030C000030000486F6D65205072696E7465720070
:1030D000D73003E803000050726576696F7573207E
:1030E00053637265656E20010003F0030400F03045
:1030F0000D310631FF30F83014310000000000229D
:1031000031000000000033310000000000423100B7
:1031100000000000255566206D207072696E746590
:10312000640020453A2565632F25456302437E25CB
:103130006F43003120636C69636B203D2031206D4B
:103140006D00453A257833206D6D0003FC030400C3
:1031500052316F31683161315A31763100000000EF
:103160000077310000000000873100000000009768
:10317000310000000000004D617820656E647374BA
:103180006F703A25735A004D696E20656E647374D2
:103190006F703A25737A005A3A257832206D6D00A7
:1031A00003FB030400A731C431BD31B631AF31CBCD
:1031B000310000000000CC310000000000DC3100D4
:1031C00000000000EC310000000000004D6178209C
:1031D000656E6473746F703A257359004D696E2083
:1031E000656E6473746F703A25737900593A257867
:1031F00031206D6D0003FA030400FC3119321232E4
:103200000B320432203200000000002132000000A6
:1032100000003132000000000041320000000000D8
:10322000004D617820656E6473746F703A25735831
:10323000004D696E20656E6473746F703A25737803
:1032400000583A257830206D6D0003EF03040051DB
:10325000326E32673260325932753200000000003F
:103260007632000000000086320000000000963236
:103270000000000000004D617820656E6473746F7B
:10328000703A25735A004D696E20656E6473746FD1
:10329000703A25737A005A3A257832206D6D000312
:1032A000EE030400A632C332BC32B532AE32CA32AB
:1032B0000000000000CB320000000000DB32000004
:1032C000000000EB320000000000004D6178206536
:1032D0006E6473746F703A257359004D696E206582
:1032E0006E6473746F703A25737900593A2578319A
:1032F000206D6D0003ED030400FB32183311330A17
:103300003303331F330000000000203300000000AF
:1033100000303300000000004033000000000000D7
:103320004D617820656E6473746F703A2573580030
:103330004D696E20656E6473746F703A2573780002
:10334000583A257830206D6D00000000040050339D
:103350006D3366335F335833743300000000007AF6
:103360003300000000008E330000000000923300A4
:1033700000000000255566206D00546F74616C20BC
:1033800046696C616D656E742055736564002555E2
:103390007400546F74616C205072696E74696E674A
:1033A0002054696D65000000000400AD33CA33C3CA
:1033B00033BC33B533D1330000000000DD330000EF
:1033C000000000EB330000000000FD3300000000AF
:1033D000004F52494F4E2044656C74610050726931
:1033E0006E746572204D6F64656C004657204461B1
:1033F00074653A203230313731313133004657204D
:1034000056657273696F6E3A20302E39322E320053
:103410000000000400173434342D3426341F343BAC
:103420003400000000003F34000000000048340079
:103430000000000051340000000000256F73005AA6
:103440003A257832206D6D00593A257831206D6D1E
:1034500000583A257830206D6D00000000040061AE
:10346000347E3477347034693485340000000000D1
:1034700089340000000000A2340000000000B534D0
:103480000000000000256F730053706565643A25E5
:103490006F6D25252520466C6F773A256F662525AB
:1034A00025004245443A256562205461726765747F
:1034B0003A254562004E4F5A3A25656320546172A1
:1034C0006765743A254563000000000000000000B5
:1034D000000000FF000001000000000000000000EC
:1034E000000000000000000024F403D950C38EB196
:1034F000C2A23D96828B3582127AE372816CCB66D2
:10350000A861015DC758EB546151204E1E4B5648CF
:10351000C14559431A41013F093D2F3B7139CD3710
:103520004036C93465331432D430A32F802E6B2D2E
:10353000632C672B752A8E29B028DC2710274B2691
:103540008F25D9242B248223E0224322AC211A2167
:103550008D200420801F001F841E0C1E971D261D19
:10356000B81C4E1CE61B821B201BC11A641A0A1AC7
:10357000B2195D190A19B9186A181C18D1178817D9
:103580004017FA16B51673163116F115B3157615E0
:103590003A150015C7148F1458142214EE13BA13D9
:1035A000881356132513F612C71299126C12401283
:1035B0001512EB11C1119811701148112111FB1056
:1035C000D610B1108D106910461024100210E10FB2
:1035D000C00FA00F800F610F420F230F060FE80EE0
:1035E000CB0EAF0E930E770E5C0E410E270E0D0E16
:1035F000F30DDA0DC10DA80D900D780D600D490D7C
:10360000320D1B0D050DEF0CD90CC30CAE0C990C33
:10361000850C700C5C0C480C350C210C0E0CFB0B53
:10362000E80BD60BC40BB20BA00B8E0B7D0B6B0BF8
:103630005A0B4A0B390B290B180B080BF80AE90A2D
:10364000D90ACA0ABB0AAC0A9D0A8E0A800A710A04
:10365000630A550A470A390A2C0A1E0A110A040A83
:10366000F709EA09DD09D009C409B709AB099F09BF
:10367000920987097B096F09630958094C094109B7
:1036800036092B09200915090A090009F508EB0874
:10369000E008D608CC08C208B808AE08A4089A0802
:1036A000900887087D0874086B08610858084F085F
:1036B00046083D0834082C0823081A08120809088F
:1036C0000108F807F007E807E007D807D007C807A0
:1036D000C007B807B007A807A1070000420FA1075D
:1036E0001605D0030D038B022E02E801B2018601FC
:1036F000630145012C0117010401F4004F52494FA9
:103700004E205265616479004F52494F4E205265F8
:10371000616479004F52494F4E20526561647900CF
:10372000207A3A0020793A0020783A00696E2071B8
:103730007565756544656C74614D6F766520746F51
:103740002063616C63756C61746544656C7461536E
:1037500075625365676D656E7473207265747572FA
:103760006E73206572726F722E0043206869742038
:10377000666C6F6F720043706F7320782073717581
:10378000617265200043706F7320782073746570D8
:1037900073200043706F73207920737175617265B7
:1037A000200043706F73207920737465707320005C
:1037B000422068697420666C6F6F720042706F738C
:1037C000207820737175617265200042706F7320DC
:1037D00078207374657073200042706F73207920B5
:1037E000737175617265200042706F732079207368
:1037F000746570732000412068697420666C6F6F77
:10380000720041706F73207820737175617265204A
:103810000041706F732078207374657073200041CD
:10382000706F73207920737175617265200041702B
:103830006F73207920737465707320006D6F7665E7
:1038400052656C617469766544697374616E636511
:10385000496E5374657073202F20717565756544CA
:10386000656C74614D6F76652072657475726E73E8
:10387000206572726F720000000A0B02090C0D0EB7
:103880000807030401000000000000000000000021
:103890000000000000000000000000000000000028
:1038A00000000012111000000000000000000000E5
:1038B00000000000000000000000000000010210F5
:1038C000202008081020401020408002010201083A
:1038D00004020101020408102040808040201008EA
:1038E0000402018004020180402010080402010843
:1038F00004020101020408102040800102040810A3
:103900002040800505050507050808080802020291
:10391000020A0A080804040404010101010101016A
:10392000010303030303030303040707070C0C0C41
:103930000C0C0C0C0C020202020606060606060619
:10394000060B0B0B0B0B0B0B0B00002000230026B0
:103950000029002C002F00320000010000030106A6
:1039600001090100002200250028002B002E003153
:1039700000340002010000050108010B01000021D4
:1039800000240027002A002D003000330001010030
:1039900000040107010A01024E414E494E495459A3
:1039A000494E46CDCCCC3D0AD7233C17B7D138770A
:1039B000CC2B329595E6241FB14F0A000020410020
:1039C00000C84200401C4620BCBE4CCA1B0E5AAE6A
:1039D000C59D74003A90739F20DEB80111241FBE6C
:1039E000CFEFD1E2DEBFCDBF00E00CBF13E0A0E01F
:1039F000B2E0EAEDF4E202E00BBF02C007900D92E4
:103A0000A039B107D9F72EE1A0E9B3E001C01D92BA
:103A1000A938B207E1F719E3CCEDD9E300E006C01D
:103A200022970109FE010BBF0F94E60DC43DD1079B
:103A300080E00807A9F70F9452090D946B120C94BB
:103A40000000CF93DF9300D01F92CDB7DEB744E0E4
:103A500050E0BC01CE0101960F94271269817A8152
:103A60008B819C810F900F900F900F90DF91CF91E1
:103A7000089522E090E0281728F4963019F0220FDC
:103A80009F5FF9CF209A289A219A229A23988091B1
:103A900064008B7F80936400892F806A86958CBD3B
:103AA00090FD03C081E0963009F480E08DBD08955B
:103AB0008091EA0283FB882780F90895179A089578
:103AC000169A0895159A089580B182FB882780F987
:103AD000089580B186958170089588E493E0B1CF10
:103AE000CF92DF92EF92FF92CF93DF9300D01F929D
:103AF0001F92CDB7DEB76B017C016093770770939F
:103B000078078093790790937A070E94DB74C982C3
:103B1000DA82EB82FC8244E050E065E773E0CE019C
:103B200001960F94491223E0B701A60188E795E0BA
:103B30000E948EA10E9437CF682F88E690E06D83A7
:103B40000F9437126D81681721F088E690E00F948A
:103B500052120F900F900F900F900F90DF91CF9116
:103B6000FF90EF90DF90CF900895CF93DF931F9257
:103B7000CDB7DEB7BC018DE793E00F9465120E94CC
:103B800037CF682F88E690E069830F9437126981F8
:103B9000681739F088E690E00F90DF91CF910D948F
:103BA00052120F90DF91CF910895CF93DF931F9220
:103BB000CDB7DEB7BC018FE793E00F9465120E948A
:103BC00037CF682F88E690E069830F9437126981B8
:103BD000681739F088E690E00F90DF91CF910D944F
:103BE00052120F90DF91CF910895CF93DF931F92E0
:103BF000CDB7DEB7BC0181E893E00F9465120E9457
:103C000037CF682F88E690E069830F943712698177
:103C1000681739F088E690E00F90DF91CF910D940E
:103C200052120F90DF91CF910895CF93C82F8091BA
:103C3000A6048823D1F01092A6040E94205A9091E5
:103C4000DF0291509093DF02911109C08091E00250
:103C5000833010F40E94AD5985E08093DF026C2F11
:103C600086E79AE0CF910C946CCACF910895809129
:103C70002C0C882349F00E94579880E0D6DF86E715
:103C80009AE00E946BCAF3CF08954F925F926F92B1
:103C90007F928F929F92AF92BF92CF92DF92EF92DC
:103CA000FF920F931F93CF93DF9300D01F92CDB756
:103CB000DEB78C018091F1079091F207A091F30794
:103CC000B091F40789839A83AB83BC83C090F507D6
:103CD000D090F607E090F707F090F8078090F9078A
:103CE0009090FA07A090FB07B090FC079C01AD01F3
:103CF000BC01CD010F94180D81110FC149805A806C
:103D00006B807C80E89477F82FEF3FEF4FE75FE719
:103D1000C301B2010F94180D81110BC02FEF3FEFBB
:103D20004FE75FE7C301B2010F94C50918160CF401
:103D3000F4C0A7019601C701B6010F94180D8111B7
:103D4000ECC026013701E89477F82FEF3FEF4FE7FB
:103D50005FE7C301B2010F94180D81110BC02FEF63
:103D60003FEF4FE75FE7C301B2010F94C509181693
:103D70000CF4D3C0A5019401C501B4010F94180D32
:103D80008111CBC024013501E89477F82FEF3FEF84
:103D90004FE75FE7C301B2010F94180D81110BC00B
:103DA0002FEF3FEF4FE75FE7C301B2010F94C50963
:103DB00018160CF4B2C02091C9073091CA0740917F
:103DC000CB075091CC0769817A818B819C810F94BC
:103DD00061092B013C012091CD073091CE07409124
:103DE000CF075091D007C701B6010F9461096B014D
:103DF0007C012091D1073091D2074091D307509197
:103E0000D407C501B4010F9461094B015C01809195
:103E10005108882329F020E732E441E25DE304C041
:103E200020E030E040E85FE3C301B2010F946D0C85
:103E3000AB01BC0122E08FE494E20E94CBA180910F
:103E40005108882329F020E732E441E25DE304C011
:103E500020E030E040E85FE3C701B6010F946D0C4D
:103E6000AB01BC0122E087E494E20E94CBA18091E7
:103E70005108882329F020E732E441E25DE304C0E1
:103E800020E030E040E85FE3C501B4010F946D0C21
:103E9000AB01BC0123E083E494E20E94CBA16091DA
:103EA000090870910A0880910B0890910C080F94F2
:103EB000980A20914D0830914E0840914F0850913A
:103EC00050080F946D0C20915108222329F020E70F
:103ED00032E441E25DE304C020E030E040E85FE32B
:103EE0000F946D0CAB01BC0124E08FE394E20F90C2
:103EF0000F900F900F90DF91CF911F910F91FF9036
:103F0000EF90DF90CF90BF90AF909F908F907F9079
:103F10006F905F904F900C948EA1C8010E94B09F4B
:103F20004ACFCF92DF92EF92FF92CF93DF93EC01D3
:103F3000893191053CF0C53F81E0D8072CF0C4EFF2
:103F4000D1E002C0C9E1D0E0BE01882777FD8095AD
:103F5000982F0F94980A6B017C0160910107709172
:103F60000207882777FD8095982F0F94980A9B0168
:103F7000AC01C701B6010F94CC099B01AC01609163
:103F800003077091040780910507909106070F942D
:103F90006D0C60930307709304078093050790935B
:103FA0000607D0930207C0930107BE0184E194E2A3
:103FB000DF91CF91FF90EF90DF90CF900C9474A0A1
:103FC000CF92DF92EF92FF926B017C0120E030E014
:103FD00040E752E40F94C50987FD11C020E030E0AE
:103FE00046E153E4C701B6010F94F90B18166CF4BF
:103FF000C12CD12C86E1E82E83E4F82E06C0C12C1A
:10400000D12C90E7E92E92E4F92EC0927707D09256
:104010007807E0927907F0927A0722E0B701A601CB
:104020008BEF93E2FF90EF90DF90CF900C948EA1F6
:104030008F929F92AF92BF92CF92DF92EF92FF92B8
:10404000CF93DF93EC018931910534F0893C9105E0
:104050002CF0C8ECD0E002C0C9E1D0E0D09300075A
:10406000C093FF06E0919003F0919103E258FF4F57
:10407000C080D180E280F38020E030E0A901C70158
:10408000B6010F94C509AE01662757FD6095762FDE
:1040900018165CF0CB01BA010F94980A2AE037EDAC
:1040A00043E25CE30F946D0C24C0CB01BA010F9482
:1040B000980A2AE037ED43E25CE30F946D0C20E0B0
:1040C00030E040E850E40F946D0C4B015C01A70117
:1040D0009601C701B6010F946D0C2BED3FE049E44A
:1040E00050E40F946D0C9B01AC01C501B4010F9419
:1040F000CC096093E5027093E6028093E702909307
:10410000E802BE0186E094E2DF91CF91FF90EF904C
:10411000DF90CF90BF90AF909F908F900C9474A041
:10412000CF93DF932091C50797FD0DC0EC018F3F22
:10413000910519F014F0CFEFD0E0209721F028601E
:104140002093C50705C0277F2093C507C0E0D0E0B6
:1041500061118DDD8091851D90E0C817D90729F088
:10416000BE0181EF93E20E9474A0C093851DDF9190
:10417000CF9108954F925F926F927F928F929F920C
:10418000AF92BF92CF92DF92EF92FF92CF93DF93E5
:1041900000D01F92CDB7DEB72FE632E143E85AE3F5
:1041A0006091E9067091EA068091EB069091EC0629
:1041B0000F946D0C6B017C0181E890E042DC9B0167
:1041C000AC01C701B6010F946109AB01BC0122E04B
:1041D0008FED93E20E94CBA18DEC93E20E94769F3B
:1041E000E0910A02F0910B0220E030E040E751E458
:1041F00063857485858596850F94F90B18160CF4E4
:104200006BC020E030E0A9018DE790E029833A837C
:104210004B835C830F943F124B015C0129813A81EF
:104220004B815C81820E931EA41EB51EC501B40194
:1042300020E831E541E050E00F94990D60E87EEA16
:104240008EEF9FEF0F94340D6B017C01C80CD91CCD
:10425000EA1CFB1CBA01A90180ED93E20E949AA01E
:10426000C701B60120E13EE040E050E00F94990D17
:1042700049015A01BA01A90186EC93E20E949AA071
:10428000A0EFB1EFA50194010F94E20D6C0D7D1D1F
:104290008E1D9F1D2CE330E040E050E00F94990DFF
:1042A000BA01A9018EEB93E20E949AA089EB93E2F6
:1042B0000F900F900F900F90DF91CF91FF90EF90A4
:1042C000DF90CF90BF90AF909F908F907F906F9036
:1042D0005F904F900C948F9F0F94FC03C090ED065D
:1042E000D090EE06E090EF06F090F0066C197D0994
:1042F0008E099F0928EE33E040E050E00F94770DDF
:1043000083CF5F988EBD0DB407FEFDCF6EBD0DB49B
:1043100007FEFDCF5F9A0895CF93DF9300D01F92E1
:104320001F92CDB7DEB795E0E7E4F3E0DE0111962A
:1043300001900D929A95E1F7E1E0F0E0EC0FFD1F9E
:10434000E80FF11D808190E00F900F900F900F907B
:104350000F90DF91CF91D5CFFF920F931F93CF9303
:10436000DF9300D01F921F92CDB7DEB785E0ECE45B
:10437000F3E0DE01119601900D928A95E1F780E05D
:1043800078DB579A8E010F5F1F4FF12CF801619176
:104390008F0170E08F2DC0DFF394F5E0FF12F6CFB0
:1043A0000F900F900F900F900F90DF91CF911F9172
:1043B0000F91FF90089567FD43C08230E9F028F423
:1043C000882341F0813061F03BC0833009F18430B3
:1043D00059F136C0662311F0A19A67C0A19865C053
:1043E00080910801662311F0806801C08F77809367
:1043F000080147FF3AC05DC080910801662311F0B3
:10440000806401C08F7B8093080147FF34C053C094
:1044100080910801662311F0886001C0877F809336
:10442000080147FF32C044C080910801662311F0A3
:10443000826001C08D7F8093080147FF2EC03AC083
:1044400047FD39C08230B9F028F4882341F081302B
:1044500061F008958330C9F08430F9F00895442361
:1044600011F0A09A0895A0980895442311F0A29AFB
:104470000895A298089580910801442311F0806264
:1044800001C08F7D80930801089580910801442325
:1044900011F08061F7CF8F7EF5CF80910801442322
:1044A00011F08460EFCF8B7FEDCF47FFD8CF089519
:1044B0000895089508950895643079F028F46130DE
:1044C00041F0623041F00895683051F0603141F0C0
:1044D000089540E003C040E004C041E060E002C055
:1044E00041E061E068CFCF93DF938AE993E20E94D5
:1044F0008F9F62B36695617070E08FE494E20E94D2
:1045000068A062B3617070E087EB93E20E9474A0D0
:10451000C6E0D1E08881992787FD9095692F661FB5
:104520006627661F70E082EB93E20E9468A062B388
:1045300062FB662760F970E087EB93E20E9474A04B
:10454000688166FB662760F970E08FEA93E20E945B
:1045500068A0688165FB662760F970E087EB93E2ED
:104560000E9474A0688163FB662760F970E08BEAA3
:1045700093E20E9468A068816295617070E087EBA9
:1045800093E20E9474A068816695617070E087EA8A
:1045900093E20E9468A0688162FB662760F970E080
:1045A00087EB93E2DF91CF910C9474A0FF920F936D
:1045B0001F93CF93DF9300D01F921F92CDB7DEB72A
:1045C00085E0E1E5F3E0DE01119601900D928A9518
:1045D000E1F7989A9A9A8091070180628093070187
:1045E00080910701806180930701809107018460B9
:1045F000809307018E010F5F1F4FF12CF80161912D
:104600008F018F2D59DFF394F5E0FF12F7CF0F9054
:104610000F900F900F900F90DF91CF911F910F91FE
:10462000FF9008950C94D0DA0E94BBDA2091080222
:10463000309109028217930724F490930902809322
:1046400008020895609108027091090280910602A3
:10465000909107026817790744F4709307026093FA
:10466000060282E594E20C9474A00895CF93C82FBB
:1046700069E170E080E99DE10F94CC006C2F80E946
:104680009DE10F946D0060E080E99DE10F94CD0005
:10469000882329F082E59DE0CF910C948F9FCF91E4
:1046A0000895CF93DF93D82FC62F69E170E080E99A
:1046B0009DE10F94CC006D2F80E99DE10F946D007A
:1046C0006C2F80E99DE10F946D0080E99DE10F94CE
:1046D000DF00882331F082E39DE0DF91CF910C94DD
:1046E0008F9FDF91CF910895C1DF41E050E069E1F4
:1046F00070E080E99DE10F94C00080E99DE10F9496
:104700001600892B31F080E99DE10F941E0081E0B5
:10471000089583E19DE00E948F9F80E008958EEED2
:104720009CE00E948F9F80E99DE10F94AB008FE099
:10473000DBDF81E3D9DF80E2D7DF6CE980E2B1DF44
:1047400080E2D2DF82E2D0DF60E482E2AADF82E2AE
:10475000CBDF85E2C9DF60E085E2A3DF85E2C4DF6D
:1047600083E2C2DF60E383E29CDF83E2BDDF84E2B9
:10477000BBDF6AE484E295DF84E2B6DF80E3B4DF86
:1047800060E280E38EDF80E3AFDF81E3ADDF82E3D1
:10479000ABDF64E182E385DF82E3A6DF83E3A4DFAE
:1047A00060E083E37EDF83E39FDF84E39DDF60E0FF
:1047B00084E377DF84E398DF86E396DF62E386E3D2
:1047C00070DF86E391DF87E38FDF60E087E369DFF7
:1047D00087E38ADF88E388DF60E188E362DF88E3DC
:1047E00083DF89E381DF8AE37FDF62E38AE359DFE6
:1047F0008AE37ACFCF9381E377DFC82F85E374DF35
:10480000811101C0C0E089E36FDF811101C0C0E008
:104810008DE26ADF811101C0C0E08C2FCF91089535
:104820006DE08AE39BE00E946FD96AE08AE39BE037
:104830000C946FD9CF93C82FE0919003F09191031E
:1048400042A953A964A975A922E08CE394E20E94CD
:10485000CBA1E0919003F091910346A957A960ADD7
:1048600071AD20E083E294E20E94CBA10E94B1519D
:10487000AB01BC0122E088E394E20E94CBA140910D
:10488000190250911A0260911B0270911C0220E0E3
:1048900083E294E20E94CBA1CC2391F061E070E02E
:1048A0008AE294E20E9468A06CEF7FE0809111029E
:1048B00090911202681B790B88E294E20E9468A032
:1048C000E0910E02F0E0EE57F24E608170E08FE270
:1048D00094E20E9468A0E091DE02EF3F29F4E091AB
:1048E0009003F0919103E081F0E0EE57F24E608189
:1048F00070E084E394E20E9468A0CF9191CF2F9260
:104900003F924F925F926F927F928F929F92AF925F
:10491000BF92CF92DF92EF92FF920F931F93CF93AC
:10492000DF93CDB7DEB729970FB6F894DEBF0FBE81
:10493000CDBF5C01DC0116968D919C9117978C3848
:10494000910509F469C608F0DBC08235910509F4C8
:104950000EC408F07EC08A31910509F4C5C208F082
:104960003FC08531910509F43DC278F4823191054B
:1049700009F417C28431910509F418C2419711F066
:104980000C94613517981698AFC58731910509F4D5
:1049900061C208F443C28831910509F489C249977C
:1049A00011F00C94613560E082E299E029960FB62F
:1049B000F894DEBF0FBECDBFDF91CF911F910F9155
:1049C000FF90EF90DF90CF90BF90AF909F908F902F
:1049D0007F906F905F904F903F902F900C94489BEA
:1049E0008E31910509F4DDC218F58C31910509F479
:1049F000B0C210F00C949A3582E299E029960FB675
:104A0000F894DEBF0FBECDBFDF91CF911F910F9104
:104A1000FF90EF90DF90CF90BF90AF909F908F90DE
:104A20007F906F905F904F903F902F900C948F9E4F
:104A30008A32910509F40FC328F4809709F4DEC285
:104A40000C9461358035910510F00C949A350C94D6
:104A500061358B36910511F40C948F2E38F58C3519
:104A6000910509F48FC460F48435910509F488C375
:104A700008F481C38535910509F460C40C9461354F
:104A80008836910509F433C530F48336910509F46D
:104A9000DDC40C9461358936910509F410C68A3657
:104AA000910511F40C947E2E0C9461358337910599
:104AB00011F40C94E02E80F48F36910511F40C94CF
:104AC000B02E8237910511F40C94FE2E8D3691058F
:104AD00011F00C94613515C68537910511F40C94CD
:104AE000012F10F40C94082E8737910511F40C94C3
:104AF0002C2F8837910511F40C94732F0C94613589
:104B00008530B1E09B0711F40C94813208F0B0C0FD
:104B10008F3C910511F40C941B3108F041C08A3C84
:104B2000910511F40C944A3070F4883C910511F40D
:104B30000C94992F10F00C94EC2F8E3B910509F4F6
:104B4000B6C70C9461358C3C910511F40C94A130DE
:104B500010F40C948F308D3C910511F40C940131BC
:104B60008E3C910511F00C946135C50129960FB664
:104B7000F894DEBF0FBECDBFDF91CF911F910F9193
:104B8000FF90EF90DF90CF90BF90AF909F908F906D
:104B90007F906F905F904F903F902F900C94D8D55E
:104BA0008F3D910511F40C94D63188F48C3D91051C
:104BB00011F40C9483318D3D910511F40C94AB31BB
:104BC000813D910511F00C9461350C946331893E5F
:104BD000910511F40C94EB3140F5883E910511F0EC
:104BE0000C94613560918A1D70918B1D83E593E271
:104BF0000E9468A04091861D5091871D6091881D7C
:104C00007091891D22E08AE493E20E948EA11092A5
:104C10008B1D10928A1D1092861D1092871D109276
:104C2000881D1092891D0C949A358B3F910511F4C3
:104C30000C9424328430914011F00C946135299603
:104C40000FB6F894DEBF0FBECDBFDF91CF911F919D
:104C50000F91FF90EF90DF90CF90BF90AF909F901B
:104C60008F907F906F905F904F903F902F9057CD97
:104C70008E3521E0920711F40C94D933C0F58E32B1
:104C800041E0940711F40C94243398F48931A1E0A5
:104C90009A0711F40C94D9328C32B1E09B0711F4CD
:104CA0000C94E9328630914011F00C9461350C94EB
:104CB000A3328034F1E09F0711F40C94973338F459
:104CC0008F32914011F40C9463330C94613581342C
:104CD00041E0940711F40C949B338234914011F01D
:104CE0000C94613580E00E940C8C0C94B0338239B6
:104CF000A1E09A0711F40C94C43498F58836E1E0E9
:104D00009E0711F40C94903438F48336914011F4DA
:104D10000C944A340C946135803931E0930711F4D6
:104D20000C94AA348139914011F00C946135299684
:104D30000FB6F894DEBF0FBECDBFDF91CF911F91AC
:104D40000F91FF90EF90DF90CF90BF90AF909F902A
:104D50008F907F906F905F904F903F902F900C942A
:104D60008686853F51E0950711F40C94F43460F485
:104D7000843F914011F00C94613580E00E944ECF49
:104D80008CEB9EE10C94FF34863FE1E09E0711F42A
:104D90000C9419358C38934011F40C9433350C94E1
:104DA00061350E945E1D0E94601D77C282E299E01B
:104DB00029960FB6F894DEBF0FBECDBFDF91CF911D
:104DC0001F910F91FF90EF90DF90CF90BF90AF9029
:104DD0009F908F907F906F905F904F903F902F901B
:104DE0000C94D89D82E299E029960FB6F894DEBF24
:104DF0000FBECDBFDF91CF911F910F91FF90EF902C
:104E0000DF90CF90BF90AF909F908F907F906F90EA
:104E10005F904F903F902F900C94CD9A82E299E052
:104E200029960FB6F894DEBF0FBECDBFDF91CF91AC
:104E30001F910F91FF90EF90DF90CF90BF90AF90B8
:104E40009F908F907F906F905F904F903F902F90AA
:104E50000C94D29AD5018D919C9197FD02C00C942F
:104E60009A3560E082E299E00E942567F501EE5AEA
:104E7000FF4F6081718140E082E299E029960FB690
:104E8000F894DEBF0FBECDBFDF91CF911F910F9180
:104E9000FF90EF90DF90CF90BF90AF909F908F905A
:104EA0007F906F905F904F903F902F900C94099E51
:104EB00082E299E029960FB6F894DEBF0FBECDBF0F
:104EC000DF91CF911F910F91FF90EF90DF90CF90E6
:104ED000BF90AF909F908F907F906F905F904F901A
:104EE0003F902F900C94379BF5018081918192FD2A
:104EF00002C00C949A35468D578D60A171A18091A6
:104F00008C09882311F40C949A35409383095093AB
:104F10008409609385097093860982E699E0299651
:104F20000FB6F894DEBF0FBECDBFDF91CF911F91BA
:104F30000F91FF90EF90DF90CF90BF90AF909F9038
:104F40008F907F906F905F904F903F902F900C9438
:104F50006B65D5018D919C9197FD02C00C949A359B
:104F6000F501EE5AFF4F6081718182E299E0299646
:104F70000FB6F894DEBF0FBECDBFDF91CF911F916A
:104F80000F91FF90EF90DF90CF90BF90AF909F90E8
:104F90008F907F906F905F904F903F902F900C94E8
:104FA000B09EF5018081918197FD02C00C949A35E5
:104FB00060E082E299E00E942567F501EE5AFF4F1A
:104FC0006081718182E299E029960FB6F894DEBF84
:104FD0000FBECDBFDF91CF911F910F91FF90EF904A
:104FE000DF90CF90BF90AF909F908F907F906F9009
:104FF0005F904F903F902F900C94129FD5018D9110
:105000009C9197FD02C00C949A3560E082E299E091
:105010000E942567F501EE5AFF4F6081718182E29F
:1050200099E029960FB6F894DEBF0FBECDBFDF9191
:10503000CF911F910F91FF90EF90DF90CF90BF9095
:10504000AF909F908F907F906F905F904F903F9028
:105050002F900C94409FF5012081318133FD02C0D7
:105060000C949A3512A1E12EF3A0E1E7FDE0449102
:1050700050E04E155F0509F45EC032964DE0E53E06
:10508000F407A9F7F7FC57C032FF2CC0D5015E9694
:105090004D915D916D917C9191974F3F51056105C7
:1050A000710509F0E0F461E0812F0F941005F5011E
:1050B000668D812F0F944905D5015E966D917C9187
:1050C0005F97812F0F94EE02B7018DE893E20E9463
:1050D00068A0F501668D778D88E893E212C08FE0B5
:1050E00095E02BC062E0812F0F941005B70188E88E
:1050F00093E20E9468A0812F0F947E05BC0183E893
:1051000093E229960FB6F894DEBF0FBECDBFDF91B4
:10511000CF911F910F91FF90EF90DF90CF90BF90B4
:10512000AF909F908F907F906F905F904F903F9047
:105130002F900C9474A089ED94E029960FB6F89402
:10514000DEBF0FBECDBFDF91CF911F910F91FF90BA
:10515000EF90DF90CF90BF90AF909F908F907F9017
:105160006F905F904F903F902F900C94B09F109253
:105170000D080C949A3581E080930D080C949A35B3
:10518000D5018D919C91119792FF14C05E962D913F
:105190003D914D915C919197A8EEB3E00F94D60D9F
:1051A00060933E0370933F038093400390934103C9
:1051B0000C949A3593FFA5C0F50182A193A1A4A1F7
:1051C000B5A182309105A105B10509F466C02CF5A1
:1051D0000097A105B10509F446C00197A105B105E5
:1051E00011F00C949A3529960FB6F894DEBF0FBED5
:1051F000CDBFDF91CF911F910F91FF90EF90DF9086
:10520000CF90BF90AF909F908F907F906F905F9066
:105210004F903F902F900C94601D83309105A10515
:10522000B10509F454C00497A105B10511F00C941F
:105230009A3529960FB6F894DEBF0FBECDBFDF9129
:10524000CF911F910F91FF90EF90DF90CF90BF9083
:10525000AF909F908F907F906F905F904F903F9016
:105260002F900C94C85129960FB6F894DEBF0FBE4C
:10527000CDBFDF91CF911F910F91FF90EF90DF9005
:10528000CF90BF90AF909F908F907F906F905F90E6
:105290004F903F902F900C945E1D29960FB6F89476
:1052A000DEBF0FBECDBFDF91CF911F910F91FF9059
:1052B000EF90DF90CF90BF90AF909F908F907F90B6
:1052C0006F905F904F903F902F900C94621D2996A5
:1052D0000FB6F894DEBF0FBECDBFDF91CF911F9107
:1052E0000F91FF90EF90DF90CF90BF90AF909F9085
:1052F0008F907F906F905F904F903F902F900C9485
:10530000BA510E94371E81E029960FB6F894DEBF8D
:105310000FBECDBFDF91CF911F910F91FF90EF9006
:10532000DF90CF90BF90AF909F908F907F906F90C5
:105330005F904F903F902F900C946F74D5018D919A
:105340009C91119792FF14C05E962D913D914D91C5
:105350005C919197A8EEB3E00F94D60D6093420351
:105360007093430380934403909345030C949A35C0
:10537000109242031092430310924403109245038B
:105380000C949A35F501808183FF0CC0828593854A
:10539000A485B5858093270390932803A0932903C0
:1053A000B0932A03D5018C9184FF0EC01E968D9177
:1053B0009D910D90BC91A02D80932B0390932C0375
:1053C000A0932D03B0932E03F501808185FF0CC0BF
:1053D00082899389A489B58980932F0390933003A0
:1053E000A0933103B09332030E94DB74D5018C91FA
:1053F00086FD02C00C949A35209190033091910360
:1054000056968D919D910D90BC91A02DF9018187AB
:105410009287A387B487808129960FB6F894DEBF60
:105420000FBECDBFDF91CF911F910F91FF90EF90F5
:10543000DF90CF90BF90AF909F908F907F906F90B4
:105440005F904F903F902F900C94F74FD501ED91C6
:10545000FC911197F2FF0DC05E962D913D914D91FB
:105460005C919197A8EEB3E00F94D60D6B017C018F
:1054700006C040E1C42E47E2D42EE12CF12CE3FD1E
:105480000E945E1DF501808184FD0E94601DD50192
:105490008C9185FD0E94621D0F94FC032B013C0141
:1054A0004C0C5D1C6E1C7F1C0F94FC03A30192012D
:1054B000261B370B480B590BDA01C901803A964875
:1054C000A140B10518F40E94D179EECFD5018C919D
:1054D00083FD1798F501808184FD1698D5018C9184
:1054E00085FD02C00C949A3515980C949A350E944B
:1054F000DE5981110C949A350F94FC0360938C1D36
:1055000070938D1D80938E1D90938F1D0E94581D4A
:1055100081110C949A35F5018081918193FF02C02D
:105520000C94843592FF0AC0868D978DA0A1B1A1FD
:10553000892B8A2B8B2B11F40C948435D5018D91FA
:105540009C91119792FD02C00C949A359C012227E0
:10555000317091FF23C0232B89F011E020E030E06F
:10556000A9015A966D917D918D919C915D970F94B3
:10557000F90B18160CF010E0212F01C020E0850176
:105580000C5A1F4FF501668D778D80A191A1298757
:105590000F94980A2985D8014C9124C0232B81F0BF
:1055A00011E020E030E0A901F501628D738D848D5A
:1055B000958D0F94F90B18160CF010E0212F01C0F7
:1055C00020E00091900310919103D5015E966D91BA
:1055D0007D918D919C91919729870F94980A2985A7
:1055E000F801408129960FB6F894DEBF0FBECDBFFB
:1055F000DF91CF911F910F91FF90EF90DF90CF90AF
:10560000BF90AF909F908F907F906F905F904F90E2
:105610003F902F900C942E550E94DE5981110C94CE
:105620009A350F94FC0360938C1D70938D1D8093AD
:105630008E1D90938F1D0E94581D81110C949A35D8
:10564000D5018D919C91119792FD02C00C949A35D1
:1056500090FF11C011E020E030E0A9015A966D9151
:105660007D918D919C915D970F94F90B18160CF01C
:1056700010E0412F01C040E0F501668D778D80A1DB
:1056800091A149870F94980A498529960FB6F894F5
:10569000DEBF0FBECDBFDF91CF911F910F91FF9065
:1056A000EF90DF90CF90BF90AF909F908F907F90C2
:1056B0006F905F904F903F902F900C94F755D501CD
:1056C0008D919C9133E0969587953A95E1F781709D
:1056D00029960FB6F894DEBF0FBECDBFDF91CF91F4
:1056E0001F910F91FF90EF90DF90CF90BF90AF9000
:1056F0009F908F907F906F905F904F903F902F90F2
:1057000099C80E94DE5981110C949A350F94FC03BC
:1057100060938C1D70938D1D80938E1D90938F1DB3
:105720000E94581D81110C949A3540E068EC74E099
:1057300086E79AE00E9499AB86E79AE00E94EDAE78
:105740000E94371E2090900330909103F5018081D4
:10575000918191FF09C0EC5AFF4F2081211104C0B3
:105760002BE5222E22E0322E92FF1EC090FF0FC0AA
:1057700011E020E030E0A901D5015A966D917D91AC
:105780008D919C915D970F94F90B18160CF010E019
:10579000F501668D778D80A191A10F94980A212F34
:1057A000D1014C910E942E55F10126A937A940AD97
:1057B00051AD62A973A984A995A90F9460092B0121
:1057C0003C0120E030E0A9010F94F90B181664F4B5
:1057D00020E030E040EA50E4C301B2010F94C50973
:1057E00087FF0EC00C949A3520E030E040EA50EC80
:1057F000C301B2010F94F90B181614F40C949A35E6
:1058000099249394D101D0962D913C91D1979E9655
:105810008D919C919F97821793070CF0912C0F9478
:10582000FC036D837E838F83988710E0412C512C7D
:1058300032010F94FC0369837A838B839C8360938A
:105840008C1D70938D1D80938E1D90938F1DDC0198
:10585000CB012D813E814F815885821B930BA40B78
:10586000B50B893E9340A105B10558F080E00E9438
:105870001A2489819A81AB81BC818D839E83AF83F9
:10588000B88781E00E94151E80919003909191034A
:105890002816390609F064C0D1019396ED90FC906A
:1058A00094971E141F040CF05BC0111158C099206E
:1058B00009F477C091966D917C919297882777FD36
:1058C0008095982F0F94980A9B01AC01F10162A971
:1058D00073A984A995A90F94F90B181614F00C94C8
:1058E0009135662777276E197F09882777FD809580
:1058F000982F0F94980A20913303309134034091EC
:105900003503509136030F946D0C0F94650A1F9266
:105910001F92D10152962C9152972F9351962C9110
:1059200051972F9350962C9150972F931F962C910F
:105930002F935B016C01E12CF12C870120E030E01A
:10594000A90160E070E0CB010E941FF80F900F905A
:105950000F900F900F900F9011E00C94913511E083
:10596000411451046104710409F050C09920F1F010
:1059700020E030E040E85FE3F10166A977A980AD5F
:1059800091AD0F9460099B01AC01D101D2966D914C
:105990007D918D919C91D5970F94F90B87FF1FC036
:1059A00045CF411451046104710481F520E030E0D9
:1059B00040E85FE3F10166A977A980AD91AD0F944E
:1059C00061099B01AC01D101D2966D917D918D91C0
:1059D0009C91D5970F94C50918160CF427CFF101A7
:1059E000A78DB0A128EE33E00F94D00D2B013C0120
:1059F00029813A814B815C81420E531E641E751EC3
:105A0000411451046104710409F413CFD301C2019C
:105A100029813A814B815C81821B930BA40BB50BCE
:105A200081159449A543B74708F403CF112309F41E
:105A3000E2C080919003909191032816390609F0F5
:105A4000DAC0D10193966D917C919497882777FD68
:105A50008095982F0F94980A209133033091340346
:105A600040913503509136030F946D0C0F94650AE5
:105A70001F921F92F10122892F9321892F93208950
:105A80002F9327852F935B016C01E12CF12C87016B
:105A900020E030E0A90160E070E0CB010E941FF837
:105AA0000F900F900F900F900F900F90A4C00E9436
:105AB000581D81110C949A3540E06CEB74E086E738
:105AC0009AE00E9499AB86E79AE00E94EDAE0E94B0
:105AD000371ED5018D919C91119792FF1FC090FFA9
:105AE00011C011E020E030E0A9015A966D917D913E
:105AF0008D919C915D970F94F90B18160CF010E0A6
:105B0000412F01C040E0F501668D778D80A191A104
:105B100049870F94980A49850E94F75520911902E8
:105B200030911A0240911B0250911C0260911502A3
:105B30007091160280911702909118020F946009DB
:105B40002B013C0120E030E0A9010F94F90B18165D
:105B50005CF420E030E040EA50E4C301B2010F946D
:105B6000C50987FF0CC0E6C720E030E040EA50ECF2
:105B7000C301B2010F94F90B18160CF4DBC70F9494
:105B8000FC032B013C0120E030E040E05FE360914A
:105B900015027091160280911702909118020F94CD
:105BA00061092091190230911A0240911B02509113
:105BB0001C020F94C50987FF1EC00F94FC036419D3
:105BC000750986099709693E73408105910578F04A
:105BD00080E00E941A240F94FC032B013C01609387
:105BE0008C1D70938D1D80938E1D90938F1D81E071
:105BF0000E94151EC8CF1092DF0A0F94FC03609319
:105C00008C1D70938D1D80938E1D90938F1D92C758
:105C10000E94581D81118EC70F94FC032B013C017B
:105C20000F94FC036419750986099709693E73404E
:105C30008105910538F080E00E941A240F94FC033E
:105C40002B013C0181E00E94151E00910A02109177
:105C50000B02D8011B968D909D90AD90BC901E9725
:105C600020E030E040EF51E4C501B4010F94F90B9E
:105C70001816BCF4F8012781308541855285C5018D
:105C8000B4010F9460099F7701E020E030E040E824
:105C90005FE30F94F90B18160CF000E011E01027E9
:105CA00001C011E0E0900C02F0900D02D7011B96AC
:105CB0008D909D90AD90BC901E9720E030E040EF1D
:105CC00051E4C501B4010F94F90B18169CF4F701C7
:105CD0002781308541855285C501B4010F94600943
:105CE0009F7720E030E040E85FE30F94F90B18164F
:105CF0000CF496CF112309F493CF1CC7D5018D91D5
:105D00009C91119793FB662760F992FF05C05E9600
:105D10008D919C915F970AC08FEF90E007C0F501CD
:105D2000618163FB662760F980E090E029960FB6F9
:105D3000F894DEBF0FBECDBFDF91CF911F910F91C1
:105D4000FF90EF90DF90CF90BF90AF909F908F909B
:105D50007F906F905F904F903F902F900C94902089
:105D6000D5018D919C91119792FF04C05E962C9164
:105D70002093EA0293FF12C0F50182A193A1A4A18E
:105D8000B5A12091EA02181619061A061B0614F48A
:105D9000822B02C0815082238093EA020E94581D08
:105DA000882309F4C7C620E040E060E070E0CB0142
:105DB0000E942E5520E040E060E070E0CB0112CC64
:105DC00088E695E20E948F9F29960FB6F894DEBF71
:105DD0000FBECDBFDF91CF911F910F91FF90EF903C
:105DE000DF90CF90BF90AF909F908F907F906F90FB
:105DF0005F904F903F902F900C94BA2086EB94E0E8
:105E000066C3D5018D919C9197FF94C6F501EE5A1A
:105E1000FF4F6081718140E086E79AE00E9412ACFA
:105E200086E79AE029960FB6F894DEBF0FBECDBF85
:105E3000DF91CF911F910F91FF90EF90DF90CF9066
:105E4000BF90AF909F908F907F906F905F904F909A
:105E50003F902F900C94EDAE0E94371E86E793E2A0
:105E60000E94769F0E94641D882319F080E893E2C7
:105E700002C08DE793E20E94769F8FE693E20E9434
:105E8000769F0E94691D882319F080E893E202C082
:105E90008DE793E20E94769F88E693E20E94769FC8
:105EA000379903C08DE793E202C080E893E20E9435
:105EB000769F29960FB6F894DEBF0FBECDBFDF9157
:105EC000CF911F910F91FF90EF90DF90CF90BF90F7
:105ED000AF909F908F907F906F905F904F903F908A
:105EE0002F900C941024F5018081918188279C705B
:105EF00081159C4009F01EC6F50162A1868D299688
:105F00000FB6F894DEBF0FBECDBFDF91CF911F91CA
:105F10000F91FF90EF90DF90CF90BF90AF909F9048
:105F20008F907F906F905F904F903F902F900C9448
:105F300097A2E0919003F09191032081D5018D917A
:105F40009C9191FF06C0F501EC5AFF4F8081882398
:105F500011F0822F01C080E0F501928192FF05C00F
:105F600046A457A460A871A803C0412C512C32014B
:105F700093FF07C0D501D2964D905D906D907C90B7
:105F8000D597082F10E0B3E88B9FF0011124E7525A
:105F9000FD4F4082518262827382821306C08091DB
:105FA000FF06909100070E94182020E030E0A90130
:105FB000C301B2010F94C509B801811103C08AE879
:105FC00094E09FC883E694E00E9468A022E0B301B9
:105FD000A2018EE594E05DC1F501808183FF0CC0D4
:105FE00082859385A485B5858093FB029093FC02FE
:105FF000A093FD02B093FE02D5018C9184FF0EC0E8
:106000001E968D919D910D90BC91A02D8093FF02C5
:1060100090930003A0930103B0930203F5018081E4
:1060200085FF0CC082899389A489B5898093030375
:1060300090930403A0930503B0930603D5018C91BC
:1060400086FF0EC056968D919D910D90BC91A02D0E
:106050008093070390930803A0930903B0930A0366
:1060600029960FB6F894DEBF0FBECDBFDF91CF915A
:106070001F910F91FF90EF90DF90CF90BF90AF9066
:106080009F908F907F906F905F904F903F902F9058
:106090000C94DB74F501808183FF0CC082859385AD
:1060A000A485B5858093EB029093EC02A093ED025A
:1060B000B093EE02D5018C9184FF0EC01E968D9197
:1060C0009D910D90BC91A02D8093EF029093F002D2
:1060D000A093F102B093F202F501808185FF0CC01C
:1060E00082899389A489B5898093F3029093F402FD
:1060F000A093F502B093F602D5018C9186FFB0CF44
:1061000056968D919D910D90BC91A02D8093F70294
:106110009093F802A093F902B093FA02A1CFF5018F
:106120008081918192FF06C5868D978DA0A1B1A136
:10613000181619061A061B060CF481E08093E0027B
:10614000F9C4E0919003F0919103BB96D5012D9194
:106150003C91119732FF11C05E968D919D910D90EB
:10616000BC91A02DB7FDE6C4892B8A2B8B2B19F08F
:10617000EEE0F2E002C0E6E8F2E023FF0BC0D5015A
:106180001A964D915D916D917C911D97428F538F21
:10619000648F758FD5018C9184FF0AC01E964D9136
:1061A0005D916D917C915197468F578F60A371A33C
:1061B000D5018C9185FF0AC052964D915D916D91EC
:1061C0007C91559742A353A364A375A3CF0129964D
:1061D0000FB6F894DEBF0FBECDBFDF91CF911F91F8
:1061E0000F91FF90EF90DF90CF90BF90AF909F9076
:1061F0008F907F906F905F904F903F902F900C9476
:10620000294F29960FB6F894DEBF0FBECDBFDF91A0
:10621000CF911F910F91FF90EF90DF90CF90BF90A3
:10622000AF909F908F907F906F905F904F903F9036
:106230002F900C9485D7F501208123FF0CC0828517
:106240009385A485B5858093FB069093FC06A09367
:10625000FD06B093FE0626FF11C0209190033091F9
:106260009103F50186899789A08DB18DF901878BFE
:10627000908FA18FB28F80810E94F74F4091FB06D3
:106280005091FC066091FD067091FE0622E082E6C8
:1062900093E229960FB6F894DEBF0FBECDBFDF9113
:1062A000CF911F910F91FF90EF90DF90CF90BF9013
:1062B000AF909F908F907F906F905F904F903F90A6
:1062C0002F900C948EA1D5018D919C91119792FFE6
:1062D00031C461E05E968D919D910D90BC91A02D91
:1062E0002091C607892B8A2B8B2B21F460E0822F0B
:1062F0008D7F02C0822F82608093C60770E085EC9C
:1063000093E00C948128F5018081918192FF05C072
:10631000868D978DA0A1B1A104C084E690E0A0E095
:10632000B0E029960FB6F894DEBF0FBECDBFDF9167
:10633000CF911F910F91FF90EF90DF90CF90BF9082
:10634000AF909F908F907F906F905F904F903F9015
:106350002F900C94911FD5018D919C91119792FFD4
:1063600007C05E968D919D910D90BC91A02D04C0AB
:1063700084E690E0A0E0B0E029960FB6F894DEBF86
:106380000FBECDBFDF91CF911F910F91FF90EF9086
:10639000DF90CF90BF90AF909F908F907F906F9045
:1063A0005F904F903F902F900C941820F5018081C2
:1063B000918192FFBFC34FB7F8948091520890919A
:1063C0005308268D378D820F931F90935308809327
:1063D00052084FBFAFC3F5018081209190033091E7
:1063E000910384FF09C086859785A089B189F90149
:1063F00085A396A3A7A3B0A7D90195964D915D91CA
:106400006D917C91989722E081E393E20E94CBA169
:106410000E94102429960FB6F894DEBF0FBECDBFA0
:10642000DF91CF911F910F91FF90EF90DF90CF9070
:10643000BF90AF909F908F907F906F905F904F90A4
:106440003F902F900C94C1742091F9073091FA0776
:106450004091FB075091FC0760910B0770910C076E
:1064600080910D0790910E070F94600960930B07C0
:1064700070930C0780930D0790930E0710920508F8
:106480001092060810920708109208080E94DB7408
:1064900061E178E08DEF97E00E940BED80E00E94D3
:1064A000E38040910B0750910C0760910D077091AC
:1064B0000E0722E086EC9FE10E948EA180E00E9400
:1064C0004ECF8BE393E20E948F9F88E594E029965C
:1064D0000FB6F894DEBF0FBECDBFDF91CF911F91F5
:1064E0000F91FF90EF90DF90CF90BF90AF909F9073
:1064F0008F907F906F905F904F903F902F900C9473
:10650000451E84E00F947E05BC018EE494E00E9459
:1065100074A029960FB6F894DEBF0FBECDBFDF91F1
:10652000CF911F910F91FF90EF90DF90CF90BF9090
:10653000AF909F908F907F906F905F904F903F9023
:106540002F900C94FA2382E30E947423F50180813A
:10655000918192FFEFC2468D578D60A171A188E3B2
:1065600094E00E94B2A0D5015E966C9182E30E94F5
:106570005123F501668D8AE30E94512382E3299617
:106580000FB6F894DEBF0FBECDBFDF91CF911F9144
:106590000F91FF90EF90DF90CF90BF90AF909F90C2
:1065A0008F907F906F905F904F903F902F900C94C2
:1065B00074238DEF93E00E94A69F80E00E946F7489
:1065C00068EC70E080E090E00F942B048FB7F894B3
:1065D000FFCFD5018D919C91119792FF05C05E96DA
:1065E0006D917C915F9702C061E070E093FF04C001
:1065F000F50102A113A102C008EE13E020E030E093
:10660000A9018FE40F94CE05B80180E090E00F94CB
:106610002B048FE429960FB6F894DEBF0FBECDBFD2
:10662000DF91CF911F910F91FF90EF90DF90CF906E
:10663000BF90AF909F908F907F906F905F904F90A2
:106640003F902F900D94DF08D5018D919C9111976B
:1066500092FF0EC021E05E968D919D910D90BC91B0
:10666000A02D892B8A2B8B2B09F420E0822F01C0CF
:1066700081E09091C707882311F0906801C09F774F
:106680009093C707882319F08EEA93E002C084E94B
:1066900093E029960FB6F894DEBF0FBECDBFDF9111
:1066A000CF911F910F91FF90EF90DF90CF90BF900F
:1066B000AF909F908F907F906F905F904F903F90A2
:1066C0002F900C948F9FF5010081118112FF03C060
:1066D000668D778D02C066E970E013FF0DC0D501AD
:1066E0009296ED90FC909397B2E0EB16F10434F0A3
:1066F00082E0E82EF12C02C0E12CF12CA3E01695EB
:106700000795AA95E1F70170882777FD8095982F66
:106710000F94980AAB01BC01F701EE0FFF1FE65F73
:10672000FD4F2E2D808191810E94785603C281E019
:106730000E94BA8715C080E00E94BA87D5018D916A
:106740009C91119792FFF6C15E968D919D910D904F
:10675000BC91A02D0097A105B10509F0D9C1EAC1EE
:10676000F5018081918192FFE5C1868D978DA0A171
:10677000B1A1892B8A2B8B2B09F4DCC180E02996EF
:106780000FB6F894DEBF0FBECDBFDF91CF911F9142
:106790000F91FF90EF90DF90CF90BF90AF909F90C0
:1067A0008F907F906F905F904F903F902F900C94C0
:1067B0004ECF8BEE93E00E948F9FD5018D919C91DF
:1067C00092FD0FC0F501808183FF16C0F50162853F
:1067D0007385848595850F946A0A80E00E945C2207
:1067E0000BC010E0D5015E966C91812F0E945C2257
:1067F0001F5F1530B9F7E6CFD5018C9184FF0BC030
:106800001E966D917D918D919C9151970F946A0A7E
:1068100081E00E945C22F501808185FF09C06289C8
:106820007389848995890F946A0A82E00E945C22A8
:10683000D5018C9186FF0BC056966D917D918D91FF
:106840009C9159970F946A0A83E00E945C22F5019B
:106850008081918193FF04C062A184E00E945C2248
:1068600029960FB6F894DEBF0FBECDBFDF91CF9152
:106870001F910F91FF90EF90DF90CF90BF90AF905E
:106880009F908F907F906F905F904F903F902F9050
:106890000C947322D5018D919C91119792FF26C083
:1068A00081E05E964D915D916D917C919197452B24
:1068B000462B472B09F480E029960FB6F894DEBFEB
:1068C0000FBECDBFDF91CF911F910F91FF90EF9041
:1068D000DF90CF90BF90AF909F908F907F906F9000
:1068E0005F904F903F902F900C94359029960FB663
:1068F000F894DEBF0FBECDBFDF91CF911F910F91F6
:10690000FF90EF90DF90CF90BF90AF909F908F90CF
:106910007F906F905F904F903F902F900C943690A7
:1069200029960FB6F894DEBF0FBECDBFDF91CF9191
:106930001F910F91FF90EF90DF90CF90BF90AF909D
:106940009F908F907F906F905F904F903F902F908F
:106950000C94449029960FB6F894DEBF0FBECDBFBD
:10696000DF91CF911F910F91FF90EF90DF90CF902B
:10697000BF90AF909F908F907F906F905F904F905F
:106980003F902F900C94371EF5018081918190FFEC
:1069900005C0E28CF38C048D158D08C0E0900307D0
:1069A000F090040700910507109106079C0146E04E
:1069B000369527954A95E1F72170AC0165E056952B
:1069C00047956A95E1F74170BC01E4E076956795DB
:1069D000EA95E1F76170F3E096958795FA95E1F70E
:1069E00081700E94E786A6C00E94ABD1E09190031F
:1069F000F091910380810E94F74F8AE99EE12996E8
:106A00000FB6F894DEBF0FBECDBFDF91CF911F91BF
:106A10000F91FF90EF90DF90CF90BF90AF909F903D
:106A20008F907F906F905F904F903F902F900C943D
:106A3000A69F29960FB6F894DEBF0FBECDBFDF919B
:106A4000CF911F910F91FF90EF90DF90CF90BF906B
:106A5000AF909F908F907F906F905F904F903F90FE
:106A60002F900C9453CD82ED93E00E948F9FD5011F
:106A70008D919C9188279C7081159C4009F05AC08B
:106A8000D5015E966D917C915F9792968C91299637
:106A90000FB6F894DEBF0FBECDBFDF91CF911F912F
:106AA0000F91FF90EF90DF90CF90BF90AF909F90AD
:106AB0008F907F906F905F904F903F902F900C94AD
:106AC0008C218091EA0282FF35C08CE594E20E941D
:106AD000769FC50129960FB6F894DEBF0FBECDBFD5
:106AE000DF91CF911F910F91FF90EF90DF90CF90AA
:106AF000BF90AF909F908F907F906F905F904F90DE
:106B00003F902F900C9464970E94371E0C949E2AFD
:106B10000397A105B10509F031CE80E00E940C8CED
:106B20002DCE411451046104710411F40C94B82C5D
:106B30000C94062D29960FB6F894DEBF0FBECDBF7C
:106B4000DF91CF911F910F91FF90EF90DF90CF9049
:106B5000BF90AF909F908F907F906F905F904F907D
:106B60003F902F9008952F923F924F925F926F9295
:106B70007F928F929F92AF92BF92CF92DF92EF92CD
:106B8000FF920F931F93CF93DF93CDB7DEB7EC97B0
:106B90000FB6F894DEBF0FBECDBF1C01DC01189606
:106BA0008D919C9119978032910509F43AC358F55B
:106BB0008531910509F45EC198F48430910509F49A
:106BC0001BC128F4029708F4EBC00C945D44449771
:106BD00011F00C945D4481E0809351080C9468445A
:106BE0008D31910509F499C128F44C9709F446C1F7
:106BF0000C945D448E31910509F4F0C14F9709F46E
:106C0000FFC20C945D448C35910511F40C948740BF
:106C100040F58534910509F463C7B8F484349105CF
:106C200011F00C945D448091030790910407A091AA
:106C30000507B09106078D879E87AF87B88B44E123
:106C4000442E512C612C712C76C58A35910511F496
:106C50000C946C408B35910511F40C9478400C9495
:106C60005D448438910511F40C941E4308F05DC016
:106C70008436910511F40C9469418338910511F023
:106C80000C945D446091F1077091F2078091F307D5
:106C90009091F4072091F5073091F6074091F7079E
:106CA0005091F807E090F907F090FA070091FB0780
:106CB0001091FC074090030750900407609005076F
:106CC000709006071092F7061092F8061092F906D7
:106CD0001092FA061092F3061092F4061092F5063E
:106CE0001092F606E0910E03EF93E0910D03EF93FF
:106CF000E0910C03EF93E0910B03EF93E0EFAE2EE6
:106D0000E3E2BE2EE4E7CE2EE9E4DE2E0E94267EEC
:106D1000409203075092040760920507709206079D
:106D200080E00E94E3800C9419438538910511F4AA
:106D30000C94AD438638910511F00C945D4440915C
:106D4000110850911208609113087091140880EA9C
:106D500095E00E949AA04091150850911608609104
:106D600017087091180887EB93E20E949AA040914F
:106D7000190850911A0860911B0870911C0887EB44
:106D800093E20E94B2A080E00E94E38082E995E055
:106D90000E94769F8CE895E00E94451E0C94684402
:106DA000F1018081918192FF11C0868D978DA0A104
:106DB000B1A12091C707892B8A2B8B2B19F0822F29
:106DC000806202C0822F8F7D8093C707C1010E941D
:106DD0005A82882359F041E061E081E00E94EFF29D
:106DE000811104C082EC9CE00E949C9F61E081E0E4
:106DF0000E94F0EC0C9468440E94371ED1018D91E2
:106E00009C91119793FF07C092968D909D90AD90A5
:106E1000BC90959703C0812C912C540192FF0BC01C
:106E2000F101268D378D40A151A1A8EEB3E00F945A
:106E3000D60D4B015C010F94FC036B017C01C80C67
:106E4000D91CEA1CFB1C0F94FC03A7019601261B0E
:106E5000370B480B590BDA01C90181159449A54339
:106E6000B74710F00C9468440E94579881E00E9444
:106E7000151EE9CF109251080C946844D1018D91F0
:106E80009C91AC01487355274115510551F49C0163
:106E900066E0369527956A95E1F7B1E02B272170DA
:106EA00001C020E086FF08C01092090810920A086D
:106EB00010920B0810920C08211117C0452BD1F02D
:106EC000AC0125E0569547952A95E1F7BC0134E0E1
:106ED000769567953A95E1F753E0969587955A959B
:106EE000E1F761704170817003C061E041E081E0D1
:106EF0000E94D48780E00E94E3800E94641D81117B
:106F00000C948B440E94691D81110C948B44379919
:106F100002C00C9468440C948B440E94FA238111A3
:106F200011C06AEF70E080E090E00F942B040E94A3
:106F3000FA23811107C08EE59CE00E948F9F85E4B3
:106F40009CE05AC180E39CE00E941D9620910307BB
:106F5000309104074091050750910607298F3A8F19
:106F60004B8F5C8F80E090E00E94B51D80E090E048
:106F70000E94D51D80E090E00E94F51D80E00E94F7
:106F80004ECF0E94ABD184E190E0A0E0B0E0898BCD
:106F90009A8BAB8BBC8B86E1482E512C612C712CCB
:106FA0001DA229893A894B895C892D873E874F87A5
:106FB000588B41E061E081E00E94D4870E94641D0B
:106FC00081110C94A8440E94691D81110C94A8445D
:106FD000379902C00C94CC440C94A844D1012D9153
:106FE0003C91119732FD02C00C94D2495E968D916E
:106FF0009D910D90BC91A02D0297A105B10511F0B6
:107000000C94D2490C944B4A81E99BE00E948F9FDB
:1070100089E79BE00E941D9686ED9FE10E94B09F4C
:10702000EDA1E1110C94684481E00E94E380298D78
:107030003A8D4B8D5C8D209303073093040740936A
:1070400005075093060787E39AE00E94451E8EE3EA
:1070500090E20E941D96212C312C8091770790910F
:107060007807A0917907B0917A07898B9A8BAB8BBF
:10707000BC8B80E00E944ECF0E94ABD181E00E9489
:10708000BA8741E061E081E00E94D48780E00E94FD
:10709000BA878FE390E20E941D960E946D1D9F9318
:1070A0008F937F936F93B0EFAB2EB3E2BB2EB4E719
:1070B000CB2EB9E4DB2E8601750120E030E0A9017A
:1070C000CA01B9010E94918520E041E060E081E0C1
:1070D0000E9463886B017C0120E041E060E081E078
:1070E0000E9463884B015C019B01AC01C701B601A2
:1070F0000F9460092B013C010F900F900F900F909F
:107100002DEC3CEC4CEC5DE30F94F90B181614F0ED
:107110000C94E3474D855E856F85788983E09AE01E
:107120000E94B2A02D853E854F85588928323105B1
:107130004105510514F00C94EF4782E30E9474233B
:107140008D859E85AF85B8890296A11DB11D8D875D
:107150009E87AF87B88BAC01BD0185EE99E00E9498
:10716000B2A06D8582E30E9451236D858AE30E945F
:10717000512382E30E947423B4E02B1631040CF4F3
:107180006CCF81E00E94BA8781E00E94E38086EDA7
:1071900098E00E94451E8EE390E20E941D96298D84
:1071A0003A8D4B8D5C8D20930307309304074093F9
:1071B00005075093060741E061E081E00E94D48713
:1071C00080E00E944ECF41E066E573E082E299E004
:1071D0000E94099E882371F082E299E00E94679BD9
:1071E00066E573E082E299E00E94129F82E299E0F4
:1071F0000E949F9A8CEB98E00E941D960C94684424
:107200008CE490E20E94769F959902C068E401C0E8
:107210006CE48AE39BE00E946FD90E9410240C94D6
:1072200068448FE390E20E941D961092D10710925D
:10723000D2071092D3071092D4071092CD07109264
:10724000CE071092CF071092D0071092C907109264
:10725000CA071092CB071092CC0780E00E94BA8731
:1072600020910307309104074091050750910607CC
:1072700029A33AA34BA35CA30E946D1D162F072FD1
:10728000F82EE92E84E393E00E94211D9B01AC01BE
:1072900080E393E029AF3AAF4BAF5CAF0E94211D72
:1072A000EF92FF920F931F9350EFA52E53E2B52E4E
:1072B00054E7C52E59E4D52E8601750129AD3AADA6
:1072C0004BAD5CAD0E94918520E041E060E081E043
:1072D0000E9463882B013C010F900F900F900F903C
:1072E00020E030E0A9010F94C50987FF02C00C948B
:1072F00068440E946D1D162F072FF82EE92E8CE38F
:1073000093E00E94211D9B01AC0188E393E029AF2B
:107310003AAF4BAF5CAF0E94211DEF92FF920F93EB
:107320001F938601750129AD3AAD4BAD5CAD0E944E
:10733000918521E041E060E080E00E9463886D87F4
:107340007E878F87988B0F900F900F900F9020E083
:1073500030E0A9010F94C50987FF02C00C9468446E
:107360000E946D1D162F072FF82EE92E84E493E05E
:107370000E94211D9B01AC0180E493E029AF3AAF4C
:107380004BAF5CAF0E94211DEF92FF920F931F93B2
:107390008601750129AD3AAD4BAD5CAD0E9491857A
:1073A00021E041E061E080E00E9463884B015C01E4
:1073B0000F900F900F900F9020E030E0A9010F94F4
:1073C000C50987FF02C00C946844850174012D85AE
:1073D0003E854F855889C301B2010E94078E809176
:1073E0009D0790919E07A0919F07B091A0078D8760
:1073F0009E87AF87B88B2091B1073091B20740913B
:10740000B3075091B407298B3A8B4B8B5C8BC090A0
:10741000A507D090A607E090A707F090A807809155
:10742000A9079091AA07A091AB07B091AC078D8BEB
:107430009E8BAF8BB88F209101083091020840914C
:107440000308509104082DA33EA34FA358A7809191
:10745000450890914608A0914708B091480889A72F
:107460009AA7ABA7BCA72091AD073091AE0740917A
:10747000AF075091B0072D8F3E8F4F8F58A380914B
:10748000A1079091A207A091A307B091A407898FAB
:107490009A8FAB8FBC8F2091FD073091FE074091F2
:1074A000FF07509100082DA73EA74FA758AB80912A
:1074B000410890914208A0914308B091440889ABDB
:1074C0009AABABABBCAB10920707109208071092B7
:1074D000090710920A07D1018D919C91119792FF93
:1074E000DCC05E968D919D910D90BC91A02DAC015C
:1074F000BD014150510961097109423051056105D1
:10750000710548F00397A105B10509F0C6C080E0F8
:107510000E944ECFC2C029893A894B895C896D850A
:107520007E858F8598890F946D0C2B013C012D89E8
:107530003E894F89588DC701B6010F946D0C9B0190
:10754000AC01C301B2010F9460092B013C016DA194
:107550007EA18FA198A50F94980A9B01AC01C3014D
:10756000B2010F946D0C29A53AA54BA55CA50F940B
:107570006D0C2B013C012D8D3E8D4F8D58A1C70107
:10758000B6010F946D0C6B017C0129893A894B89F6
:107590005C89698D7A8D8B8D9C8D0F946D0C9B0110
:1075A000AC01C701B6010F9460096B017C016DA5A8
:1075B0007EA58FA598A90F94980A9B01AC01C701DD
:1075C000B6010F946D0C29A93AA94BA95CA90F9497
:1075D0006D0C9B01AC01C301B2010F9461096B01F9
:1075E0007C01F7FAF094F7F8F0942D893E894F89E1
:1075F000588D698D7A8D8B8D9C8D0F946D0C2B0120
:107600003C012D8D3E8D4F8D58A16D857E858F85DA
:1076100098890F946D0C9B01AC01C301B2010F94CA
:1076200060099B01AC01C701B6010F94CC099B0115
:10763000AC01C501B4010F9461092091F9073091A3
:10764000FA074091FB075091FC070F9460092091C5
:107650000B0730910C0740910D0750910E070F94C6
:107660006109AB01BC0140930B0750930C07609379
:107670000D0770930E0722E086EC9FE10E948EA119
:1076800081E00E94BA87F101868D978DA0A1B1A1FA
:107690000297A105B10509F43ACF81E00E94BA87AB
:1076A0000E94DB7481E00E94E38084E698E00E94FF
:1076B000451E41E061E081E00E94D48729A13AA102
:1076C0004BA15CA120930307309304074093050767
:1076D000509306070C9468442DEC3CEC4CEC5DEBAD
:1076E000C701B6010F94C50987FF85C0B301A20188
:1076F00084E498E00E94B2A038E243165104610489
:107700007104CCF482E30E94742342E0440E511CC5
:10771000611C711CB301A20186E298E00E94B2A034
:10772000642D82E30E945123642D8AE30E94512339
:1077300082E30E947423209177073091780740916B
:10774000790750917A07298F3A8F4B8F5C8F80E0B1
:107750000E944ECF0E94ABD141E061E081E00E94E7
:10776000D4878FE390E20E941D9680E00E94BA8742
:107770000E946D1D9F938F937F936F9330EFA32E85
:1077800033E2B32E34E7C32E39E4D32E86017501DC
:1077900020E030E0A901CA01B9010E94918520E0F2
:1077A00041E060E081E00E946388698B7A8B8B8B7B
:1077B0009C8B20E041E060E081E00E9463886D8B5B
:1077C0007E8B8F8B988F9B01AC0169897A898B891D
:1077D0009C890F9460096B017C010F900F900F90B2
:1077E0000F902DEC3CEC4CEC5DE30F94F90B18166C
:1077F0000CF072CF7BCF0E946D1D162F072FF82E35
:10780000E92E84E493E00E94211D9B01AC0180E4F9
:1078100093E029AF3AAF4BAF5CAF0E94211DEF92CE
:10782000FF920F931F9320EFA22E23E2B22E24E7A4
:10783000C22E29E4D22E8601750129AD3AAD4BAD99
:107840005CAD0E94918521E041E061E080E00E9412
:1078500063884B015C0121E041E061E080E00E942F
:1078600063886B017C019B01AC01C501B4010F94DD
:1078700060096D8F7E8F8F8F98A30F900F900F9060
:107880000F902DEC3CEC4CEC5DE30F94F90B1816CB
:1078900064F02DEC3CEC4CEC5DEB6D8D7E8D8F8DB2
:1078A00098A10F94C50987FF13C0B301A20186E018
:1078B00098E00E94B2A082E30E94742352E0450E39
:1078C000511C611C711CB301A20188EE97E026CF08
:1078D00029893A894B895C896D897E898F89988D40
:1078E0000F94610920E030E040E05FE30F946D0CFD
:1078F000698B7A8B8B8B9C8B20E030E0A9010F94F5
:10790000C50987FD18CFA5019401C701B6010F94E1
:10791000610920E030E040E05FE30F946D0C9B01D3
:10792000AC0169897A898B899C890F94600920E070
:1079300030E040EA52E40F946D0C6B017C0120E0D2
:1079400030E0A9010F94C50987FF31C0F7FAF09420
:10795000F7F8F09422E0B701A6018AE690E20E94CF
:107960008EA1209177073091780740917907509147
:107970007A07C701B6010F94CC099B01AC010F94A3
:1079800061096B017C0122E0AB01BC018AE690E257
:107990000E948EA1A70196016091770770917807E8
:1079A0008091790790917A070F94600918C08090B0
:1079B000770790907807A0907907B0907A07A50193
:1079C0009401C701B6010F94CC099B01AC010F943F
:1079D00061099B01AC01C501B4010F946109609379
:1079E0007707709378078093790790937A0722EC52
:1079F00035EF41EB52E46091770770917807809101
:107A0000790790917A070F94CC096B017C012DECDA
:107A10003CEC4CE85FE30F94F90B181654F026E6A3
:107A200036E646E65FE3C701B6010F94C50987FF56
:107A300012C082EC95EFA1EBB2E4809377079093AC
:107A40007807A0937907B0937A0722E0AC01BD01D3
:107A50008DEC97E014C022E0498D5A8D6B8D7C8DA2
:107A600080EC97E00E948EA14091770750917807B3
:107A70006091790770917A0722E083EB97E00E948A
:107A80008EA18D859E85AF85B889809303079093DD
:107A90000407A0930507B093060781E00E94BA8708
:107AA00081E00E94E3808EEA97E00E94451E8EE30B
:107AB00090E20E941D962D853E854F855889209322
:107AC000030730930407409305075093060741E0EE
:107AD00061E081E00E94D48780E00E944ECFF8C62A
:107AE0008091030790910407A0910507B0910607C4
:107AF0008D8F9E8FAF8FB8A324E130E040E050E03F
:107B00002D873E874F87588BD1018D919C9111977E
:107B100092FF0CC05E968D919D910D90BC91A02D11
:107B20000297A105B10511F40C94974B41E061E077
:107B300081E00E94D4878FE390E20E941D9680E04E
:107B40000E94BA870E946D1D162F072FF82EE92E6E
:107B500084E393E00E94211D9B01AC0180E393E04C
:107B600029AF3AAF4BAF5CAF0E94211DEF92FF925D
:107B70000F931F9300EFA02E03E2B02E04E7C02E58
:107B800009E4D02E8601750129AD3AAD4BAD5CAD4F
:107B90000E94918520E041E060E081E00E946388DE
:107BA000698F7A8F8B8F9C8F20E041E060E081E0CD
:107BB0000E94638869A37AA38BA39CA39B01AC0159
:107BC000698D7A8D8B8D9C8D0F9460096B017C0182
:107BD0000F900F900F900F902DEC3CEC4CEC5DE370
:107BE0000F94F90B181654F02DEC3CEC4CEC5DEBBB
:107BF000C701B6010F94C50987FF2BC04D855E856F
:107C00006F8578898EE897E00E94B2A02D853E8529
:107C10004F85588928323105410551050CF074CF44
:107C200082E30E947423D1018D919C9192FF6CCFCD
:107C30002D853E854F8558892E5F3F4F4F4F5F4FB3
:107C40002D873E874F87588BBA01A90180E797E0BF
:107C500086C08DE793E00F9444129A8B898B0E9423
:107C60006D1D162F072FF82EE92E8CE393E00E944E
:107C7000211D9B01AC0188E393E029AF3AAF4BAFE4
:107C80005CAF0E94211DEF92FF920F931F9310EFA4
:107C9000A12E13E2B12E14E7C12E19E4D12E8601D4
:107CA000750129AD3AAD4BAD5CAD0E94918521E0E7
:107CB00041E060E080E00E9463886DA37EA38FA313
:107CC00098A721E041E060E080E00E94638869A716
:107CD0007AA78BA79CA79B01AC016DA17EA18FA168
:107CE00098A50F9460096B017C010F900F900F9085
:107CF0000F902DEC3CEC4CEC5DE30F94F90B181657
:107D000054F02DEC3CEC4CEC5DEBC701B6010F944C
:107D1000C50987FF32C04D855E856F85788980E50E
:107D200097E00E94B2A08D859E85AF85B88988971F
:107D3000A105B1050CF0E8CE82E30E9474232D85E5
:107D40003E854F8558892E5F3F4F4F4F5F4F2D87A0
:107D50003E874F87588BBA01A90182E397E00E94C2
:107D6000B2A06D8582E30E9451236D858AE30E9453
:107D7000512382E30E947423C7CE8FE793E00F94D0
:107D800044129E8B8D8B0E946D1D162F072FF82E8F
:107D9000E92E84E493E00E94211D9B01AC0180E464
:107DA00093E029AF3AAF4BAF5CAF0E94211DEF9239
:107DB000FF920F931F93B0EFAB2EB3E2BB2EB4E74D
:107DC000CB2EB9E4DB2E8601750129AD3AAD4BAD62
:107DD0005CAD0E94918521E041E061E080E00E947D
:107DE00063884B015C0121E041E061E080E00E949A
:107DF00063886B017C019B01AC01C501B4010F9448
:107E000060092B013C010F900F900F900F902DEC0B
:107E10003CEC4CEC5DE30F94F90B181654F02DEC90
:107E20003CEC4CEC5DEBC301B2010F94C50987FF3C
:107E300025C04D855E856F85788982E197E00E9437
:107E4000B2A08D859E85AF85B8898897A105B105BB
:107E50000CF05ACE82E30E9474232D853E854F8517
:107E600058892E5F3F4F4F4F5F4F2D873E874F877B
:107E7000588BBA01A90184EF96E071CFA501940156
:107E8000C701B6010F94610920E030E040E05FE3F4
:107E90000F946D0C6DA77EA78FA798AB81E893E038
:107EA0000F9444128C01D1018D919C91119792FFF6
:107EB0000CC05E968D919D910D90BC91A02D892B4B
:107EC0008A2B8B2B11F00C94AA4B298D3A8D4B8D5C
:107ED0005C8D69A17AA18BA19CA10F94610920E01E
:107EE00030E040E05FE30F946D0C698F7A8F8B8FE9
:107EF0009C8F2D8D3E8D4F8D58A12093030730937D
:107F00000407409305075093060781E00E94BA8753
:107F1000D1018D919C91119792FFABC05E968D918E
:107F20009D910D90BC91A02D0297A105B10509F07E
:107F3000A0C020E030E040EA52E4698D7A8D8B8D5C
:107F40009C8D0F946D0C20E030E048EC54E40F94CD
:107F500060090F94650A6B017C0129893A894427DD
:107F600037FD4095542F298B3A8B4B8B5C8B2DA181
:107F70003EA14FA158A569A57AA58BA59CA50F94F4
:107F8000610920E030E040E05FE30F946D0C20E0F9
:107F900030E040EA52E40F946D0C20E030E048EC11
:107FA00054E40F9460090F94650A2B013C018D89FC
:107FB0009E89AA2797FDA095BA2F8D8B9E8BAF8B9C
:107FC000B88F20E030E040EA52E46DA57EA58FA591
:107FD00098A90F946D0C20E030E048EC54E40F9425
:107FE00060090F94650A4B015C01222717FD20955B
:107FF000322FC414D504E604F70414F00C94C24BD9
:10800000C814D904EA04FB0414F00C94EA4B4C188D
:108010005D086E087F088D899E89AF89B88D480EEE
:10802000591E6A1E7B1E8C189D08AE08BF08800E64
:10803000911EA21EB31EC2010E94D51DC4010E9442
:10804000F51DC12CD12C7601A1E94A16A1E05A06F2
:108050006104710414F00C941E4CB1E98B16B1E06C
:108060009B06A104B10414F00C941E4C80E00E9405
:108070004ECF20E030E0A901698D7A8D8B8D9C8DEB
:108080000F94C50987FD40CD20E030E0A9016DA522
:108090007EA58FA598A90F94C50987FD35CD81E0F0
:1080A0000E94E3808AEB96E00E94451E8EE390E2F8
:1080B0000E941D962D8D3E8D4F8D58A12093030754
:1080C00030930407409305075093060741E061E0B1
:1080D00081E00E94D487FCC310920E08F101EB5A94
:1080E000FF4F8081882309F4F3C385EA96E00CC032
:1080F00081E080930E08F101EB5AFF4F80818823C5
:1081000009F4E6C380E996E00E94A69FE1C380904F
:10811000C9079090CA07A090CB07B090CC074090B9
:10812000CD075090CE076090CF077090D007C090D9
:10813000D107D090D207E090D307F090D407D101B7
:108140001C9113FF2BC01A96EC911A971B96FC9169
:108150001B971C960C911C971D96BC908091510802
:10816000882361F023E333E34BEC51E4BF01802F1C
:108170009B2D0F946D0CFB01DC0102C0A02FBB2DC9
:108180002091F1073091F2074091F3075091F407E5
:10819000BF01CD010F9460094B015C0114FF2CC09D
:1081A000D1011E96EC911E971F96FC911F97509639
:1081B0000C91509751967C9080915108882361F0E2
:1081C00023E333E34BEC51E4BF01802F972D0F9451
:1081D0006D0CFB01DC0102C0A02FB72D2091F5072B
:1081E0003091F6074091F7075091F807BF01CD0194
:1081F0000F9460092B013C0115FF2CC0D101529650
:10820000EC9152975396FC91539754961C91549726
:1082100055960C9180915108882361F023E333E354
:108220004BEC51E4BF01812F902F0F946D0CFB019B
:10823000DC0102C0A12FB02F2091F9073091FA077D
:108240004091FB075091FC07BF01CD010F946009DD
:108250006B017C0187017601A3019201C501B40184
:108260000E94B079F101808186FF32C3E689D10195
:108270005796FC91579758961C91589759960C9180
:1082800080915108882361F023E333E34BEC51E400
:10829000BF01812F902F0F946D0CFB01DC0102C0F8
:1082A000A12FB02F20913303309134034091350337
:1082B00050913603BF01CD010F946D0C0F94650AE8
:1082C0006093090870930A0880930B0890930C0838
:1082D000FFC28090F9079090FA07A090FB07B0903A
:1082E000FC0720910B0730910C0740910D0750912E
:1082F0000E07C501B4010F94CC092DEC3CEC4CECFD
:108300005DE30F94F90B18162CF48AE596E00E94B1
:10831000B09FDEC2F10122818081918122FF0CC0D9
:1083200083FF02C00C943A4C80739927892B11F07B
:108330000C943A4C0C94404C83FF6FC0C284D3849D
:10834000E484F58420E030E0A901C701B6010F9470
:10835000F90B181664F420E030E040E251E4C70164
:10836000B6010F94C50918160CF459C00AC020E0D4
:1083700030E040E251ECC701B6010F94F90B87FDE4
:108380004EC0A5019401C701B6010F9461099B017C
:10839000AC016091170770911807809119079091AF
:1083A0001A070F9461096093170770931807809359
:1083B000190790931A070E94DB7440911707509198
:1083C00018076091190770911A0723E08DE595E071
:1083D0000E948EA18091170790911807A09119070C
:1083E000B0911A0789879A87AB87BC8744E050E031
:1083F00065E870E0CE0109960F9449120E9437CFCC
:10840000682F88E690E069AF0F94371269AD68175E
:1084100021F088E690E00F94521210E001C011E0C4
:10842000F101808184FF71C0C684D784E088F1881F
:1084300020E030E0A901C701B6010F94F90B18162E
:1084400064F420E030E040E251E4C701B6010F944B
:10845000C50918160CF458C00AC020E030E040E20C
:1084600051ECC701B6010F94F90B87FD4DC0A50172
:108470009401C701B6010F9461099B01AC016091A1
:108480000F077091100780911107909112070F94B8
:10849000610960930F077093100780931107909301
:1084A00012070E94DB7440910F07509110076091F2
:1084B00011077091120723E082E495E00E948EA1DB
:1084C00080910F0790911007A0911107B0911207AA
:1084D0008D839E83AF83B88744E050E069E870E005
:1084E000CE0105960F9449120E9437CF682F88E677
:1084F00090E069AF0F94371269AD681731F088E6E4
:1085000090E00F94521201C011E0D1018C9185FFCF
:1085100074C05296CD90DD90ED90FC90559720E080
:1085200030E0A901C701B6010F94F90B18165CF4ED
:1085300020E030E040E251E4C701B6010F94C509E4
:1085400018165CF00EC020E030E040E251ECC701AC
:10855000B6010F94F90B87FF04C08BEA95E00C94E9
:108560003C4CA5019401C701B6010F9461099B0120
:10857000AC016091070770910807809109079091FD
:108580000A070F94610960930707709308078093A7
:10859000090790930A070E94DB74409107075091E6
:1085A00008076091090770910A0723E087E295E0C8
:1085B0000E948EA18091070790910807A09109075A
:1085C000B0910A0789839A83AB83BC8344E050E06F
:1085D0006DE870E0CE0101960F9449120E9437CFEA
:1085E000682F88E690E069AF0F94371269AD68177D
:1085F00021F088E690E00F9452121111AECF89E479
:108600008F9384E78F9383E28F9380EF8F93F0EFC4
:10861000AF2EF3E2BF2EF4E7CF2EF9E4DF2EE12CEC
:10862000F12C00E411E4A6019501C601B5010E94F8
:1086300091850F900F900F900F904AC180E00E949B
:10864000BA871092C9071092CA071092CB071092EE
:10865000CC071092CD071092CE071092CF07109240
:10866000D0071092D1071092D2071092D307109220
:10867000D4076091130370911403809115039091B6
:1086800016030E94337A8091470790914807A09182
:108690004907B0914A0740913F07509140076091C8
:1086A000410770914207C0904307D0904407E09083
:1086B0004507F09046075A01F62FE72F481759074C
:1086C0006A077B071CF45C01FA2FEB2F85012F2F23
:1086D0003E2F0C151D052E053F0514F4970186014C
:1086E000480159018C189D08AE08BF08680179013E
:1086F000C41AD50AE60AF70A28013901481A590AA4
:108700006A0A7B0AB501A40180E093E20E94B2A04C
:10871000B701A60187EF92E20E94B2A0B301A201C5
:108720008EEE92E20E94B2A0F1018081918192FFCF
:10873000CDCC868D978DA0A1B1A1181619061A0669
:108740001B060CF0C3CCC4010E94B51DC6010E94DB
:10875000D51DC2010E94F51DB9CC7090C80775FAED
:10876000772470F880E00E94BA871092FD0710927B
:10877000FE071092FF071092000810920108109255
:108780000208109203081092040810920508109233
:10879000060810920708109208081092C907109254
:1087A000CA071092CB071092CC071092CD071092F7
:1087B000CE071092CF071092D0071092D1071092D7
:1087C000D2071092D3071092D4071092110810927A
:1087D00012081092130810921408109215081092A3
:1087E0001608109217081092180810921908109283
:1087F0001A0810921B0810921C08609113037091C4
:10880000140380911503909116030E94337A00910E
:108810002B0710912C0720912D0730912E07809166
:108820001F0790912007A0912107B0912207081BF4
:10883000190B2A0B3B0B08511C4F2F4F3F4F8091B8
:108840003F0790914007A0914107B091420748012E
:108850005901881A990AAA0ABB0A80914707909180
:108860004807A0914907B0914A0768017901C81AE1
:10887000D90AEA0AFB0A8091430790914407A09124
:108880004507B0914607B901A801481B590B6A0B6F
:108890007B0B80E093E20E94B2A0B501A40187EFB8
:1088A00092E20E94B2A0B701A6018EEE92E20E946F
:1088B000B2A0872D0E94BA8709CC8091EA0282FF7C
:1088C00007C08CE594E20E94769FC1010E946497E4
:1088D0000F94FC0360938C1D70938D1D80938E1DEF
:1088E00090938F1DEC960FB6F894DEBF0FBECDBFF0
:1088F000DF91CF911F910F91FF90EF90DF90CF907C
:10890000BF90AF909F908F907F906F905F904F90AF
:108910003F902F9008958FEA9CE00E941D9687EA71
:108920009CE00E94769F0E94641D882321F084EAC7
:108930009CE00E94769F0E94691D882321F081EAB5
:108940009CE00E94769F379922C08EE79CE01CC075
:108950008DE19CE00E941D9685E19CE00E94769F3F
:108960000E94641D882321F082E19CE00E94769F92
:108970000E94691D882321F08FE09CE00E94769F71
:108980003799F1C48CEE9BE00E948F9FA1CF8EE9B6
:108990009CE00E94769FD9CF8FE390E20E941D96C3
:1089A00080E00E94BA870E946D1D162F072FF82EB7
:1089B000E92E84E393E00E94211D9B01AC0180E33A
:1089C00093E029AF3AAF4BAF5CAF0E94211DEF920D
:1089D000FF920F931F9350EFA52E53E2B52E54E74D
:1089E000C52E59E4D52E8601750129AD3AAD4BADA2
:1089F0005CAD0E94918520E041E060E081E00E9452
:108A0000638869A77AA78BA79CA720E041E060E074
:108A100081E00E94638869A37AA38BA39CA39B0136
:108A2000AC0169A57AA58BA59CA50F9460096B0183
:108A30007C010F900F900F900F902DEC3CEC4CECC4
:108A40005DE30F94F90B181654F02DEC3CEC4CEC54
:108A50005DEBC701B6010F94C50987FF1AC04989AC
:108A60005A896B897C8982EC9BE00E94B2A089893B
:108A70009A89AB89BC898897A105B10511F40C943A
:108A8000043882E30E947423B301A20184EA9BE0CC
:108A90001BC18DE793E00F9444129E8B8D8BD10107
:108AA0008D919C91119792FF0BC05E968D919D9137
:108AB0000D90BC91A02D0297A105B10509F458C4F1
:108AC0000E946D1D162F072FF82EE92E8CE393E0E0
:108AD0000E94211D9B01AC0188E393E029AF3AAFCE
:108AE0004BAF5CAF0E94211DEF92FF920F931F933B
:108AF00000EFA02E03E2B02E04E7C02E09E4D02E32
:108B00008601750129AD3AAD4BAD5CAD0E949185F2
:108B100020E041E060E081E00E9463886DA77EA7CD
:108B20008FA798AB20E041E060E081E00E9463887D
:108B300069AB7AAB8BAB9CAB9B01AC016DA57EA501
:108B40008FA598A90F9460096B017C010F900F907D
:108B50000F900F902DEC3CEC4CEC5DE30F94F90B77
:108B6000181654F02DEC3CEC4CEC5DEBC701B60153
:108B70000F94C50987FF21C049895A896B897C896F
:108B80008FE49BE00E94B2A029893A894B895C89D5
:108B9000283231054105510541F082E30E947423DA
:108BA000B301A20181E39BE08FC08EE19BE00E94B4
:108BB0008F9F86E09BE00C940A388FE793E00F9438
:108BC00044129E8F8D8FD1018D919C91119792FFB0
:108BD0000BC05E968D919D910D90BC91A02D02973A
:108BE000A105B10509F4D1C30E946D1D162F072FF1
:108BF000F82EE92E84E493E00E94211D9B01AC0134
:108C000080E493E029AF3AAF4BAF5CAF0E94211DE7
:108C1000EF92FF920F931F9310EFA12E13E2B12E4C
:108C200014E7C12E19E4D12E8601750129AD3AADA4
:108C30004BAD5CAD0E94918520E041E060E081E0B9
:108C40000E9463886B017C0120E041E060E081E0EC
:108C50000E9463886DAB7EAB8FAB98AF9B01AC017C
:108C6000C701B6010F9460094B015C010F900F9092
:108C70000F900F902DEC3CEC4CEC5DE30F94F90B56
:108C8000181654F02DEC3CEC4CEC5DEBC501B40136
:108C90000F94C50987FF42C049895A896B897C892D
:108CA0008CED9AE00E94B2A029893A894B895C89AF
:108CB000283231054105510549F182E30E947423B0
:108CC000B301A2018EEB9AE00E94B2A0642D82E370
:108CD0000E945123642D8AE30E94512382E30E9463
:108CE0007423F2E04F0E511C611C711C29893A89D2
:108CF0004B895C892E5F3F4F4F4F5F4F298B3A8BDB
:108D00004B8B5C8B31E03DA30C94D1378BEA9AE01E
:108D10000E948F9F83E99AE00C940A3829A13AA116
:108D20004BA15CA169A57AA58BA59CA50F946109AF
:108D300020E030E040E05FE30F946D0C20E030E095
:108D400040EA52E40F946D0C20E030E048EC54E42B
:108D50000F9460090F94650A4B015C018D899E890F
:108D6000AA2797FDA095BA2F8D8B9E8BAF8BB88FBE
:108D700029A93AA94BA95CA96DA57EA58FA598A99B
:108D80000F94610920E030E040E05FE30F946D0C48
:108D900020E030E040EA52E40F946D0C20E030E037
:108DA00048EC54E40F9460090F94650A2B013C01D0
:108DB0002D8D3E8D442737FD4095542F2D8F3E8FAE
:108DC0004F8F58A32DA93EA94FA958ADC701B60191
:108DD0000F94610920E030E040E05FE30F946D0CF8
:108DE00020E030E040EA52E40F946D0C20E030E0E7
:108DF00048EC54E40F9460090F94650A6B017C0100
:108E000081E893E00F9444129C01442737FD40957C
:108E1000542F29A33AA34BA35CA380E00E94E380D4
:108E20000E94DB748BE590E20E94A69F40910B07A5
:108E300050910C0760910D0770910E0722E086ECAF
:108E40009FE10E948EA1898D9A8DAB8DBC8D809300
:108E5000030790930407A0930507B09306078414B3
:108E60009504A604B70414F58C149D04AE04BF0445
:108E70000CF042C0481859086A087B082D8D3E8DB9
:108E80004F8D58A1420E531E641E751EC818D90876
:108E9000EA08FB0889A19AA1ABA1BCA1C80ED91E02
:108EA000EA1EFB1E812C912C540152C04814590417
:108EB0006A047B040CF54C145D046E047F04E4F436
:108EC00084189508A608B7082D893E894F89588DC2
:108ED000820E931EA41EB51EC418D508E608F70816
:108EE00089A19AA1ABA1BCA1C80ED91EEA1EFB1E86
:108EF000412C512C320125C0C814D904EA04FB04CA
:108F000004F5C414D504E604F704DCF48C189D08B9
:108F1000AE08BF082D893E894F89588D820E931E59
:108F2000A41EB51E4C185D086E087F088D8D9E8DA1
:108F3000AF8DB8A1480E591E6A1E7B1EC12CD12CC4
:108F4000760191E9891691E09906A104B10474F4BF
:108F5000A1E94A16A1E05A06610471043CF4B1E9A2
:108F6000CB16B1E0DB06E104F104FCF049895A8933
:108F70006B897C8982E69AE00E94B2A088E49AE03C
:108F80000E941D96B501A40184E49AE00E94B2A05B
:108F9000B301A20180E49AE00E94B2A0B701A60149
:108FA0008CE39AE00E94B2A093CCC4010E94B51D4C
:108FB000C2010E94D51DC6010E94F51D80E00E94DD
:108FC0004ECF0C9414382DEC3CEC4CEC5DEBC30113
:108FD000B2010F94C50987FF09C00C948A3882ED4D
:108FE00099E00E948F9F8AEB99E0D0C09FEF291AE9
:108FF000390AA5019401C701B6010F94610920E067
:1090000030E040E05FE30F946D0C2B013C01409198
:109010000B0750910C0760910D0770910E0722E02D
:109020008CEA99E00E948EA12091F9073091FA070D
:109030004091FB075091FC07C301B2010F946009F6
:109040009B01AC0160910B0770910C0780910D079B
:1090500090910E070F94610960930B0770930C07B2
:1090600080930D0790930E070E94DB7440910B07CD
:1090700050910C0760910D0770910E0722E08EE968
:1090800099E00E948EA10E946D1D162F072FF82EC9
:10909000E92E84E493E00E94211D9B01AC0180E451
:1090A00093E029AF3AAF4BAF5CAF0E94211DEF9226
:1090B000FF920F931F93A0EFAA2EA3E2BA2EA4E76C
:1090C000CA2EA9E4DA2E8601750129AD3AAD4BAD61
:1090D0005CAD0E94918520E041E060E081E00E946B
:1090E00063886B017C0120E041E060E081E00E9448
:1090F00063886D8B7E8B8F8B988F9B01AC01C70132
:10910000B6010F9460094B015C010F900F900F9016
:109110000F902DEC3CEC4CEC5DE30F94F90B181622
:1091200054F02DEC3CEC4CEC5DEBC501B4010F941C
:10913000C50987FF33C04D855E856F8578898FE6C9
:1091400099E00E94B2A02D853E854F85588928322E
:10915000310541055105A4F482E30E9474238D85F5
:109160009E85AF85B8890296A11DB11D8D879E870A
:10917000AF87B88BAC01BD0181E599E00C94AF38A5
:109180008EE399E00E948F9F86E299E00E941D96EF
:1091900086ED9FE10E94B09F0C94C1382D893E89D5
:1091A0004F89588DC701B6010F94610920E030E066
:1091B00040E05FE30F946D0C9B01AC01C301B20171
:1091C0000F94600920E030E040EA52E40F946D0C07
:1091D0006B017C0120E030E0A9010F94C50987FFF5
:1091E00027C0C701B60190582091770730917807C2
:1091F0004091790750917A070F94CC099B01AC01FB
:109200000F9461096B017C0122E0AB01BC018AE68D
:1092100090E20E948EA1A70196016091770770915C
:1092200078078091790790917A070F94600918C0A8
:109230008090770790907807A0907907B0907A0790
:10924000A5019401C701B6010F94CC099B01AC01A3
:109250000F9461099B01AC01C501B4010F94610930
:1092600060937707709378078093790790937A07D4
:10927000C0907707D0907807E0907907F0907A0750
:1092800022EC35EF41EB52E4C701B6010F94CC0953
:109290004B015C012DEC3CEC4CE85FE30F94F90BC7
:1092A000181654F026E636E646E65FE3C501B4013B
:1092B0000F94C50987FF13C022E0B701A6018BE018
:1092C00099E00E948EA182EC95EFA1EBB2E480932D
:1092D000770790937807A0937907B0937A0722E0F5
:1092E00049895A896B897C8983EF98E00E948EA115
:1092F00040917707509178076091790770917A07CC
:1093000022E08BED98E00E948EA194E029163104B2
:1093100014F00C94C13829893A894B895C89609191
:109320007707709178078091790790917A070F9469
:1093300060096B017C012DEC3CEC4CEC5DE30F947F
:10934000F90B181614F40C942D382DEC3CEC4CEC65
:109350005DEBC701B6010F94C50987FF02C00C94ED
:109360002D380C94C1388CE09CE00E94769F0ACB8B
:1093700041E061E081E00E94D4878FE390E20E94A7
:109380001D9680E00E94BA879BCB41E061E081E0BE
:109390000E94D4878FE390E20E941D9680E00E9495
:1093A000BA8722CCC90188719927489709F474C1FA
:1093B00020E041E060E081E00E9463882091F907AD
:1093C0003091FA074091FB075091FC070F94600918
:1093D0004B015C0120E041E061E080E00E94638895
:1093E0002091F9073091FA074091FB075091FC0753
:1093F0000F9460092B013C019B01AC01C501B40134
:109400000F9460096B017C012DEC3CEC4CEC5DE3AE
:109410000F94F90B181654F02DEC3CEC4CEC5DEB72
:10942000C701B6010F94C50987FF21C022E0B7012B
:10943000A6018AE998E00E948EA182E30E9474232B
:1094400046E150E060E070E08CE798E00E94B2A056
:1094500066E182E30E94512366E18AE30E94512380
:1094600082E30E94742388E798E00C94FC38A301FF
:109470009201C501B4010F94610920E030E040E0A1
:109480005FE30F946D0CAB01BC0122E089E698E02C
:109490000E948EA11DCA8091030790910407A0919C
:1094A0000507B09106078D879E87AF87B88BF101BE
:1094B0008081918192FF09C0868D978DA0A1B1A175
:1094C0000297A105B10509F4AEC041E061E081E079
:1094D0000E94D4878FE390E20E941D9680E00E9454
:1094E000BA870E946D1D9F938F937F936F93F0EFC8
:1094F000AF2EF3E2BF2EF4E7CF2EF9E4DF2E860184
:10950000750120E030E0A901CA01B9010E949185EE
:1095100020E041E060E081E00E9463884B015C0153
:1095200020E041E060E081E00E9463886B017C0103
:109530009B01AC01C501B4010F9460092B013C01F2
:109540000F900F900F900F902DEC3CEC4CEC5DE3E6
:109550000F94F90B181654F02DEC3CEC4CEC5DEB31
:10956000C301B2010F94C50987FF05C086ED9FE1D5
:109570000E94B09F9CCFA5019401C701B6010F9432
:10958000610920E030E040E05FE30F946D0C6B0177
:109590007C0120E030E040E85FE30F94C50987FDDF
:1095A00086CFD1018D919C91119792FF0BC05E9651
:1095B0008D919D910D90BC91A02D892B8A2B8B2B89
:1095C00009F043C02D853E854F85588920930307B8
:1095D00030930407409305075093060781E00E94EB
:1095E000BA87D1018D919C91119792FF0BC05E9625
:1095F0008D919D910D90BC91A02D0297A105B10573
:1096000009F446C081E00E94E38087EB98E00E9465
:10961000451E8EE390E20E941D962D853E854F8566
:1096200058890C945E4020E030E046E653E42093F5
:109630000B0730930C0740930D0750930E0780E003
:109640000E944ECF0E94ABD140CF2091F9073091BC
:10965000FA074091FB075091FC07C701B6010F9430
:1096600060099B01AC0160910B0770910C07809120
:109670000D0790910E070F94610960930B0770938B
:109680000C0780930D0790930E070E94DB749ACF0E
:1096900080E00E944ECFB6CF30FF27C0D1011E968A
:1096A0002D913D914D915C9151971A966D917D91BF
:1096B0008D919C911D975D96EC915D97EF935C96D3
:1096C000EC915C97EF935B96EC915B97EF935A96D6
:1096D000EC91EF93E0EFAE2EE3E2BE2EE4E7CE2E68
:1096E000E9E4DE2E860175011BC00E946D1DF101AB
:1096F00026853785408951894284538464847584E2
:109700009F938F937F936F9360EFA62E63E2B62EA5
:1097100064E7C62E69E4D62E86017501C301B20145
:109720000E9491850F900F900F900F9041CE80E096
:1097300090E00E94B51D80E090E00E94D51D80E081
:1097400090E00E94F51D80E00E944ECF0E94ABD1B8
:109750000C94963D80E00E94E3800E94DB748BE5D0
:1097600090E20E94A69F40910B0750910C076091D8
:109770000D0770910E0722E086EC9FE10E948EA1FA
:109780000C94653F4C145D046E047F041CF5481472
:1097900059046A047B04F4F4C418D508E608F708F1
:1097A00089899A89AB89BC89C80ED91EEA1EFB1E1D
:1097B00084189508A608B708800E911EA21EB31E35
:1097C000C6010E94B51DC4010E94F51D412C512CFB
:1097D00032012BC08C149D04AE04BF0434F58414F4
:1097E0009504A604B7040CF5C818D908EA08FB08C4
:1097F00029893A894B895C89C20ED31EE41EF51E65
:10980000481859086A087B088D899E89AF89B88DE8
:10981000480E591E6A1E7B1EC6010E94B51DC2015C
:109820000E94D51D812C912C540191E9C91691E01B
:10983000D906E104F10414F40C9424404D855E85AE
:109840006F8578898BEC96E00E94B2A0B701A601E3
:1098500087EC96E00E94B2A0B301A20183EC96E0EF
:109860000E94B2A0B501A4018FEB96E00E94B2A0C5
:109870000C94843D80E396E00E94B09F0C94FF42DC
:10988000C6A4D7A4E0A8F1A820E030E0A901C70150
:10989000B6010F94C509882361F120E030E0A901E9
:1098A000C701B6010F94F90B18165CF420E030E004
:1098B00040E251E4C701B6010F94C5091816B4F08F
:1098C0000AC020E030E040E251ECC701B6010F943D
:1098D000F90B87FD0BC085E793E00E94211D9B01DA
:1098E000AC01C701B6010F9461094DC087E096E055
:1098F000C3CF20E030E0A9016091F1077091F20739
:109900008091F3079091F4070F94C509811161C00C
:1099100020E030E0A9016091F5077091F607809191
:10992000F7079091F8070F94C509811152C08091F3
:10993000C80787FF2CC0C0908307D0908407E090B1
:109940008507F09086076091150870911608809140
:109950001708909118080F94960A9B01AC010F9478
:109960006D0C9B01AC01C701B6010F9460090F9407
:10997000DA0C2091490830914A0840914B085091E7
:109980004C080F946D0C0E94701D0C94FF42C09007
:109990008307D0908407E0908507F0908607609158
:1099A00015087091160880911708909118089B016E
:1099B000AC010F94340DC61AD70AE80AF90AC70198
:1099C000B6010E94E1D9BC0180E090E00F94960AB4
:1099D000D0CF84ED95E050CFCF93DF93EC01409151
:1099E000EA028881998144FF09C082FD2AC081FF73
:1099F00005C02E813F812F36310519F582FF05C044
:109A0000CE01DF91CF910C94B33581FF05C0CE011B
:109A1000DF91CF910C947F2491FF08C00E94371EE4
:109A2000CC5ADF4F8881DF91CF91E1C242FF13C052
:109A30008CE594E20E94769FCE01DF91CF910C9449
:109A400064970F94FC0360938C1D70938D1D80931D
:109A50008E1D90938F1DDF91CF9108958091C60741
:109A600080FD1DC00E9457980E94E392EC0186E79A
:109A70009AE00E946BCA2097B1F080918D098823EB
:109A800041F0888181FF12C08E819F814D9771F4D2
:109A900016C0CE01A1DFCE010E94429804C086E725
:109AA0009AE00E946BCA0E94D179D8CFBE0182E2AF
:109AB00099E00E947F9BCE010E943198ECCF82E218
:109AC00099E00E94F49EF7CF0E945F8C0C948F2344
:109AD000C5CFCF93DF93FC01E05CFF4F208121FDD8
:109AE0001FC0DB014D915D916D917C91DC01AF5BFD
:109AF000BF4F4D935D936D937C931397EC01CB5BBC
:109B0000DF4FDC0117964D915D916D917C911A9715
:109B1000488359836A837B83822F897F8260808315
:109B2000DF91CF9108959F92AF92BF92CF92DF9233
:109B3000EF92FF920F931F93CF93DF93EC015B01A2
:109B40008C01005C1F4FF801908092FC32C0CB84E6
:109B5000DC84ED84FE84A70196016F817885898578
:109B60009A850F9460099F7720E030E040E85FE33A
:109B70000F94610920E030E040EA51E40F94F90BC2
:109B80001816BCF0F50180819181A281B381FE019C
:109B9000EF5BFF4F80839183A283B383CB5BDF4F67
:109BA000C882D982EA82FB82892D897F8460F8018C
:109BB0008083DF91CF911F910F91FF90EF90DF9005
:109BC000CF90BF90AF909F9008958091C807846018
:109BD0008093C80708952F923F924F925F926F92A1
:109BE0007F928F929F92AF92BF92CF92DF92EF922D
:109BF000FF920F931F93CF93DF93CDB7DEB7649798
:109C00000FB6F894DEBF0FBECDBF382E292E7A874F
:109C100069875A834983098B1A8B2B8B3C8B4AA407
:109C20005BA46CA47DA423E333E948E853E4C501B5
:109C3000B4010F9461096D837E838F83988720E040
:109C400030E0A901C301B2010F94C509882359F17D
:109C50002EA53FA548A959A9C301B2010F946109D6
:109C60004B015C0120E030E040EA50E4C301B20166
:109C70000F946D0CA50194010F94CC096D877E871C
:109C80008F87988BA30192016EA57FA588A999A9BA
:109C90000F946D0CA50194010F94CC096EA77FA7BA
:109CA00088AB99AB08C080E090E0A0EAB0E48D8773
:109CB0009E87AF87B88B2D813E814F8158856989FA
:109CC0007A898B899C8990580F94CC090F94390A12
:109CD0009B01AC01C701B6010F946D0C6D837E83AF
:109CE0008F83988769817A81A985BA856A1B7B0BE6
:109CF000882777FD8095982F0F94980A20E030E010
:109D000040E05DE30F946D0C69877A878B879C87B1
:109D1000032D122D212C312C89819A81AA2797FDA0
:109D2000A095BA2F89839A83AB83BC83A895698158
:109D30007A818B819C810F94980A6B017C01B1011F
:109D4000882777FD8095982F0F94980A29853A8562
:109D50004B855C850F946D0C9B01AC01C701B6016E
:109D60000F9460096B017C0123E333E548E853E479
:109D70000F9461099B01AC0169897A898B899C895F
:109D80000F94CC090F94390A2D813E814F8158855B
:109D90000F946D0C4B015C0120E030EC4FE755E473
:109DA0000F946D0C2D853E854F8558890F946D0C51
:109DB0002B013C01A50194016EA57FA588A999A955
:109DC0000F94610920E030E040EA50E40F946D0CFC
:109DD0009B01AC01C301B2010F94CC090F94650A39
:109DE0006D3F9FE0790714F06CEF7FE0D8016D9331
:109DF0007C9320E030E040E051E4C701B6010F94CD
:109E00006D0C0F94650AF80173836283FFEF2F1ABC
:109E10003F0A0C5F1F4F81E22816310409F086CFFC
:109E200064960FB6F894DEBF0FBECDBFDF91CF9121
:109E30001F910F91FF90EF90DF90CF90BF90AF9068
:109E40009F908F907F906F905F904F903F902F905A
:109E50000895CF92DF92EF92FF92CF93DF93EC01C0
:109E60008B898130A9F5CE8CDF8CE8A0F9A020E0A9
:109E700030E0A901C701B6010F94C509882341F15B
:109E8000688D70E080E090E00F94960A20E030E06A
:109E900040E251E40F946D0CA70196010F94CC0998
:109EA0006FA378A789A79AA7698D70E080E090E0FA
:109EB0000F94960A20E030E040E251E40F946D0CDC
:109EC000A70196010F94CC096BA77CA78DA79EA72D
:109ED000DF91CF91FF90EF90DF90CF9008958EE0CB
:109EE00092E0B7CF7F928F929F92AF92BF92CF9224
:109EF000DF92EF92FF920F931F93CF93DF938BE547
:109F000092E0909391038093900385E4782E7F9262
:109F1000D2E9DF93C0EECF931F921F921F921F9240
:109F20001F92812C912C98ECA92E91E4B92EC12C72
:109F300020E5D22E23ECE22E27E4F22E00E010E101
:109F40002BE835E44CE251E06EEC7FEF87E194E0E2
:109F500042DE7F92DF93CF931F921F921F921F9238
:109F60001F9200E018E728E835E44CE251E06CEE7F
:109F70007FEF83E993E02FDE80910A018064809374
:109F80000A013B9A809168022DB73EB7205F3F4F90
:109F90000FB6F8943EBF0FBE2DBF87FD0CC061E029
:109FA0000F94100580916902811105C061E08091D4
:109FB00068020F9449050F94FC0360939502709317
:109FC000960280939702909398026D9A759887DF16
:109FD000DF91CF911F910F91FF90EF90DF90CF9085
:109FE000BF90AF909F908F907F900C94D5DA4F9256
:109FF0005F926F927F92AF92BF92CF92DF92EF9279
:10A00000FF920F931F93CF93DF93CDB7DEB72C97BB
:10A010000FB6F894DEBF0FBECDBF809109089091B6
:10A020000A08A0910B08B0910C08E0919003F09100
:10A030009103838F948FA58FB68F2BE532E03093F9
:10A040009103209390038093E1079093E207A093FC
:10A05000E307B093E407409064025090650260907B
:10A06000660270906702409233035092340360920C
:10A07000350370923603A301920160E070E080E83E
:10A080009FE30F94CC0960934D0870934E08809322
:10A090004F0890935008C0906A02D0906B02E090F5
:10A0A0006C02F0906D02C0922303D0922403E092E0
:10A0B0002503F092260360916E0270916F028091E9
:10A0C0007002909171026093F7027093F80280938E
:10A0D000F9029093FA026093070370930803809348
:10A0E000090390930A03A30192010F946D0C0F943E
:10A0F0006A0A60933D0870933E0880933F089093EE
:10A10000400860932D0870932E0880932F08909339
:10A110003008209172023091730240917402509184
:10A120007502C301B2010F946D0C9B01AC0160E09C
:10A1300074E284E798E40F94CC090F94D30A0F9447
:10A140006A0A162F60935508A3019201C701B60150
:10A150000F946D0C9B01AC0160E074E284E798E41D
:10A160000F94CC090F94D30A0F946A0A603118F443
:10A170006093540803C08FE0809354088091540882
:10A18000811710F0109354086091540870E080E03B
:10A1900090E00F94960AA30192010F946D0C9B011D
:10A1A000AC0160E074E284E798E40F94CC092B01E1
:10A1B0003C01A70196010F94C50987FF08C0409292
:10A1C000230350922403609225037092260386E8AD
:10A1D00092E03FDE2091F1073091F2074091F307C2
:10A1E0005091F4072D833E834F8358874090F507A5
:10A1F0005090F6076090F7077090F8078091F90784
:10A200009091FA07A091FB07B091FC0789879A8784
:10A21000AB87BC8720910307309104074091050765
:10A220005091060729833A834B835C83E090900327
:10A23000F0909103F70181819281A381B4819C0107
:10A24000AD0166277727CB01621B730B840B950B3F
:10A250000F94980A20914108309142084091430898
:10A26000509144080F946D0C6093F7067093F806B4
:10A270008093F9069093FA06F70185819681A7816C
:10A28000B0859C01AD0166277727CB01621B730B5C
:10A29000840B950B0F94980A20914508309146083D
:10A2A00040914708509148080F946D0C6093F30655
:10A2B0007093F4068093F5069093F6068091FF065E
:10A2C000909100070E94911F8091C70780FF24C0D2
:10A2D00080910E038F9380910D038F9380910C03D7
:10A2E0008F9380910B038F9330EFA32E33E2B32E25
:10A2F00034E7C32E39E4D32EE984FA840B851C8518
:10A30000A30192016D817E818F8198850E94267EB6
:10A310000F900F900F900F9089819A81AB81BC8133
:10A320008093030790930407A0930507B093060753
:10A3300080E00E94E3802C960FB6F894DEBF0FBE3B
:10A34000CDBFDF91CF911F910F91FF90EF90DF90E4
:10A35000CF90BF90AF907F906F905F904F900C9494
:10A36000EBDCE0910C02F0910D0267817085818534
:10A3700092850895E0919003F0919103858587FD82
:10A3800006C061E09685911160E00D94490508953D
:10A390008091680287FD07C061E090916902911188
:10A3A00060E00D94490508952F923F924F925F927D
:10A3B0006F927F928F929F92AF92BF92CF92DF92D5
:10A3C000EF92FF920F931F93CF93DF9300D01F92D2
:10A3D000CDB7DEB79C838B83DC011196EC91E5331E
:10A3E00038F4E23348F5EE2369F0ED3090F50DC016
:10A3F000E43628F4E13648F4EC33F1F02AC0E436D0
:10A40000D9F027C049E150E026C0AB81BC8112964B
:10A410008C91A82FB0E0AA0FBB1FA556BB4F4D9142
:10A420005C918CEF9FE0841B950BAB81BC811496F3
:10A430009C938E93139715C0AB81BC8112968C911F
:10A44000A82FB0E0AA0FBB1FA556BB4F4D915C9142
:10A4500002C04FEF5FE0AB81BC8114965C934E93DA
:10A460001397AB81BC8113960D911C911497E53322
:10A4700038F5E23308F0A0C0EE2309F450C0ED3007
:10A4800008F081C1E1508E2F90E0FC01E45AF14FB9
:10A490004491440FFC01EE0FFF1FE859F14F8591E5
:10A4A0009491FC0185909490FC013296A590B49013
:10A4B0007CEF672E7FE0772E601A710A52E03CC075
:10A4C000E436C0F4E13608F0DBC0EC3309F05BC1E0
:10A4D000B801882777FD8095982F0F94980A20E07F
:10A4E00030E04AE754E40F946D0C20E030E040E89F
:10A4F00059E325C1E43609F046C1B801882777FD44
:10A500008095982F0F94980A20E030E04AEF53E4AA
:10A510000F946D0C20E030E040E859E32CC180E05E
:10A5200090E0A8ECB1E4EB81FC8187839087A18760
:10A53000B28729C151014801541708F011C1FC012B
:10A54000E50FF11DE50FF11D05911491FC0161E08E
:10A55000650FE60FF11D5E5FE60FF11D259034904B
:10A56000601671063CF7B501882777FD8095982F16
:10A570000F94980A6B017C01B30168197909882747
:10A5800077FD8095982F0F94980A2B013C01B1011B
:10A590006A197B09882777FD8095982F0F94980A70
:10A5A0009B01AC01C301B2010F946D0C2B013C0166
:10A5B000B80168197909ADC0EE528E2F90E0FC0108
:10A5C000E45AF14F6491660FFC01EE0FFF1FE8594A
:10A5D000F14F85919491FC0125903490FC013296C5
:10A5E0008590949072E0761708F044C0FC01E70F64
:10A5F000F11DE70FF11DA590B490FC0121E0270F9C
:10A60000E20FF11D7E5FE20FF11D259134910A15D5
:10A610001B056CF5B401882777FD8095982F298359
:10A620003A830F94980A6B017C01B801621973098F
:10A63000882777FD8095982F0F94980A2B013C016D
:10A6400029813A81B90168197909882777FD8095B0
:10A65000982F0F94980A9B01AC01C301B2010F948B
:10A660006D0C2B013C01B5016219730952C04901FF
:10A670001501B9CFB901882777FD8095982F75C04E
:10A68000E23639F0A0901704B0901804E7E1F4E046
:10A6900006C0A0909303B0909403E3E9F3E08280B6
:10A6A00093804CEF642E4FE0742E601A710A82E0A2
:10A6B000048115818E5F26803780601671060CF04C
:10A6C00049C0B401882777FD8095982F0F94980A88
:10A6D0006B017C01B3016A197B09882777FD80959E
:10A6E000982F0F94980A2B013C01B1016819790940
:10A6F000882777FD8095982F0F94980A9B01AC01CD
:10A70000C301B2010F946D0C2B013C01B8016A1911
:10A710007B09882777FD8095982F0F94980A9B01D5
:10A72000AC01C301B2010F94CC099B01AC01C7017C
:10A73000B6010F94610920E030E040E05EE30F9441
:10A740006D0CAB81BC8117966D937D938D939C931B
:10A750001A9719C03496823419F041015801A8CFD4
:10A76000B101882777FD8095982F0F94980A20E0F3
:10A7700030E040E05EE30F946D0CEB81FC81678379
:10A780007087818792870F900F900F900F90DF91C5
:10A79000CF911F910F91FF90EF90DF90CF90BF90DE
:10A7A000AF909F908F907F906F905F904F903F9071
:10A7B0002F9008958F929F92AF92BF92CF92DF9287
:10A7C000EF92FF920F931F93CF93DF93EC01CB0196
:10A7D000BA016B877C878D879E87FE01E05CFF4F07
:10A7E0002081297F208320E030E040E051E40F9475
:10A7F0006D0C0F94650A4B012981253318F522331E
:10A8000008F08AC0222309F448C02D3008F019C18D
:10A81000215030E0F901E45AF14FB490BB0CF9013A
:10A82000EE0FFF1FE859F14F25913491F901E590A2
:10A83000F490F901329645915491C12CD12CB2E09B
:10A84000AB2E30C02436B0F4213608F0B4C02C331F
:10A8500009F0F7C0882777FD8095982F2CE0660FC8
:10A86000771F881F991F2A95D1F728EE33E040E023
:10A8700050E09CC0243609F0E4C0882777FD80951D
:10A88000982F0CE0660F771F881F991F0A95D1F744
:10A8900024EF31E040E050E089C01E821D82D1C02B
:10A8A000A8017D01AB1498F5F901EA0DF11DEA0D3F
:10A8B000F11DA591B4916D01F90111E01A0DE10F9F
:10A8C000F11DA394A394E10FF11D059114910815B6
:10A8D000190534F79A01261B370BC7018A1B9B0BFE
:10A8E000DC016CEFC62E6FE0D62ECE18DF080F9479
:10A8F000BB0D9A01201B310B442737FD4095542F87
:10A900000F94990DC20ED31EDE82CD829AC08CEFB9
:10A910009FE08C199D0993C02E5230E0F901E45A52
:10A92000F14FA491AA0FF901EE0FFF1FE859F14F63
:10A9300025913491F90105911491F90132964591CF
:10A940005491C12CD12CB2E0BA1768F5F901EB0F84
:10A95000F11DEB0FF11DA590B4906501F901FF24E5
:10A96000F394FB0EEF0DF11DBE5FEF0DF11DE590B1
:10A97000F4908E149F04A4F49A01261B370BD8017F
:10A98000AA19BB090F94BB0D9A012E193F09442740
:10A9900037FD4095542F0F94990D200F311F08C09B
:10A9A000A7018501D1CFCD82DE824BC00F94990DD6
:10A9B0003E832D8346C0223639F0E0901704F09094
:10A9C0001804A7E1B4E006C0E0909303F09094036C
:10A9D000A3E9B3E012964D915C91139722E014968F
:10A9E0000D911C9115972E5F1696ED91FC9117977E
:10A9F000E815F905D4F49A01261B370BD701A01BE3
:10AA0000B10B0CEF1FE00E191F090F94BB0D9A013B
:10AA10002E1B3F0B442737FD4095542F0F94990D63
:10AA2000020F131F1E830D830CC01496223419F0DD
:10AA3000AF017801D4CF8CEF9FE0801B910B9E83F8
:10AA40008D83DF91CF911F910F91FF90EF90DF9059
:10AA5000CF90BF90AF909F908F9008959F92AF92AC
:10AA6000BF92CF92DF92EF92FF920F931F93CF93FB
:10AA7000DF936B017C01042F922EE0910A02F0918A
:10AA80000B02C1E020E030E040E751E463857485CB
:10AA9000858596850F94F90B18160CF0C0E011E02F
:10AAA0001C2720E030E041E953E4C701B6010F94D0
:10AAB000F90B18166CF020E030E0A901C701B601CF
:10AAC0000F94C50987FF0AC0C12CD12C760106C09E
:10AAD000C12CD12C91E9E92E93E4F92EC02FD0E0BE
:10AAE000FE01EE0FFF1FE65FFD4FA080B180F50174
:10AAF0008181811103C0C12CD12C7601B701A6013F
:10AB0000C50158DE992081F020E030E040EF51E4AB
:10AB1000C701B6010F94F90B181634F4F501E05C87
:10AB2000FF4F80818160808320E030E040E252E48A
:10AB3000C701B6010F94F90B87FD0EC023E82C9FC7
:10AB4000C0012D9F900D1124855A9D4FFC01E458A2
:10AB5000FF4F208131962083602F70E080E090E0ED
:10AB60000F94960AAB01BC0120E084E292E20E94BD
:10AB7000CBA120E0B701A60188E294E20E948EA159
:10AB8000E0910A02F0910B0220E030E040E751E44E
:10AB900063857485858596850F94F90B18167CF06E
:10ABA000111119C0DF91CF911F910F91FF90EF907C
:10ABB000DF90CF90BF90AF909F900C946CD61123F4
:10ABC00051F00F94FC036093ED067093EE068093B2
:10ABD000EF069093F006DF91CF911F910F91FF90B8
:10ABE000EF90DF90CF90BF90AF909F900895CF925D
:10ABF000DF92EF92FF92CF936B017C01C42F20E094
:10AC000030E040EF52E40F94F90B18166CF020E09E
:10AC100030E0A901C701B6010F94C50987FF0AC03A
:10AC2000C12CD12C760106C0C12CD12C20EFE22EF4
:10AC300022E4F22EA70196016091190270911A0286
:10AC400080911B0290911C020F94C509882341F149
:10AC5000B701A6018EE092E0ADDDCC2379F020E0D3
:10AC600030E040EF51E4C701B6010F94F90B18161C
:10AC70002CF480914E02816080934E024091190223
:10AC800050911A0260911B0270911C0220E089E130
:10AC900092E2CF91FF90EF90DF90CF900C948EA135
:10ACA000CF91FF90EF90DF90CF900895E0910A024E
:10ACB000F0910B021682158213861486158616866D
:10ACC000E081F0E0EE57F24E1082E0910C02F0913C
:10ACD0000D02168215821386148615861686E0816B
:10ACE000F0E0EE57F24E10828FEF8093DE0208956F
:10ACF0002F923F924F925F926F927F928F929F928C
:10AD0000AF92BF92CF92DF92EF92FF920F931F9379
:10AD1000CF93DF93CDB7DEB7E5970FB6F894DEBFDC
:10AD20000FBECDBF9DAB8CAB4E8B5F8B688F798F89
:10AD30002E8F0BAB0F94FC036A8F7B8F8C8F9D8FB4
:10AD4000ACA9BDA996968C9190E0959587952C011C
:10AD5000662457FC6094762C86E092E20E94A69FBF
:10AD6000A5DFBE8DB093DE02ACA9BDA9EC91F0E0E9
:10AD7000EE57F24E96968C918083BE8DB11104C031
:10AD80008091D7028093D802530142012A8D3B8DD6
:10AD90004C8D5D8D2BA33CA34DA35EA32F8F38A3B9
:10ADA00049A35AA319821F8630EA388B41E4498BA4
:10ADB0001A8A1B8A50EA5C8B81E48D8B1BA61CA629
:10ADC0001DA61EA61FA218A619A61AA6C12CD12C14
:10ADD00076011FA618AA19AA1AAA91E099871E86B9
:10ADE0001D86A8958CA99DA9DFDAACA9BDA91796E7
:10ADF0003C90179718960C91189719961C911997D3
:10AE00001A962C900F94FC036D837E838F83988712
:10AE1000232D302F412F522D6A897B898C899D8962
:10AE20000F94C50987FF04C03A8A0B8B1C8B2D8AAF
:10AE3000232D302F412F522D69817F858889998953
:10AE40000F94C50987FD04C039820F87188B298AA2
:10AE5000B985BB2309F449C02E893F89488D598D96
:10AE6000632D702F812F922D0F94F90B18160CF073
:10AE700086C08D819E81AF81B8852BA13CA14DA15B
:10AE80005EA1821B930BA40BB50B3E8D311105C047
:10AE900044EC59E060E070E004C04CED55E060E047
:10AEA00070E0481759076A077B0708F068C0ECA9EB
:10AEB000FDA92081E22FF0E0EE57F24E242D281953
:10AEC00020838FA798ABA9ABBAABFE89FA8B2F89E9
:10AED0002B8B388D3C8B498D4D8B8D819E81AF8125
:10AEE000B8858F8F98A3A9A3BAA32E893F89488DCF
:10AEF000598D632D702F812F922D0F94C50987FFD7
:10AF000011C28D819E81AF81B8852F8D38A149A155
:10AF10005AA1821B930BA40BB50B3E8D3111EFC0D0
:10AF200048E853E160E070E0481759076A077B077B
:10AF300008F0F8C14D855E85452B09F0E5C0ACA948
:10AF4000BDA9EC91F0E0EE57F24E882D840D808380
:10AF5000ED85FE853196FE87ED87FE89F9832F8981
:10AF60002F87388D388B498D498B8D819E81AF819C
:10AF7000B8858BA39CA3ADA3BEA391E0998720E0E5
:10AF800030E040E252E46E897F89888D998D0F947C
:10AF900061099B01AC01632D702F812F922D0F94BD
:10AFA000F90B18161CF487E991E23BC08D819E8154
:10AFB000AF81B8852A8D3B8D4C8D5D8D821B930BA7
:10AFC000A40BB50B893E9340A105B10558F080E074
:10AFD0000E941A248D819E81AF81B8858A8F9B8FB4
:10AFE000AC8FBD8F8D819E81AF81B885880F991FF1
:10AFF000AA1FBB1F2BA13CA14DA15EA1821B930BDD
:10B00000A40BB50B2F8D38A149A15AA1821B930B1C
:10B01000A40BB50B81389F44A241B105E8F08AE743
:10B0200091E20E94B09FE5960FB6F894DEBF0FBE86
:10B03000CDBFDF91CF911F910F91FF90EF90DF90E7
:10B04000CF90BF90AF909F908F907F906F905F90C8
:10B050004F903F902F902ACE4D855E85463051050A
:10B060000CF443C08FE191E20E94A69F1FDE5BA912
:10B07000552309F459C1ACA9BDA95A96CD92DD92C8
:10B08000ED92FC925D972FA138A549A55AA55E9631
:10B090002D933D934D935C9391972BA53CA54DA586
:10B0A0005EA592962D933D934D935C93959781E089
:10B0B00053968C9380E0E5960FB6F894DEBF0FBEF2
:10B0C000CDBFDF91CF911F910F91FF90EF90DF9057
:10B0D000CF90BF90AF909F908F907F906F905F9038
:10B0E0004F903F902F900C944ECF86E79AE00E94AD
:10B0F0006BCA61E086E79AE00E946CCA72CE48EBA8
:10B100005BE060E070E010CF2FA538A949A95AA9EB
:10B11000280F391F4A1F5B1F29873A874B875C8797
:10B120002FA538A949A95AA9281B390B4A0B5B0B33
:10B13000CA01B901A50194010F94340D29853A85FE
:10B140004B855C850F94990D240D351D461D571DAB
:10B150002431310541055105A4F0ACA9BDA996964D
:10B160008C9190E04497AA2797FDA095BA2F2901CA
:10B170003A0182179307A407B50744F42C013D0157
:10B1800005C044E1442E512C612C712CECA9FDA981
:10B1900026A1822F869590E0A0E0B0E08415950569
:10B1A000A605B7056CF4822F90E001974C01AA2404
:10B1B00097FCA094BA2C84189508A608B70802C07A
:10B1C00053014201B301A2018EEF91E20E949AA0C5
:10B1D000B501A40189EF91E20E949AA022E0498181
:10B1E0005F856889798982EF91E20E94CBA122E094
:10B1F0004A895B896C897D898BEE91E20E948EA1E0
:10B200002D853E85233031050CF499CEC501B4015E
:10B210000F94980A20E030E040E850E40F946D0C61
:10B220006B017C0129813F85488959896A897B891D
:10B230008C899D890F94600920ED3FE049E450E43A
:10B240000F946D0C9B01AC01C701B6010F94CC09A2
:10B250006B017C0169857A858B859C850F94980AA2
:10B2600020E030E04AE754E40F94CC0969837A8304
:10B270008B839C8322E0B701A60185EE91E20E94B8
:10B28000CBA122E049815A816B817C818FED91E2D3
:10B290000E948EA12AE939E949E15FE3C701B601BD
:10B2A0000F946D0C6B017C019B01AC010F94610943
:10B2B00029813A814B815C810F94CC096FA378A7D7
:10B2C00089A79AA729813A814B815C81C701B60180
:10B2D0000F946D0C20E030E040E05EE30F946D0CC5
:10B2E0006BA77CA78DA79EA782ED91E20E948F9FFE
:10B2F00022E0B701A6018CEC91E20E948EA122E02F
:10B300004FA158A569A57AA586EC91E20E948EA16D
:10B3100022E04BA55CA56DA57EA580EC91E20E9484
:10B320008EA10DCE19862BCEE5960FB6F894DEBF12
:10B330000FBECDBFDF91CF911F910F91FF90EF9086
:10B34000DF90CF90BF90AF909F908F907F906F9045
:10B350005F904F903F902F900895CF93DF930F947D
:10B36000FC03AB01BC0188E191E20E949AA0E0914C
:10B37000E002F0E0EE0FFF1FE65FFD4FC081D181DC
:10B380004F81588569857A8522E085EB93E20E949A
:10B39000CBA14B855C856D857E8520E085EB93E2B6
:10B3A0000E94CBA1E881F0E0EE57F24E608170E0A0
:10B3B00085EB93E2DF91CF910C9474A08091C80744
:10B3C00082FF3CC060E070E083E091E20E9468A0F0
:10B3D000E0910A02F0910B02678170858185928568
:10B3E0000F94650A605171096D31714018F484EE53
:10B3F00090E202C08EEE90E20E948F9F8DE091E27B
:10B400000E94769FE0910C02F0910D026781708599
:10B41000818592850F94650A605171096D31714083
:10B4200018F08EEE90E202C084EE90E20E948F9FB0
:10B4300087EB90E20E94B09F81E0089580E008953C
:10B440002F923F924F925F926F927F928F929F9234
:10B45000AF92BF92CF92DF92EF92FF920F931F9322
:10B46000CF93DF93CDB7DEB72B970FB6F894DEBF3F
:10B470000FBECDBFA8950F94FC0369837A838B839D
:10B480009C832AE032E03B872A8748ED52E05F83C5
:10B490004E8352E35987212C1D82AA85BB850D91CD
:10B4A0001D91BB87AA87211027C020E030E040E231
:10B4B00052E4F80167817085818592850F94C509F2
:10B4C00087FF13C020E030E040E252E4D8011B9631
:10B4D0006D917D918D919C911E970F94C50987FF69
:10B4E00004C0EE81FF81108207C0EE81FF81319799
:10B4F0008081AE81BF818C938091DE02281609F491
:10B50000B8C2C8010E94D4518091C80782FD26C0EC
:10B51000F801C780D084E184F28420E030E040E884
:10B5200051E4C701B6010F94C50987FD0AC020E0A8
:10B5300030E046E953E4C701B6010F94F90B181641
:10B540006CF4809192038F5F809392038B3008F4A8
:10B55000C3C20E94E54D32DFF1E0FD838091C80750
:10B5600082FD87C233243394D8011B962D913D91DF
:10B570004D915C911E9717966D917D918D919C9147
:10B580001A970F94F90B87FD312CB1E03B2641F45B
:10B590007801E0E4EE0EF11CD7018C9180FD9FC292
:10B5A000C980DA80EB80FC80F801E75BFF4F4080C8
:10B5B0005180628073805801B1E4AB0EB11CF5017B
:10B5C00080819181A281B381A7019601281B390B4B
:10B5D0004A0B5B0B421653066406750608F068C0FA
:10B5E000480130E4830E911CD401BC91B8878B2FA5
:10B5F000867009F45DC08091C70786FF59C0B88581
:10B60000B1FF81C27801E5E4EE0EF11CD7012D9166
:10B610003D914D915C91F80167817085818592859E
:10B620000F94600920E030E040E85FE30F94C50923
:10B6300087FF5EC2809192038F5F809392038B306D
:10B64000A8F10E94E54D41E069E978E186E79AE0DA
:10B650000E9499AB82E598E10E94B09FD7012D919D
:10B660003D914D915C91F80167817085818592854E
:10B670000F946009AB01BC0122E08CEE9DE00E94BA
:10B68000CBA149815A816B817C81F50180819181B7
:10B69000A281B381481B590B6A0B7B0B84EE9DE0A2
:10B6A0000E949AA080EE9DE00E948F9FF1E0FD83B2
:10B6B000F80187A5C780D084E184F28424E0829FCA
:10B6C000E00DF11D1124C0AAD1AAE2AAF3AA8F5F4E
:10B6D0008370D8019F968C939F9753968C91539724
:10B6E000813009F0CAC01B968D909D90AD90BC90A2
:10B6F0001E9720E030E040EA51E4C501B4010F9408
:10B70000C50987FDCCC0A7019601C501B4010F94FE
:10B7100060094B015C0120E030E040EA51E40F9405
:10B72000F90B18161CF4F801F6A0D3C020E030E0A5
:10B7300040EA51ECC501B4010F94C50987FDDAC098
:10B74000BE016F5F7F4FC8010E94934DD8015A968A
:10B750002D913D914D915C915D97C501B4010F9480
:10B760006D0C6B017C01F801248935894689578964
:10B77000C501B4010F9461094B015C01D8019B968E
:10B780005C909B979C966C909C979D967C909D97C7
:10B790009E964C90252D362D472D542D0F94C5097E
:10B7A00087FD13C0F80157A060A471A442A4252D01
:10B7B000362D472D542DB401C5010F94F90B1816E1
:10B7C00024F0582C692C7A2C4B2C852D962DA72DE6
:10B7D000B42DF801848B958BA68BB78B268D378D76
:10B7E00040A151A1652D762D872D942D0F946D0CC0
:10B7F0002DEC3CEC4CEC5DE30F946D0C9B01AC012B
:10B80000C701B6010F9461096B017C01D8019F96B5
:10B810008C91F801B4E08B9FE00DF11D1124D8014B
:10B8200017962D913D914D915C911A9760A971A940
:10B8300082A993A90F946009F80122A133A144A120
:10B8400055A10F946D0C2FED3FE445E550E40F94A6
:10B850006D0C9B01AC01C701B6010F9461090F94F7
:10B86000650A77FD47C0D80196962C9130E02617DF
:10B8700037070CF4B901F62E98C0833009F09CC04C
:10B88000F80183849484A584B68420E030E040EA03
:10B8900051E4C501B4010F94C50987FF07C0F80141
:10B8A000E05CFF4F8081897F808324C0A7019601DF
:10B8B000C501B4010F9460096B017C0120E030E008
:10B8C00040EA51E40F94F90B181654F4D8019696F7
:10B8D000FC90BE016F5F7F4FC8010E94694D65C03B
:10B8E00020E030E040EA51ECC701B6010F94C509F1
:10B8F00087FF02C0F12C59C0BE016F5F7F4FC801A6
:10B900000E94934DF801C780D084E184F28420E046
:10B9100030E040E450E464897589868997890F9402
:10B920006D0C4B015C01D8019F968C91F801B4E03D
:10B930008B9FE00DF11D112420A931A942A953A923
:10B94000C701B6010F9460092FED3FE445E550E4CF
:10B950000F946D0C9B01AC01C501B4010F946109FA
:10B9600020E030E040E85EE30F946D0CF801648B5A
:10B97000758B868B978B228D338D448D558D0F94CF
:10B980006D0C9B01AC01C701B6010F946109D80190
:10B990001B962D913D914D915C911E970F94F90B43
:10B9A00018160CF4A7CFF801F08CD801EC91F0E058
:10B9B000EE57F24EF0823DC0823021F589819A81A6
:10B9C000AB81BC81F80147855089618972896C011E
:10B9D0007D01C41AD50AE60AF70A29E8C21623E14E
:10B9E000D206E104F10428F12081E22FF0E0EE57C5
:10B9F000F24E232D21952083F8018787908BA18B10
:10BA0000B28B08C0D801EC91F0E0EE57F24E832DD6
:10BA100081958083332039F0BE016F5F7F4FC8016D
:10BA20000E94694D06C0F801E05CFF4F8081897F6C
:10BA3000808320E030E041E953E4F80167817085BC
:10BA4000818592850F94F90B181634F4D801EC9186
:10BA5000F0E0EE57F24E10828091900390919103A6
:10BA60008B960817190729F4332011F02F9A01C07B
:10BA70002F982394B985BE5CB987EE81FF81ED577D
:10BA8000FF4FFF83EE83F2E02F1207CDCD80C11070
:10BA900007C080919203882319F08150809392030C
:10BAA0008091C80782FF88C0E0910A02F0910B02E2
:10BAB000E081F0E0EE57F24E1082E0910C02F0913E
:10BAC0000D02E081F0E0EE57F24E10828091EA0222
:10BAD00088608093EA0270C021E02D833FCD63E04F
:10BAE00089850E9497A2D7018C918E7F8C9358CD27
:10BAF0008885897FD4018C93BE016F5F7F4FC80119
:10BB00000E94694DD5CDF80123853485458556853C
:10BB100067817085818592850F9460099F7720E009
:10BB200030E040EA51E40F94F90B1816A4F5809127
:10BB300092038F5F809392038B3008F4B7CD0E94FD
:10BB4000E54D41E069E978E186E79AE00E9499AB2A
:10BB500082E598E10E94B09FF801EB5BFF4F4081C6
:10BB600051816281738122E08EEB9DE00E94CBA126
:10BB7000D80117964D915D916D917C911A9722E0B5
:10BB800083EB9DE00E94CBA18BEA9DE00E948F9FFA
:10BB9000B1E0BD838DCDE8EECE0EE3E0DE1EE11C0C
:10BBA000F11CC418D508E608F708D501CD92DD923E
:10BBB000ED92FC9213977CCD2B960FB6F894DEBFD6
:10BBC0000FBECDBFDF91CF911F910F91FF90EF90EE
:10BBD000DF90CF90BF90AF909F908F907F906F90AD
:10BBE0005F904F903F902F9008958FEF8EBD0DB4D2
:10BBF00007FEFDCF8EB50895DC01680F791F80E048
:10BC000090E0A617B70779F02D91E92FFF27E227DB
:10BC1000EE0FFF1FEE51FD4E25913491982F88278E
:10BC200082279327EECF08958EBD0DB407FEFDCF7A
:10BC30000895CF93FB0120E030E22F5F31932B304A
:10BC4000E1F7DC0190E037E02A2FEB2F8D91811195
:10BC50000AC0DA012C931196EC9381E0FB019081EC
:10BC6000903241F526C08F32A1F3282F8E3219F081
:10BC7000E2EEF4E108C03A30E1F098E03AE0E4CFD7
:10BC80003196C817B1F0C491C111FACF391718F025
:10BC900080528F3508F02FE581E0890FFB01E90F15
:10BCA000F11D9FE9920F9A3108F420522083982FBA
:10BCB000CBCF80E0CF9108959B01255F3F4F80E07F
:10BCC000FB019191BF01482F4695F0E88F9F400DF1
:10BCD0001124842F890F6217730791F7089561E08B
:10BCE000FC0180810F9449058FEF9ECFCF93DF93A6
:10BCF000EC018A810E94391D60E08881DF91CF913B
:10BD00000D944905CF92DF92EF92FF920F931F930C
:10BD1000CF93DF93EC018B017A010F94FC036B014D
:10BD200064DF8B838F3F49F40F94FC036C197D090A
:10BD30006D327140A8F381E131C08E3F11F08FE088
:10BD40002DC0E114F104D9F0C70101972FEF2EBDEA
:10BD5000F8014FEF9F01201B310B2817390738F4EA
:10BD60000DB407FEFDCF2EB521934EBDF3CF0DB41C
:10BD700007FEFDCF2EB5F801E80FF91F20831B82C7
:10BD800034DFD82E32DFC82EB701C80135DF2C2DA5
:10BD900030E03D292817390731F08BE18983CE0146
:10BDA0009EDF80E003C0CE019ADF81E0DF91CF917A
:10BDB0001F910F91FF90EF90DF90CF9008950F9318
:10BDC0001F93CF93DF931F921F92CDB7DEB78C01E5
:10BDD00069837A838BDF40E052E069817A81C80110
:10BDE0000F900F90DF91CF911F910F918BCF0F93F9
:10BDF0001F93CF93DF93EB010F94FC038B01F5DED0
:10BE00008F3F49F00F94FC03601B710B6C177D078B
:10BE1000B0F380E001C081E0DF91CF911F910F91DD
:10BE20000895BF92CF92DF92EF92FF920F931F93EC
:10BE3000CF93DF93CDB7DEB72A970FB6F894DEBF66
:10BE40000FBECDBF8C01B62E2F83388749875A8706
:10BE50004DDF6CE271E0C801CADFFE01319686E079
:10BE6000DF011D928A95E9F78B2D806489838A858D
:10BE70008A8389858B8388858C838F818D83CE018E
:10BE80000696DF0120E059E04D9138E0220F642F43
:10BE9000622767FD2527440F3150C1F7A817B9075E
:10BEA00099F7220F21602E837F016E01B7E0CB0E40
:10BEB000D11CF70181917F01B7DEEC14FD04C9F7B5
:10BEC000FCE0BF1201C091DEF12C8FDED801139689
:10BED0008C9387FF05C0BFEFFB1611F0F394F5CFED
:10BEE0002A960FB6F894DEBF0FBECDBFDF91CF917B
:10BEF0001F910F91FF90EF90DF90CF90BF9008952A
:10BF0000BF92CF92DF92EF92FF920F931F93CF9346
:10BF1000DF93EC01B62E1C82198248830F94FC0338
:10BF20008B0161E088810F94100561E088810F9496
:10BF300049052398229A219A209A8BE08A830E94AD
:10BF4000391DE4E1FE2E8FEF6FDEFA94E1F720E079
:10BF500030E0A90160E0CE0164DF813049F00F9448
:10BF6000FC03601B710B613D774088F381E057C093
:10BF700021E030E040E050E06BE3CE0152DF813061
:10BF800011F08AE14CC02AEA31E040E050E068E07C
:10BF9000CE0147DF853011F481E009C074E0F72E4F
:10BFA00024DE8B83FA94E1F78A3A59F482E08C8399
:10BFB0008C81823079F4C12CD12CE12C60E4F62EF6
:10BFC0000CC00F94FC03601B710B613D7740D8F2ED
:10BFD00082E025C0C12CD12C760120E030E0A901FF
:10BFE00067E3CE011EDFA701960169E2CE0119DFEA
:10BFF000882349F00F94FC03601B710B613D77406F
:10C0000060F38AE00CC08C818230B1F420E030E033
:10C01000A9016AE3CE0105DF882329F088E089833E
:10C02000CE015DDE14C0E1DD807C803C11F483E054
:10C030008C83DBDDDADDD9DDCE0151DE8EE08B15C0
:10C0400018F488E1898303C0BA8281E001C080E0EE
:10C05000DF91CF911F910F91FF90EF90DF90CF90E4
:10C06000BF9008950F931F93CF93DF93EC01890145
:10C070008C81833039F0F9E0440F551F661F771F1C
:10C08000FA95D1F79A01AB0161E1CE01CADE8111C7
:10C0900009C040E052E0B801CE01DF91CF911F917D
:10C0A0000F9130CE84E08983CE0119DE80E0DF91EC
:10C0B000CF911F910F910895CF93DF93EC018C8165
:10C0C000833039F089E0440F551F661F771F8A952A
:10C0D000D1F79A01AB0162E1CE01A3DE882331F0F2
:10C0E00085E08983CE01FBDD80E003C0CE01F7DD72
:10C0F00081E0DF91CF910895CF93DF93EC01F6DDDE
:10C1000020E030E0A9016CE0CE018BDE882331F025
:10C1100083E08983CE01E3DD80E003C0CE01DFDD73
:10C1200081E0DF91CF910895CF92DF92EF92FF925D
:10C130000F931F93CF93DF931F92CDB7DEB78C0180
:10C14000E62E6A0160E072E0CA0156DDF82E8E2DFF
:10C1500099836ADDF60180818EBD418122E030E065
:10C1600099810DB407FEFDCF4EBD2115F2E03F07CA
:10C1700039F0F601E20FF31F40812F5F3F4FF1CFFF
:10C180000DB407FEFDCF892F4FDD8F2D4DDD2DDD49
:10C19000F80183838F71853031F083E18183C80199
:10C1A0009EDD80E001C081E00F90DF91CF911F9173
:10C1B0000F91FF90EF90DF90CF9008950F931F9312
:10C1C000CF93DF93EC0189018C81833039F039E022
:10C1D000440F551F661F771F3A95D1F79A01AB019F
:10C1E00068E1CE011EDE882311F086E01EC0A801A2
:10C1F0006EEFCE0199DF8823C9F068E572E0CE01C9
:10C20000F6DD182F811102C087E10FC020E030E079
:10C21000A9016DE0CE0105DE811106C0E6DC8111C9
:10C2200003C0CE015CDD05C086E18983CE0157DD08
:10C2300010E0812FDF91CF911F910F9108950F93FF
:10C240001F93CF93DF93EC018B0150DD68E572E023
:10C25000CE01CDDD882351F0A8016CEFCE0164DF63
:10C26000182F882319F0CE013ADD05C085E18983B6
:10C27000CE0135DD10E0812FDF91CF911F910F911D
:10C2800008958F929F92AF92BF92CF92DF92EF92DA
:10C29000FF920F931F93CF93DF93EC016A017B0111
:10C2A0004801590120E030E0A90167E3BADDA501AA
:10C2B000940167E1CE01B5DD882311F089E012C059
:10C2C0008C81833039F049E0CC0CDD1CEE1CFF1C66
:10C2D0004A95D1F7A701960169E1CE01A2DD882335
:10C2E00031F087E08983CE01FADC80E003C0CE0123
:10C2F000F6DC81E0DF91CF911F910F91FF90EF90DD
:10C30000DF90CF90BF90AF909F908F9008951F9334
:10C31000CF93DF93EC01EADC68E572E0CE0167DDE4
:10C32000882361F08DEF80DC68E572E0CE015FDD8F
:10C33000182F882319F0CE01D2DC05C082E1898351
:10C34000CE01CDDC10E0812FDF91CF911F910895B8
:10C350000F931F93CF938091AF0480FF41C0409112
:10C36000B0045091B1046091B2047091B30424EB15
:10C3700034E08091A9049091AA0420DFC82F811194
:10C3800002C0C0E02EC08091AF0481FD06C0809144
:10C39000AF048E7F8093AF0424C00091AB04109152
:10C3A000AC042091AD043091AE04011511052105B6
:10C3B000310569F34091B0045091B1046091B20429
:10C3C0007091B304400F511F621F731F24EB34E0C0
:10C3D0008091A9049091AA04F1DE8111D8CFD1CF28
:10C3E000C1E08C2FCF911F910F910895CF92DF92D2
:10C3F000EF92FF92CF936B017C01C42F8091B00428
:10C400009091B104A091B204B091B3048C159D0534
:10C41000AE05BF05F9F09CDF811103C080E090E01C
:10C4200021C0C2FF0BC01092AF04C092B004D092E2
:10C43000B104E092B204F092B3040CC024EB34E0F7
:10C44000B701A6018091A9049091AA040BDE811185
:10C45000EACFE4CFC3708091AF048C2B8093AF04FC
:10C4600084EB94E0CF91FF90EF90DF90CF90089510
:10C47000CF93DF93EC01462F6F85788989899A895C
:10C48000B5DF009739F02C8130E2239F800D911D9C
:10C49000112402C080E090E0DF91CF9108950F93C6
:10C4A0001F93CF93DF93EC018B818823D1F1898196
:10C4B00087FF32C061E0CE01DBDF8C01009789F19C
:10C4C000FC018081853E69F18B81823040F44B898B
:10C4D0005C896D897E89448F558F668F778F4F89F0
:10C4E000588D698D7A8DF801538F428F758B648BCF
:10C4F000E091B406F091B506309759F0B8016A5E44
:10C500007F4FC80148961995F801808D918D938BC6
:10C51000828B89818F778983DF91CF911F910F91D2
:10C5200017CF81E0888380E0DF91CF911F910F9139
:10C530000895CF93DF93EC01B2DF1B82DF91CF919F
:10C5400008958FEF9FEFDC018093B0049093B104C6
:10C55000A093B204B093B3041092AF0408958F92E5
:10C560009F92AF92BF92CF92DF92EF92FF920F9382
:10C570001F93CF93DF93EC016A017B018901423065
:10C5800051056105710508F454C089859A85AB850C
:10C59000BC850196A11DB11D84179507A607B70795
:10C5A00008F447C08F89803129F49927872F762F87
:10C5B000652F0BC08032E9F5CB01BA0127E09695D3
:10C5C0008795779567952A95D1F78B889C88AD8854
:10C5D000BE88680D791D8A1D9B1D42E007DF00970C
:10C5E00041F12F89203169F4DD24EE24FF24F60186
:10C5F000EE0FFF1FE80FF91F80819181A0E0B0E0EE
:10C6000011C0E894C7F8DD24EE24FF24F601EE0FF4
:10C61000FF1FEE0FFF1FE80FF91F80819181A2819C
:10C62000B381BF70F80180839183A283B38381E0DB
:10C6300001C080E0DF91CF911F910F91FF90EF90AB
:10C64000DF90CF90BF90AF909F908F9008952F92E2
:10C650003F924F925F927F928F929F92AF92BF9242
:10C66000CF92DF92EF92FF920F931F93CF93DF93BE
:10C67000EC017B016A018B81811103C08FEF9FEF79
:10C6800017C1898180FFFACF4B895C896D897E89CA
:10C690008B859C85AD85BE854601A12CB12C8A0178
:10C6A0009B01081B190B2A0B3B0B80169106A20657
:10C6B000B30618F06A01C81AD90A86014E0127E0AC
:10C6C000820E911C0115110509F46EC02B843C8467
:10C6D0004D845E84510181E0B8228D819E81B2013A
:10C6E000A101E9E07695679557954795EA95D1F7C9
:10C6F000FC0174807A9474222B81223049F4228CBC
:10C70000338C448C558C240E351E461E571E37C064
:10C71000A114B104C1F4711016C0232824282528BF
:10C7200049F48F89988DA98DBA8D8F839887A987B1
:10C73000BA8709C04F81588569857A8594010FDFD2
:10C74000882309F49BCFED81FE81A4812F81388558
:10C7500049855A852250310941095109B0E00F94A9
:10C76000D60D1B012C0186859785A089B189280EDD
:10C77000391E4A1E5B1E270C311C411C511CA11482
:10C78000B104A1F40115F2E01F0780F08091B0041C
:10C790009091B104A091B204B091B3042816390667
:10C7A0004A065B06D9F402C0C60182C040E0C2015D
:10C7B000B1011CDE009709F461CF20E032E02A19B4
:10C7C0003B0928012017310708F42901BC016A0D33
:10C7D0007B1DA201C7010F94DE112AC00115E4E000
:10C7E0001E07B8F1B12EB6942B81223009F040C05B
:10C7F000281639064A065B0608F043C0B201A101BB
:10C800008091A9049091AA0457DC882309F436CFBB
:10C810001701412C8091A9049091AA044B103BC0B0
:10C820006BDC882309F42ACF512C542C4424550C5A
:10C83000E40CF51C8B859C85AD85BE85840D951D0E
:10C84000A11DB11D8B879C87AD87BE870419150973
:10C8500039CF9701B201A1018091A9049091AA0456
:10C8600001DC882309F40ACF412C42E0542EE0CFAA
:10C87000ED81FE81248127192B1508F0B9CFB22E46
:10C88000B7CF8B0D911DA11DB11D281639064A0683
:10C890005B0650F0B3CFB10192DA2EEF321A882343
:10C8A00009F4ECCE4394B6CF53DD8111A7CFE6CE89
:10C8B000DF91CF911F910F91FF90EF90DF90CF907C
:10C8C000BF90AF909F908F907F905F904F903F90E0
:10C8D0002F900895CF93DF931F92CDB7DEB741E03D
:10C8E00050E0BE016F5F7F4FB2DE019719F489817E
:10C8F00090E002C08FEF9FEF0F90DF91CF910895EE
:10C900001F93CF93DF93EC018B81823018F480E08A
:10C9100090E023C04B855C856D857E85A5E076958E
:10C92000679557954795AA95D1F7142F1F70CE019B
:10C93000D1DF97FDECCF4B855C856D857E85415EB3
:10C940005F4F6F4F7F4F4B875C876D877E8720E2FD
:10C95000129FC00111248C549B4FDF91CF911F91E6
:10C960000895AF92BF92CF92DF92EF92FF920F9312
:10C970001F93CF93DF931F92CDB7DEB77C018A015F
:10C980004115510511F0DA011C9241E0BDE0CB2EBA
:10C99000A895C7014983B4DF5C014981009709F478
:10C9A0007AC0FC012081222309F475C0253009F4E6
:10C9B00067C0253E09F464C0FC018385982F9F73EE
:10C9C0009F3009F054C00115110511F3828D938D2C
:10C9D000892BF1F62F71E1F22330D4F6332727FDAE
:10C9E000309521503109C29EF001C39EF00D1124F3
:10C9F000E00FF11FD50111968C911197808313964A
:10CA00008C911397818315968C9115978283179635
:10CA10008C911797838319968C91199784831E960E
:10CA20008C911E97858350968C9150978683529651
:10CA30008C915297878354968C9154978087569601
:10CA40008C915697818758968C91589782875C96DF
:10CA50008C915C9783875E968C915E978487442344
:10CA600009F496CF1D96DC90158640E091CF982F63
:10CA7000967031F42E3261F4F50191819E3241F0CD
:10CA80000115110511F441E083CFD8011C92FBCFB1
:10CA900083FD7ECF03C080E090E011C00115110539
:10CAA00069F0411105C0B501C70106D9D81631F0AA
:10CAB000A501B80182E299E00E94549DC5010F9042
:10CAC000DF91CF911F910F91FF90EF90DF90CF906A
:10CAD000BF90AF9008954F925F926F927F92AF9206
:10CAE000BF92CF92DF92EF92FF920F931F93CF935B
:10CAF000DF93EC016A017B012B81222349F08B89B2
:10CB00009C89AD89BE8984179507A607B70710F4DD
:10CB100080E073C0223049F4CB86DC86ED86FE8649
:10CB20001F82188619861A8667C0C114D104E104D1
:10CB3000F10449F41F82188619861A861B861C8602
:10CB40001D861E8659C08B859C85AD85BE85ED8171
:10CB5000FE81E585F0E03996AC01BD0141505109F7
:10CB6000610971090E2E04C0769567955795479512
:10CB70000A94D2F797018601015011092109310960
:10CB800004C03695279517950795EA95D2F70417AF
:10CB900015072607370720F0892B8A2B8B2B49F4A2
:10CBA0008F89988DA98DBA8D8F839887A987BA8729
:10CBB00004C0041B150B260B370B280139015E013D
:10CBC00087E0A80EB11C411451046104710481F086
:10CBD0004F81588569857A8595018D819E81BFDC5D
:10CBE00091E0491A5108610871088111ECCF05C024
:10CBF000CB86DC86ED86FE8681E0DF91CF911F91AA
:10CC00000F91FF90EF90DF90CF90BF90AF907F900B
:10CC10006F905F904F90089540E050E0BA015BCF75
:10CC2000AF92BF92CF92DF92EF92FF920F931F933A
:10CC3000CF93DF936C01A42E7901E801FC0183817D
:10CC4000823008F43DC0C601E7DFB12CA895C601CB
:10CC500057DE0097B9F1FC012081222399F125309C
:10CC600011F0253E91F7FC0183858F738F3031F1F0
:10CC7000209721F11A1414F5BA1404F108811981CE
:10CC80002A813B81012B022B032BC1F4F601838502
:10CC90009485A585B6858097A109B109FB2D40E251
:10CCA000F40290011124821B930BA109B10988831E
:10CCB0009983AA83BB83F701B08202C0B394C6CF25
:10CCC00081E001C080E0DF91CF911F910F91FF9033
:10CCD000EF90DF90CF90BF90AF900895AF92BF924A
:10CCE000CF92DF92EF92FF920F931F93CF93DF9338
:10CCF00000D01F92CDB7DEB78C01FC018789908DE3
:10CD0000A18DB28D89839A83AB83BC83A12CB12C76
:10CD100049815A816B817C819E012F5F3F4FD801F1
:10CD200015968D919C9116971ADC8823C1F1D80134
:10CD30001596ED91FC9116978481A80EB11CA11453
:10CD4000B0E1BB0658F5C980DA80EB80FC808789AA
:10CD5000803149F481E0E8EFCE16EFEFDE06E10422
:10CD6000F10450F4D5CF81E0F8EFCF16FFEFDF06E6
:10CD7000EF06FFE0FF0660F2A50160E070E099E0D9
:10CD8000440F551F661F771F9A95D1F7D801539608
:10CD90004D935D936D937C93569701C080E00F9007
:10CDA0000F900F900F90DF91CF911F910F91FF90F7
:10CDB000EF90DF90CF90BF90AF900895CF93DF9327
:10CDC000EC01FB018B81882311F080E03BC07E8366
:10CDD0006D838789803101F18032B9F783E08B83DD
:10CDE000428D538D648D758D4F8B588F698F7A8FDF
:10CDF000CE0174DF882349F381E089831F8218867E
:10CE000019861A861B861C861D861E861F86188A12
:10CE1000198A1A8A1C8216C082E08B831F8A188E98
:10CE2000198E1A8E408D518D60E070E025E0440F20
:10CE3000551F661F771F2A95D1F74B8B5C8B6D8B27
:10CE40007E8BDACFDF91CF9108950F931F93CF930D
:10CE5000DF938C01EC01A396662321F0D093B706F3
:10CE6000C093B606F80186A1882311F0CE0161DBDC
:10CE7000B8016B5F7F4FCE01DF91CF911F910F9172
:10CE80009DCF8F929F92AF92BF92CF92DF92EF92FF
:10CE9000FF920F931F93CF93DF93EC016A017B0105
:10CEA00048015901423051056105710508F44DC032
:10CEB00049855A856B857C854F5F5F4F6F4F7F4FEC
:10CEC0004C155D056E057F0508F43FC08F898031E4
:10CED00029F499278F2D7E2D6D2D0BC08032A9F559
:10CEE000C701B60157E096958795779567955A954E
:10CEF000D1F70B891C892D893E89600F711F821F14
:10CF0000931F43E073DA009701F12F89203159F420
:10CF1000DD24EE24FF24F601EE0FFF1FE80FF91FBA
:10CF20009182808210C0E894C7F8DD24EE24FF24AB
:10CF3000F601EE0FFF1FEE0FFF1FE80FF91F8082B3
:10CF40009182A282B38281E001C080E0DF91CF9123
:10CF50001F910F91FF90EF90DF90CF90BF90AF9017
:10CF60009F908F9008952F923F924F925F926F9271
:10CF70007F928F929F92AF92BF92CF92DF92EF9269
:10CF8000FF920F931F93CF93DF93CDB7DEB72F9709
:10CF90000FB6F894DEBF0FBECDBF1C014C875D8776
:10CFA0006E877F873B872A87DC0119960D911D913B
:10CFB0002D913C911C970F5F1F4F2F4F3F4F0D83BB
:10CFC0001E832F833887EA85FB8580809180A2802D
:10CFD000B38081149104A104B10431F0FFEF8F1AE2
:10CFE0009F0AAF0ABF0A10C0DC018D909D90AD90E2
:10CFF000BC90B1E0B9870C851D852E853F85013039
:10D0000011052105310509F0198675016401412CCE
:10D01000512C3201F10181859285A385B485481692
:10D0200059066A067B0608F04EC00D811E812F81CD
:10D0300038850C151D052E053F0550F472E0C72EEE
:10D04000D12CE12CF12CE2E08E2E912CA12CB12CD4
:10D050009E012F5F3F4FB701A601C10180DA8823EF
:10D0600091F149815A816B817C81D701C60101967A
:10D07000A11DB11D452B462B472B19F04C015D011D
:10D080000FC0AC01BD01481959096A097B090C851B
:10D090001D852E853F85401751076207730741F0B4
:10D0A0001FEF411A510A610A710A6C017D01B2CF6A
:10D0B0000FEF1FEF2FEF3FE0B701A601C101E1DE47
:10D0C0008D83811113C01D823DC02601370121E0EF
:10D0D000421A51086108710897018601B301A20143
:10D0E000C101CFDE882379F3730162018C149D04A2
:10D0F000AE04BF0450F3AA85BB854D915D916D913F
:10D100007C914115510561057105A9F4EA85FB85FE
:10D1100080829182A282B382F985FF2399F00FEF7A
:10D12000801A900AA00AB00AD1018D929D92AD9208
:10D13000BC92139707C095018401C101A2DE811141
:10D14000E5CFC1CF8D812F960FB6F894DEBF0FBE0D
:10D15000CDBFDF91CF911F910F91FF90EF90DF90A6
:10D16000CF90BF90AF909F908F907F906F905F9087
:10D170004F903F902F900895CF93DF93EC019C0147
:10D18000295F3F4F41E050E060E070E08D819E817B
:10D19000EADE882399F04F89588D698D7A8D452B69
:10D1A000462B472B59F44F81588569857A854F8BDB
:10D1B000588F698F7A8F998190689983DF91CF9189
:10D1C00008952F923F924F925F926F927F928F922B
:10D1D0009F92AF92BF92CF92DF92EF92FF920F9306
:10D1E0001F93CF93DF93CDB7DEB728970FB6F89490
:10D1F000DEBF0FBECDBF7C015B014A01DC01119691
:10D200008C9181FFB0C182FD02C064018DC0F70125
:10D21000438954896589768983859485A585B685F2
:10D2200084179507A607B70781F3C70154DC81115E
:10D23000ECCF99C1D70115968D919C911697FC0161
:10D2400034803A94B901A80129E0769567955795FD
:10D2500047952A95D1F734221170332009F470C014
:10D26000D70113968C9113971596ED91FC91169713
:10D27000823009F0A9C01B964D905D906D907C9016
:10D280001E9789E076946794579447948A95D1F7CE
:10D29000828D938DA48DB58D480E591E6A1E7B1EFE
:10D2A0000115110509F4AFC080E092E0801B910BDD
:10D2B00016018C159D0508F41C010115110509F0D6
:10D2C000A7C0F70143855485658576858389948950
:10D2D000A589B689481759076A077B0708F498C0DB
:10D2E00045E0C301B20182D8009709F43CC1A10115
:10D2F000B501800F911F0F94DE11020D131D011552
:10D30000124009F487C0F70183859485A585B68509
:10D31000820D931DA11DB11D83879487A587B687B4
:10D32000A20CB31CC218D308D7011B960D911D91F6
:10D330002D913C911E97C114D10409F07BCFE7C019
:10D340000115110509F08CCF17964D915D916D91E6
:10D350007C911A97411551056105710509F19E01EE
:10D360002F5F3F4FFCD8882309F4FDC089819A8143
:10D37000AB81BC81F70125813681F90127892031F4
:10D3800039F4883FFFEF9F07A105B10590F416C05F
:10D39000883F2FEF9207A2072FE0B20778F009C06D
:10D3A000F7018789908DA18DB28D0097A105B105F8
:10D3B00029F4C701E1DE811153CFD5C0F70187837E
:10D3C0009087A187B2874CCF8481D70117962D9182
:10D3D0003D914D915C911A972250310941095109B3
:10D3E000A82FB0E00F94D60D2B013C0186859785C0
:10D3F000A089B189480E591E6A1E7B1E430C511C20
:10D40000611C711C4DCFC114B2E0DB0640F44CCF5F
:10D4100041E067CF0E94A861811175CFA4C0C114FB
:10D4200024E0D206F0F48091B0049091B104A09170
:10D43000B204B091B30484159505A605B70509F4A7
:10D4400080D89501B301A2018091A9049091AA040A
:10D450000E94DE60882309F486C0212CA2E03A2EC7
:10D4600052CF848183193D2C3694831508F4382ECD
:10D47000032D10E020E030E0B301A2018091A90467
:10D480009091AA040E944161882309F46CC085012F
:10D490004D825E826F8278868D818419831548F56E
:10D4A0008091B0049091B104A091B204B091B30402
:10D4B0002D813E814F815885281739074A075B0720
:10D4C00009F43FD8B8018091A9049091AA040E9460
:10D4D0001F611E5F2D813E814F8158852F5F3F4F19
:10D4E0004F4F5F4F2D833E834F8358878111D4CF99
:10D4F0003AC08091A9049091AA040E948761882370
:10D5000091F1232C312C322C2224330CFCCE539657
:10D510008D919D910D90BC91A02DF70141818017B7
:10D520009107A207B30738F4038B148B258B368B36
:10D53000406841830CC08091B4069091B506892B58
:10D5400031F08114910419F04068F7014183D7014B
:10D5500011968C9183FD02C0C4010AC0C7010E94CC
:10D560004F628111F9CF81E0F70180838FEF9FEF48
:10D5700028960FB6F894DEBF0FBECDBFDF91CF91D6
:10D580001F910F91FF90EF90DF90CF90BF90AF90E1
:10D590009F908F907F906F905F904F903F902F90D3
:10D5A0000895AF92BF92CF92DF92EF92FF920F93C6
:10D5B0001F93CF93DF9300D01F92CDB7DEB75C01EE
:10D5C0006A017B0182E090E0A0E0B0E0F501808399
:10D5D0009183A283B3839E012F5F3F4FB701A601C2
:10D5E000C5010E94AF62811102C080E023C000E04B
:10D5F00010E09801B701A601C50143DC8823A9F317
:10D60000C980DA80EB80FC80F5018789803149F49C
:10D6100081E0F8EFCF16FFEFDF06E104F10450F4EC
:10D62000DACF81E098EFC9169FEFD906E9069FE0AF
:10D63000F90688F20F900F900F900F90DF91CF9125
:10D640001F910F91FF90EF90DF90CF90BF90AF9020
:10D6500008954F925F926F927F92AF92BF92CF9256
:10D66000DF92EF92FF920F931F93CF93DF9300D03F
:10D670001F92CDB7DEB75C016A017B01FC0183819B
:10D680008130E9F4818181FF1AC0F5018389948991
:10D69000A589B68984179507A607B70780F0892B57
:10D6A0008A2B8B2B09F474C0F50143845484658460
:10D6B0007684B701A601C5010EDA811102C080E0AF
:10D6C00068C0F50185819681C114D104E104F1049B
:10D6D00069F44789508D618D728D63DF882379F3FA
:10D6E000F501178A108E118E128E38C0F501478110
:10D6F0005085618572859E012F5F3F4F0E94AF620A
:10D700008823E9F249815A816B817C81F501858109
:10D710009681FC012789203139F4483FFFEF5F07EC
:10D7200061057105D8F407C0483F2FEF5207620723
:10D730002FE0720798F435DF882309F4C0CFF50194
:10D7400047815085618572850FEF1FEF2FEF3FE016
:10D750008581968196DB882309F4B1CFF501C38AD0
:10D76000D48AE58AF68A818180688183C5010E9416
:10D770004F62882309F4A3CFB701A6014C145D04BE
:10D780006E047F0410F4B301A201C501A4D901C045
:10D7900081E00F900F900F900F90DF91CF911F912C
:10D7A0000F91FF90EF90DF90CF90BF90AF907F9060
:10D7B0006F905F904F900895BF92CF92DF92EF925B
:10D7C000FF920F931F93CF93DF93EC01B42E80E26F
:10D7D000689FF0011124EC54FB4F8091B0049091AC
:10D7E000B104A091B204B091B3048F87988BA98B38
:10D7F000BA8B6C830489158920E030E098011127E9
:10D800000027C28CD38CE12CF12C0C291D292E2948
:10D810003F290F8B188F298F3A8F8385887151F498
:10D82000048D158D268D378D0B8B1C8B2D8B3E8B90
:10D8300081E00BC08031F1F4CE0150DA811104C0D7
:10D840001B8A1C8A1D8A1E8A84E08B838B2D8F7015
:10D8500089831F82188619861A861B861C861D8658
:10D860001E86B4FE0AC040E050E0BA01CE01F1DEEF
:10D87000811103C01B8280E012C0B5FE0FC04B892E
:10D880005C896D897E89CE01DF91CF911F910F91C7
:10D89000FF90EF90DF90CF90BF901DC981E0DF91A6
:10D8A000CF911F910F91FF90EF90DF90CF90BF909D
:10D8B0000895DF92EF92FF920F931F93CF93DF9320
:10D8C0008C01EB017A01D22E8D819E81F801968325
:10D8D00085838381811128C0209731F127FD24C0E1
:10D8E000A70165E0440F551F6A95E1F760E070E01D
:10D8F000CE01F1D88823C1F0CE0102D80097A1F063
:10D90000FC018081882381F0853E71F08E3261F0C8
:10D910006E2D6F704D2DC801DF91CF911F910F912A
:10D92000FF90EF90DF9048CF80E0DF91CF911F9183
:10D930000F91FF90EF90DF9008952F923F924F92BA
:10D940005F926F927F928F929F92AF92BF92CF928F
:10D95000DF92EF92FF920F931F93CF93DF93CDB798
:10D96000DEB7C454D1090FB6F894DEBF0FBECDBFE9
:10D970004C017B016A01422E302E1EAA1FAA18AE4E
:10D9800019AEDB0115968D919C911697F401968343
:10D990008583CB0141D946FE1AC0F60101900020D3
:10D9A000E9F73197EC1977247394E9300CF0712C76
:10D9B0008E2F6DE00F94430D21E0911101C020E006
:10D9C0008E2F6DE00F94430D582E520E03C0552438
:10D9D0005A94712C8E010A5C1F4F252D44EE59E09C
:10D9E000B501C7010E94B1645C01009779F1A89567
:10D9F000D7011B968D919D910D90BC91A02D2396E2
:10DA00008CAF9DAFAEAFBFAF2397B60184EE99E068
:10DA10000E946B9D8111DECF47FE02C080E08FC166
:10DA200023968CAD9DADAEADBFAD23974F97A109A9
:10DA3000B109F5E0B695A79597958795FA95D1F731
:10DA4000682F6F70442DC401B7DE79C1842D8274B4
:10DA5000823421F79E01265C3F4F452DFE01319611
:10DA60005F01BF01C701DCD88EA99FA9A8ADB9ADE0
:10DA7000892B8A2B8B2BA9F4D70113962C91139702
:10DA80001B968D919D910D90BC91A02D223009F097
:10DA900046C18115E0E49E07A105B10508F0BECF9F
:10DAA0003EC122242394D70111968C911197826054
:10DAB00011968C934EA95FA968AD79ADC7010BD8BB
:10DAC000711037C06EE270E0C6010F94F2113C0194
:10DAD00086010A5F1F4F009761F044E050E0BC01EF
:10DAE000CE01C1960F940D121DAA0615170518F444
:10DAF00001C019AA38016C187D087724A301B6016A
:10DB0000CE0181960F94DE11E1E2F0E0EC0FFD1FF3
:10DB1000E60DF71D108263E673E0CE0181960F9447
:10DB2000E711BE016F5C7F4FCE0181960F94E71124
:10DB300005C0B601CE0181960F940612AE014F5C6E
:10DB40005F4FB501CE0181960E94195EB501C401F7
:10DB50000E945C5E782EF60101900020E9F78F01AB
:10DB6000015011090C191D09652C252D332727FD9E
:10DB7000309525963FAF2EAF259711279E01215F47
:10DB80003F4F3CAF2BAF225F3F4F3EAF2DAF6620E4
:10DB900009F460C0862D90E0BC01615071093DE040
:10DBA000639F602D1124D501E0E21D92EA95E9F70B
:10DBB0002FE02C8725962EAD3FAD25978217930732
:10DBC00011F480E401C080E08629898340E050E0C0
:10DBD000FE01329670E0C601860F971F21969FAF17
:10DBE0008EAF2197CF0102969A01260F371F021799
:10DBF000130734F49C01AFEFBFEFB183A0830DC0D6
:10DC00009C012196AEADBFAD2197A40FB51F8C919D
:10DC1000992787FD909591838083443029F04A307D
:10DC200029F42DAD3EAD02C02BAD3CAD4F5F5F4F33
:10DC30004D30510511F0F901D5CF7E8640E250E01C
:10DC4000B501C701BEDA97FDE9CEC7010E944F6258
:10DC50006A949DCF80E2F50111928A95E9F7AE01B1
:10DC60004F5C5F4FB501CE0181960E94195E332053
:10DC700011F080E101C080E28C8781E298E29A8B0A
:10DC8000898B20E038E0388B2F879C8B8B8B9A8F89
:10DC9000898F388F2F8B40E250E0B501C70191DAB0
:10DCA00097FDBCCEC7010E944F6280E2D5011D9254
:10DCB0008A95E9F7222011F085EE8983D12C052D74
:10DCC000112707FD10958AAD992787FD9095801B38
:10DCD000910B2D2D332727FD30952817390764F434
:10DCE00040E250E0B501C7016CDA97FD97CEC7015D
:10DCF0000E944F62D394E7CF242D2F774EA95FA9BE
:10DD000068AD79ADE5E07695679557954795EA95C5
:10DD1000D1F7400F511FB701C401CBDD10C021E086
:10DD2000250D2AAF0097A105B10539F08097A1090B
:10DD3000B1098EAB9FABA8AFB9AF212CB4CECC5BF1
:10DD4000DF4F0FB6F894DEBF0FBECDBFDF91CF918E
:10DD50001F910F91FF90EF90DF90CF90BF90AF9009
:10DD60009F908F907F906F905F904F903F902F90FB
:10DD70000895BF92CF92DF92EF92FF920F931F937D
:10DD8000CF93DF93CDB7DEB7A0970FB6F894DEBF81
:10DD90000FBECDBF7C016B01FB018381823088F116
:10DDA00001E023ECC701C9DDB82E882351F18E01B3
:10DDB0000F5F1F4F80E2F80111928A95E9F721E287
:10DDC00038E23A8B298B80E098E0988B8F873C8BE8
:10DDD0002B8B3A8F298F988F8F8B8EE2898380E1EE
:10DDE0008C87FE013296CE010C9620E22193E81733
:10DDF000F907E1F740E250E0B801C701E2D997FF27
:10DE000002C0B12C37C0C7010E944F628EE28A83E4
:10DE1000F60183818250823028F41C8E1B8E1E8A6C
:10DE20001D8A09C0F6014789508D618D728D5C8F06
:10DE30004B8F7E8B6D8B40E250E0B801C701C1D99A
:10DE400097FDDFCFC7010E944F6280E2F801119277
:10DE50008A95E9F740E250E0B801C701B2D997FDD1
:10DE6000D0CFC7010E944F6284E0F7018383818194
:10DE7000806881838B2DA0960FB6F894DEBF0FBE0D
:10DE8000CDBFDF91CF911F910F91FF90EF90DF9069
:10DE9000CF90BF9008952F923F924F925F926F92D2
:10DEA0007F928F929F92AF92BF92CF92DF92EF922A
:10DEB000FF920F931F93CF93DF93CDB7DEB7C1547B
:10DEC000D1090FB6F894DEBF0FBECDBF4B016A017A
:10DED00039011801EFAE1E8E19A219821C82F901B8
:10DEE00010826115710511F480E08AC0FC01838104
:10DEF0008111FACFFA0180818F3261F4CA016C017D
:10DF00000196F60120812F32D1F3F40183818250F2
:10DF1000823010F454010CC0F40165817681CE0189
:10DF200001960E94DE668823F9F2CE0101965C011B
:10DF30007E019EE1E90EF11CFCAEEBAEFE013196D6
:10DF4000FEAFEDAF2196EFAE21972296FFAE22975E
:10DF500034C092012C193D09022F112707FD10959D
:10DF6000A801B601C3010F94DE11F301E00FF11F08
:10DF70001082F20181818823D9F100E021E0A30120
:10DF8000B501C701DADC882309F1A814B90419F036
:10DF9000C5010E9499628BAD9CADE816F90609F1A6
:10DFA00021969FAD219722968FAD22976201EFEFC8
:10DFB000CE1ADE0A5701E92EF82E6FE270E0C60194
:10DFC0000F94F2112C01009721F60EC0FFADFF2334
:10DFD00009F48ACFA301B501C701CBDE8111D5CFEA
:10DFE00083CF9DAD8EADE2CFB601C3010F94061273
:10DFF0008DE1F501D10101900D928A95E1F781E063
:10E00000CF5BDF4F0FB6F894DEBF0FBECDBFDF9101
:10E01000CF911F910F91FF90EF90DF90CF90BF9025
:10E02000AF909F908F907F906F905F904F903F90B8
:10E030002F900895CF92DF92EF920F931F93CF937B
:10E04000DF93CDB7DEB7E9970FB6F894DEBF0FBE0A
:10E05000CDBF6C0119821C82E22E8E010F5F1F4F13
:10E060009E01225E3F4F17DF882339F0AE01425EEA
:10E070005F4FB801C6017DDE01C080E0E9960FB6B2
:10E08000F894DEBF0FBECDBFDF91CF911F910F91EE
:10E09000EF90DF90CF900895CF93DF93CDB7DEB7A9
:10E0A0006D970FB6F894DEBF0FBECDBF242F198237
:10E0B0001C828396AB01BC01CE010196BBDF6D963D
:10E0C0000FB6F894DEBF0FBECDBFDF91CF9108959C
:10E0D000CF92DF92EF92FF920F931F93CF93DF9334
:10E0E000CDB7DEB7E9970FB6F894DEBF0FBECDBF50
:10E0F0006C01F22E19821C82E12C8E010F5F1F4FE2
:10E100009E01225E3F4FC7DE882371F08E8D8823EB
:10E1100069F000E02F2DAE01425E5F4FBE016F5FE0
:10E120007F4FC6010ADC03C080E001C081E0E996B0
:10E130000FB6F894DEBF0FBECDBFDF91CF911F9118
:10E140000F91FF90EF90DF90CF900895FF920F9383
:10E150001F93CF93DF93CDB7DEB76D970FB6F894CB
:10E16000DEBF0FBECDBFFB01F42E19821C822081C1
:10E170002F3239F42181211104C0642F0E942567B8
:10E180001EC08C010D5D1F4F21E0AF01B801CE0113
:10E1900001969EDF882399F09C81923078F09DE172
:10E1A000FE013196D80101900D929A95E1F7FF207A
:10E1B00031F01093B7060093B60601C080E06D966B
:10E1C0000FB6F894DEBF0FBECDBFDF91CF911F9188
:10E1D0000F91FF900895FB01242F6091B606709176
:10E1E000B706AF0175CFCF93DF93EC0140E050E06D
:10E1F000BA012FDA882371F061E0CE010E94386203
:10E20000009741F025EEFC0120831B82DF91CF9126
:10E210000C94A86180E0DF91CF910895CF93DF93B4
:10E22000CDB7DEB76D970FB6F894DEBF0FBECDBF8A
:10E23000AB0119821C8222E0BC01CE01019648DFAD
:10E24000882319F0CE010196CEDF6D960FB6F894B3
:10E25000DEBF0FBECDBFDF91CF9108958396DECF95
:10E260000F931F93CF93DF93EC018B81843061F583
:10E27000CE010E940C660B851C852D853E854B8941
:10E280005C896D897E89041715072607370748F4CE
:10E29000CE010E9480640097B9F0FC012081211119
:10E2A0000BC081E08B83898182608983CE01DF91FD
:10E2B000CF911F910F9197CF253EE9F22E32D9F2DF
:10E2C000FC01838583FDD7CF80E0DF91CF911F9143
:10E2D0000F910895CF93DF93CDB7DEB76D970FB64B
:10E2E000F894DEBF0FBECDBF19821C8241E0CE0183
:10E2F000019671DF882319F0CE010196B1DF6D968A
:10E300000FB6F894DEBF0FBECDBFDF91CF91089559
:10E310004F925F926F927F92AF92BF92CF92DF92B5
:10E32000EF92FF920F931F93CF93DF93EC01142F83
:10E330007093AA046093A9041F8A82E090E0A0E091
:10E34000B0E088839983AA83BB831092AF048FEFD8
:10E350009FEFDC018093B0049093B104A093B204CA
:10E36000B093B3041092AB041092AC041092AD04BD
:10E370001092AE04442361F1453008F0D6C040E06D
:10E3800060E070E0CB010E94F661009709F4CDC017
:10E39000FC0120E1129FE00DF11D1124E255FE4F1A
:10E3A00080818F7709F0C1C0448555856685778562
:10E3B000443651056105710508F4B7C0C084D184A5
:10E3C000E284F384C114D104E104F10421F4ADC06A
:10E3D000C12CD12C760140E0C701B6010E94F66144
:10E3E000FC01009709F4A1C08385948581159240B2
:10E3F00009F09BC02089222309F497C08685978560
:10E40000892B09F492C08585882309F48EC02A8B54
:10E4100025852C831D8630E041E050E06D85062F78
:10E42000CA01062E02C0880F991F0A94E2F7281726
:10E43000390731F081E0860F8D87683078F375C039
:10E44000268937892115310519F040E050E004C0D4
:10E4500024A135A146A157A12D833E834F83588720
:10E460002093AB043093AC044093AD045093AE04BE
:10E470008685978526013701480E591E611C711C3F
:10E480004B8A5C8A6D8A7E8AA188B288B98EA88EF2
:10E49000A089B0E00F94D60D640D751D861D971DE3
:10E4A0006A8F7B8F8C8F9D8F15E0AA0CBB1C1A95F1
:10E4B000E1F741E0A41A4EEFB40AAB2CBB24A694BA
:10E4C000DC01CB018A0D9B1DA11DB11D8E879F878D
:10E4D000A88BB98B438854884114510419F0612CDE
:10E4E000712C04C040A051A062A073A0A7019601A6
:10E4F000281B390B4A0B5B0BDA01C901840D951DF2
:10E50000A61DB71D04C0B695A795979587950A9542
:10E51000D2F789879A87AB87BC87853F3FE093070F
:10E52000A105B10520F48CE08F8B80E012C0853FFF
:10E530009F4FA105B10510F480E109C084A595A500
:10E54000A6A5B7A58A8F9B8FAC8FBD8F80E28F8BDE
:10E5500081E0DF91CF911F910F91FF90EF90DF90BD
:10E56000CF90BF90AF907F906F905F904F90089545
:10E570000F931F93CF93DF93EC01842F462F682FC7
:10E58000CE010E94805F8823B9F08E010B5F1F4F80
:10E5900041E0BE01C801BCDE882341F061E0CE014C
:10E5A000DF91CF911F910F910C94256740E0BE0140
:10E5B000C801AEDE8111F2CF80E0DF91CF911F91D3
:10E5C0000F9108950C94E168682F8AE39BE00C9406
:10E5D0006FD92F923F924F925F926F927F928F925C
:10E5E0009F92AF92BF92CF92DF92EF92FF920F93E2
:10E5F0001F93CF93DF93CDB7DEB76D970FB6F89427
:10E60000DEBF0FBECDBF7B01342E59014801CB01C7
:10E610000E940C66C12CD12C22242394230C00E0F0
:10E6200010E020E044EE59E0B601C7010E94B16459
:10E630006C01009739F0A895D6011B961C9113FF29
:10E6400003C0EDCF80E0C2C068E673E084EE99E0DD
:10E650000F94FD11892B19F31871103109F067C05F
:10E66000B1E0B315E0F2A114B10491F4332041F00C
:10E670008BEA99E00E94BA9F86E294E20E94769F1C
:10E6800084EE99E00E94BA9F86E294E20E948F9FF6
:10E6900019821C82332031F066E673E08BEA99E040
:10E6A0000F94E71164EE79E08BEA99E00F94E7119B
:10E6B000F7014384548465847684FFE14F1A51083E
:10E6C0006108710845E076946794579447944A9599
:10E6D000D1F721E0A201B701CE010196EAD8882343
:10E6E00051F084019501422DBE016F5F7F4FCB0138
:10E6F00070DF81116AC08FEF481A580A35E0440C68
:10E70000551C3A95E1F7A20160E070E0C7010E9454
:10E710006B656FE270E08BEA99E00F941C12009732
:10E7200019F0DC011C927BCF1092AB0978CFA114B9
:10E73000B10489F1EBEAF9E0DF010D900020E9F77F
:10E740008D01015011090B5A1940702E402F552789
:10E7500047FD5095B501CF010E94A89D81115FCF63
:10E7600010161CF477247394700EB501670D711D9B
:10E7700077FC7A9584EE99E00E946B9D81114FCFD2
:10E780008114910411F18DE1F701D40101900D92F2
:10E790008A95E1F71AC0332041F08BEA99E00E9494
:10E7A000BA9F86E294E20E94769F84EE99E00E94EE
:10E7B000BA9FF601448D558D668D778D85EB93E27A
:10E7C0000E949AA00E9410242ACF81E06D960FB675
:10E7D000F894DEBF0FBECDBFDF91CF911F910F9197
:10E7E000FF90EF90DF90CF90BF90AF909F908F9071
:10E7F0007F906F905F904F903F902F900895EF9291
:10E80000FF920F931F93CF93DF93CDB7DEB76D9732
:10E810000FB6F894DEBF0FBECDBF7C0119821C82FB
:10E820000E940C66EBEAF9E01082D7015C96FC933B
:10E83000EE935B978DE1F701DE01119601900D9249
:10E840008A95E1F700E010E020E030E040E0BE0112
:10E850006F5F7F4FC701BDDE6D960FB6F894DEBFC8
:10E860000FBECDBFDF91CF911F910F91FF90EF9021
:10E870000895882321F080910B018D7F03C0809142
:10E880000B01826080930B010895882321F0809111
:10E890000B01816003C080910B018E7F80930B017F
:10E8A0000895882321F080910B018B7F03C0809114
:10E8B0000B01846080930B010895FB01DC018091C2
:10E8C0005108882349F023E333E34BEC51E4CD01B5
:10E8D0000F946D0CFB01DC01BF01CD010895CF93B6
:10E8E000DF931F92CDB7DEB79091C80790FF02C0AB
:10E8F000811143C02091C70723FD3FC091609093D1
:10E90000C807179A169A159A89830E94C851898157
:10E91000811125C020E040E060E070E0CB010E9462
:10E920002E5520E041E060E070E0CB010E942E55C2
:10E9300040E060E070E0CB010E94F75540E069E8FC
:10E9400077E186E79AE00E9499AB86E79AE00E9419
:10E95000EDAE8091C70788608093C7070EC040E086
:10E9600068E777E186E79AE00E9499AB86E79AE04C
:10E970000F90DF91CF910C94EDAE0F90DF91CF917E
:10E980000895CF93C091C807CD7FC093C80720E0FA
:10E9900030E0A90160918002709181028091820231
:10E9A000909183020F94C509882319F0C260C09327
:10E9B000C807CF9108952F923F924F925F926F9226
:10E9C0007F928F929F92AF92BF92CF92DF92EF92FF
:10E9D000FF920F931F93CF93DF93CDB7DEB76D9761
:10E9E0000FB6F894DEBF0FBECDBF8BE793E00F9458
:10E9F000441290934E0780934D0789E793E00F945C
:10EA0000441290934C0780934B07C0902F03D090F3
:10EA10003003E0903103F0903203C0922B03D09288
:10EA20002C03E0922D03F0922E03C0922703D09284
:10EA30002803E0922903F0922A0380910303909126
:10EA40000403A0910503B09106038093FF02909305
:10EA50000003A0930103B09302038093FB02909301
:10EA6000FC02A093FD02B093FE02809113039091EB
:10EA70001403A0911503B091160380930F03909394
:10EA80001003A0931103B093120380930B03909390
:10EA90000C03A0930D03B0930E0380911F0390917C
:10EAA0002003A0912103B091220380931B03909334
:10EAB0001C03A0931D03B0931E0380931703909330
:10EAC0001803A0931903B0931A038091F302909155
:10EAD000F402A091F502B091F6028093EF029093B8
:10EAE000F002A093F102B093F2028093EB029093B4
:10EAF000EC02A093ED02B093EE0220910B0730914F
:10EB00000C0740910D0750910E07C701B6010F94F5
:10EB10006D0C0F94650A60932B0770932C078093FC
:10EB20002D0790932E0720911707309118074091D9
:10EB3000190750911A07C701B6010F946D0C0F9475
:10EB4000650A60932707709328078093290790939D
:10EB50002A0720910F07309110074091110750911B
:10EB60001207C701B6010F946D0C0F94650A6093EC
:10EB700023077093240780932507909326072091FD
:10EB80000707309108074091090750910A07C7010C
:10EB9000B6010F946D0C0F94650A60931F07709374
:10EBA00020078093210790932207C0907707D09089
:10EBB0007807E0907907F0907A0781E993E00E9466
:10EBC000211D9B01AC01C701B6010F9461092B0106
:10EBD0003C01C0907707D0907807E0907907F090DB
:10EBE0007A0785E993E00E94211D9B01AC01C701D2
:10EBF000B6010F9461094B015C01C0907707D0907A
:10EC00007807E0907907F0907A0789E993E00E940D
:10EC1000211D9B01AC01C701B6010F9461096B0175
:10EC20007C0185E893E00E94211D2BED3FE049E443
:10EC300050E40F946D0C20E030E044E353E40F9473
:10EC4000CC090F94C9099B01AC01C301B2010F9417
:10EC50006D0C20912F03309130034091310350917E
:10EC600032030F946D0C20E030E040E05FE30F943E
:10EC700061090F94D30A0F94650A60936F0770932C
:10EC80007007809371079093720785E893E00E9464
:10EC9000211D2BED3FE049E450E40F946D0C20E082
:10ECA00030E044E353E40F94CC090F94D00C9B0163
:10ECB000AC01C301B2010F946D0C20912F03309170
:10ECC000300340913103509132030F946D0C20E0DA
:10ECD00030E040E05FE30F9461090F94D30A0F9492
:10ECE000650A60936B0770936C0780936D07909330
:10ECF0006E0789E893E00E94211D2BED3FE049E477
:10ED000050E40F946D0C20E030E044E353E40F94A2
:10ED1000CC090F94C9099B01AC01C501B4010F9442
:10ED20006D0C20912F0330913003409131035091AD
:10ED300032030F946D0C20E030E040E05FE30F946D
:10ED400061090F94D30A0F94650A60936707709363
:10ED500068078093690790936A0789E893E00E94A7
:10ED6000211D2BED3FE049E450E40F946D0C20E0B1
:10ED700030E044E353E40F94CC090F94D00C9B0192
:10ED8000AC01C501B4010F946D0C20912F0330919B
:10ED9000300340913103509132030F946D0C20E009
:10EDA00030E040E05FE30F9461090F94D30A0F94C1
:10EDB000650A609363077093640780936507909377
:10EDC00066078DE893E00E94211D2BED3FE049E4AA
:10EDD00050E40F946D0C20E030E044E353E40F94D2
:10EDE000CC090F94C9099B01AC01C701B6010F946E
:10EDF0006D0C20912F0330913003409131035091DD
:10EE000032030F946D0C20E030E040E05FE30F949C
:10EE100061090F94D30A0F94650A60935F0770939A
:10EE2000600780936107909362078DE893E00E94EA
:10EE3000211D2BED3FE049E450E40F946D0C20E0E0
:10EE400030E044E353E40F94CC090F94D00C9B01C1
:10EE5000AC01C701B6010F946D0C20912F033091C6
:10EE6000300340913103509132030F946D0C20E038
:10EE700030E040E05FE30F9461090F94D30A0F94F0
:10EE8000650A60935B0770935C0780935D079093BE
:10EE90005E0785EA93E00E94211D6B017C0181E7FA
:10EEA00093E00E94211D9B01AC01C701B6010F94A4
:10EEB000610920912F03309130034091310350912B
:10EEC00032030F946D0C0F946A0A60938707709356
:10EED00088078093890790938A0789EA93E00E94C4
:10EEE000211D6B017C0181E793E00E94211D9B01A4
:10EEF000AC01C701B6010F94610920912F03309135
:10EF0000300340913103509132030F946D0C0F94F4
:10EF10006A0A6093830770938407809385079093B0
:10EF200086078DEA93E00E94211D6B017C0181E739
:10EF300093E00E94211D9B01AC0140902F03509053
:10EF400030036090310370903203C701B6010F9413
:10EF50006109A30192010F946D0C0F946A0A4B0191
:10EF60005C01C0908707D0908807E0908907F090F7
:10EF70008A071091C8078FEFC816D806E104F1047C
:10EF8000C0F460917707709178078091790790912C
:10EF90007A079B01AC010F946109A30192010F94C0
:10EFA0006D0C20E03EEF4FE757E40F94F90B181675
:10EFB000D4F510681093C807C701B6010F94960ADC
:10EFC0009B01AC010F946D0C6093870770938807C9
:10EFD0008093890790938A076091830770918407D3
:10EFE00080918507909186070F94960A9B01AC014A
:10EFF0000F946D0C6093830770938407809385074B
:10F0000090938607C501B4010F94960A9B01AC0149
:10F010000F946D0C60937F07709380078093810736
:10F020009093820733C01F771093C807A7019601FA
:10F03000C701B6010F94340D60938707709388075A
:10F040008093890790938A07609183077091840762
:10F0500080918507909186079B01AC010F94340D38
:10F060006093830770938407809385079093860746
:10F07000A5019401C501B4010F94340D60937F077D
:10F080007093800780938107909382078DE993E0C6
:10F090000E94211D9B01AC010F946D0C60937B07B6
:10F0A00070937C0780937D0790937E07198A1A8A54
:10F0B0001B8A1C8A1D861E861F86188A80912B0734
:10F0C00090912C07A0912D07B0912E078D8B9E8BD0
:10F0D000AF8BB88FBE016F5F7F4FCE010D960E9440
:10F0E0000BED89819A81AB81BC8180938B079093D2
:10F0F0008C07A0938D07B0938E0780912B0790917A
:10F100002C07A0912D07B0912E0780932F07909385
:10F110003007A0933107B093320780933307909361
:10F120003407A0933507B093360710921F0710924B
:10F1300020071092210710922207109223071092A5
:10F140002407109225071092260710922707109285
:10F1500028071092290710922A0740902F035090F9
:10F160003003609031037090320320E030E040E7DC
:10F1700051E4C301B2010F946D0C0F94650A6093C2
:10F18000730770937407809375079093760787E2EF
:10F19000882E83E0982E91E4A92E98E0B92E0BEFEB
:10F1A00012E021E3222E28E0322EEBEEF2E0FD8F7A
:10F1B000EC8F81E298E09B8F8A8F198EF401C190C9
:10F1C000D190E190F1904F01A701960160E070E0CD
:10F1D00080E89FE30F94CC09F501619371938193CB
:10F1E00091935F01F80161917191819191918F01EA
:10F1F000A70196010F946D0C0F946A0AF1016193B7
:10F200007193819391931F01EC8DFD8D61917191AB
:10F2100081919191FD8FEC8FA70196010F946D0C58
:10F220000F946A0AEA8DFB8D619371938193919398
:10F23000FB8FEA8FF98DFF5FF98FF43009F0BECFB5
:10F24000A090EB02B090EC02C090ED02D090EE02E4
:10F25000E090FB02F090FC020091FD021091FE0292
:10F260009501A601B701C8010F94C50987FF02C027
:10F2700075018601209127033091280340912903CD
:10F2800050912A03B701C8010F946D0C9B01AC018A
:10F2900060E070E080E090E40F94CC090F94DA0C09
:10F2A0009B01AC01B701C8010F946D0C60933B0743
:10F2B00070933C0780933D0790933E07A090F30224
:10F2C000B090F402C090F502D090F602E0900303F3
:10F2D000F090040300910503109106039501A60127
:10F2E000B701C8010F94C50987FF02C075018601E7
:10F2F0009701A801C301B2010F946D0C9B01AC01F1
:10F3000060E070E080E090E40F94CC090F94DA0C98
:10F310009B01AC01B701C8010F946D0C60933707D6
:10F32000709338078093390790933A072ADB6D96DC
:10F330000FB6F894DEBF0FBECDBFDF91CF911F9106
:10F340000F91FF90EF90DF90CF90BF90AF909F9084
:10F350008F907F906F905F904F903F902F90089587
:10F36000EF92FF920F931F936093C9077093CA07A0
:10F370008093CB079093CC072093CD073093CE0793
:10F380004093CF075093D007E092D107F092D20775
:10F390000093D3071093D4071F910F91FF90EF9024
:10F3A0000895CF92DF92EF92FF9281E00E94151EA6
:10F3B00086E79AE00E946BCA0F94FC0320912C0C04
:10F3C000211148C02091C50722FD44C0C0908C1D6A
:10F3D000D0908D1DE0908E1DF0908F1D9B01AC0193
:10F3E0002C193D094E095F0969017A018091420398
:10F3F00090914303A0914403B09145030097A10568
:10F40000B10541F08C159D05AE05BF0518F480E0EF
:10F4100066DA05C08091C707877F8093C707809110
:10F420003E0390913F03A0914003B09141030097A8
:10F43000A105B10539F08C159D05AE05BF0510F489
:10F4400081E04DDA82E299E0FF90EF90DF90CF907B
:10F450000C94E99A60938C1D70938D1D80938E1D82
:10F4600090938F1DEFCFAF92BF92CF92DF92EF922A
:10F47000FF920F931F93CF93DF93EB01D82EC92EEA
:10F480001092FD071092FE071092FF0710920008DD
:10F4900010920108109202081092030810920408BA
:10F4A000109205081092060810920708109208089A
:10F4B00061E178E08DEF97E00E940BED60912B0702
:10F4C00070912C0780912D0790912E070F94980A28
:10F4D00020E030E040EC5FE30F946D0C0F94650A80
:10F4E0007B018C0121E02F932F93CF92DF92DF934A
:10F4F000CF93A12CB12C650120E030E0A90160E0A0
:10F5000070E0CB010E941FF81092F7061092F806E7
:10F510001092F9061092FA061092F3061092F40671
:10F520001092F5061092F6060F900F900F900F9024
:10F530000F900F90DF91CF911F910F91FF90EF905F
:10F54000DF90CF90BF90AF9008954F925F926F92EF
:10F550007F928F929F92AF92BF92CF92DF92EF9263
:10F56000FF920F931F93CF93DF9300D01F92CDB7DD
:10F57000DEB760911303709114038091150390918D
:10F58000160371DF60912F03709130038091310376
:10F59000909132039B01AC010F94610920E030E0AF
:10F5A00040EA50EC0F946D0C0F94650A2B013C015E
:10F5B0001F92992493949F9220E030E040E05FE313
:10F5C00060911303709114038091150390911603B9
:10F5D0000F946D0C9F938F937F936F93A12CB12CFD
:10F5E00065018301720120E030E0A90160E070E074
:10F5F000CB010E941FF820E030E040E05FE3609123
:10F6000013037091140380911503909116030F94C6
:10F610006D0C29DF20E030E040EA50EC60912F03D0
:10F620007091300380913103909132030F946D0CEF
:10F630000F94650A1F929F92209116032F93209199
:10F6400015032F93209114032F93209113032F93CD
:10F650007B018C0120E030E0A90160E070E0CB018B
:10F660000E941FF88DE793E00F94441280902707C3
:10F6700090902807A0902907B0902A07B094A094F2
:10F6800090948094811C911CA11CB11CAA2797FD09
:10F69000A095BA2F881A990AAA0ABB0A8FE793E0A5
:10F6A0000F944412C0902307D0902407E0902507C0
:10F6B000F0902607F094E094D094C094C11CD11C23
:10F6C000E11CF11CAA2797FDA095BA2FC81AD90AE8
:10F6D000EA0AFB0A81E893E00F94441240911F0765
:10F6E00050912007609121077091220770956095D5
:10F6F000509541955F4F6F4F7F4FAA2797FDA0957B
:10F70000BA2F481B590B6A0B7B0B0FB6F894DEBF60
:10F710000FBECDBF2A013B018C149D04AE04BF0473
:10F7200044F484169506A606B70654F42401350160
:10F7300007C0C416D506E606F70614F426013701FD
:10F7400084189508A608B708C418D508E608F7086D
:10F75000DB01CA0184199509A609B70989839A832F
:10F76000AB83BC831092FD071092FE071092FF0737
:10F7700010920008109201081092020810920308DB
:10F780001092040880912B0790912C07A0912D07CF
:10F79000B0912E078093050890930608A093070860
:10F7A000B093080861E178E08DEF97E00E940BEDDF
:10F7B0008091110890911208A0911308B09114083B
:10F7C00088199909AA09BB09809311089093120816
:10F7D000A0931308B093140880911508909116080F
:10F7E000A0911708B09118088C199D09AE09BF099E
:10F7F0008093150890931608A0931708B0931808E3
:10F800008091190890911A08A0911B08B0911C08CA
:10F8100029813A814B815C81821B930BA40BB50B30
:10F820008093190890931A08A0931B08B0931C08A2
:10F830001F9281E08F93809116038F93809115031F
:10F840008F93809114038F93809113038F93A12C36
:10F85000B12C65018301720120E030E0A90160E074
:10F8600070E0CB010E941FF81092FD071092FE0776
:10F870001092FF07109200081092010810920208DF
:10F88000109203081092040880912B0790912C0786
:10F89000A0912D07B0912E0780930508909306083C
:10F8A000A0930708B09308081092C9071092CA07DE
:10F8B0001092CB071092CC071092CD071092CE0772
:10F8C0001092CF071092D0071092D1071092D20752
:10F8D0001092D3071092D40761E178E08DEF97E0A2
:10F8E0000E940BED8091110890911208A0911308CD
:10F8F000B091140880934F0790935007A09351073D
:10F90000B09352078091150890911608A09117089E
:10F91000B09118088093530790935407A09355070C
:10F92000B09356078091190890911A08A0911B086E
:10F93000B0911C088093570790935807A0935907DC
:10F94000B0935A0760918B0770918C0780918D0757
:10F9500090918E070F94980A6B017C0120E030E0B3
:10F9600040EA50E460912F0370913003809131039D
:10F97000909132030F946D0C9B01AC01C701B6014D
:10F980000F9461090F94650A60938B0770938C073D
:10F9900080938D0790938E070F900F900F900F908C
:10F9A0000F900F90E0919003F091910380810F9060
:10F9B0000F900F900F90DF91CF911F910F91FF90BB
:10F9C000EF90DF90CF90BF90AF909F908F907F90FF
:10F9D0006F905F904F900C94F74F0F931F93CF93BE
:10F9E000DF9380910F08C1E018161CF0C0E08F5F14
:10F9F00001C0815080930F08179816981598809130
:10FA0000C8078E7F8093C8070091090110910901F2
:10FA1000D09109018C2F0E9439748C2F0E9445745B
:10FA20008C2F0E94517481E090E00F945004409A12
:10FA3000419A429A82E090E00F9450044098419895
:10FA40004298C1E001FB882780F98C270E94397415
:10FA5000812F81700E944574D2FB882780F98C2702
:10FA6000DF91CF911F910F910C9451744F925F923F
:10FA70006F927F928F929F92AF92BF92CF92DF92BE
:10FA8000EF92FF920F931F93CF93DF93CDB7DEB723
:10FA900028970FB6F894DEBF0FBECDBF2B013C01F7
:10FAA00029833A834B835C83ED82FE820F83188720
:10FAB0008501740120919D0730919E0740919F0719
:10FAC0005091A0070F946D0C4B015C012091A90788
:10FAD0003091AA074091AB075091AC0769817A81B8
:10FAE0008B819C810F946D0C9B01AC01C501B4010D
:10FAF0000F9461094B015C012091B5073091B60765
:10FB00004091B7075091B8076D817E818F819885AC
:10FB10000F946D0C9B01AC01C501B4010F946109F8
:10FB2000F60160837183828393832091A1073091D2
:10FB3000A2074091A3075091A407C301B2010F94FB
:10FB40006D0C4B015C012091AD073091AE074091E7
:10FB5000AF075091B00769817A818B819C810F94A6
:10FB60006D0C9B01AC01C501B4010F9461094B01FF
:10FB70005C012091B9073091BA074091BB075091C1
:10FB8000BC076D817E818F8198850F946D0C9B01E0
:10FB9000AC01C501B4010F946109F8016083718360
:10FBA000828393832091A5073091A6074091A707F0
:10FBB0005091A807C301B2010F946D0C4B015C0179
:10FBC0002091B1073091B2074091B3075091B4072B
:10FBD00069817A818B819C810F946D0C9B01AC01B2
:10FBE000C501B4010F9461094B015C012091BD076F
:10FBF0003091BE074091BF075091C0076D817E8153
:10FC00008F8198850F946D0C9B01AC01C501B401E7
:10FC10000F946109F701608371838283938328962F
:10FC20000FB6F894DEBF0FBECDBFDF91CF911F910D
:10FC30000F91FF90EF90DF90CF90BF90AF909F908B
:10FC40008F907F906F905F904F9008954F925F924A
:10FC50006F927F928F929F92AF92BF92CF92DF92DC
:10FC6000EF92FF920F931F93CF93DF93CDB7DEB741
:10FC700064970FB6F894DEBF0FBECDBF69837A8359
:10FC80008B839C832D833E834F835887E986FA8636
:10FC90000B871C8725013601E62EF72E082F192F1A
:10FCA00020EF33E244E759E4B701C8010F94C509D6
:10FCB00081110DC08091F1079091F207A091F30797
:10FCC000B091F40789839A83AB83BC830AC0C701D0
:10FCD000D8018093F1079093F207A093F307B093B4
:10FCE000F407CD80DE80EF80F88420EF33E244E734
:10FCF00059E4C701B6010F94C50981110DC0809167
:10FD0000F5079091F607A091F707B091F8078D835A
:10FD10009E83AF83B88708C0C092F507D092F607DC
:10FD2000E092F707F092F807C984DA84EB84FC8448
:10FD300020EF33E244E759E4C701B6010F94C50947
:10FD400081110DC08091F9079091FA07A091FB07EE
:10FD5000B091FC0789879A87AB87BC8708C0C0929F
:10FD6000F907D092FA07E092FB07F092FC07809126
:10FD7000C80785FF3DC029853A854B855C852D8761
:10FD80003E874F87588B2091F3063091F4064091BF
:10FD9000F5065091F6066D817E818F8198850F94CE
:10FDA0006109698B7A8B8B8B9C8B2091F706309144
:10FDB000F8064091F9065091FA0669817A818B81A3
:10FDC0009C810F946109AE01475F5F4F4A01DE01DC
:10FDD00015965D019E012F5F3F4F6901ED84FE8402
:10FDE0000F85188929893A894B895C893FDE24C0AF
:10FDF0002091F7063091F8064091F9065091FA06E5
:10FE000069817A818B819C810F94610969837A83EE
:10FE10008B839C832091F3063091F4064091F50684
:10FE20005091F6066D817E818F8198850F946109CE
:10FE30006D837E838F8398872091270330912803D9
:10FE40004091290350912A0369817A818B819C8199
:10FE50000F946D0C20E030E040E05FE30F94610907
:10FE60000F94D30A0F94650A6093D5077093D60751
:10FE70008093D7079093D80720912B0330912C03C0
:10FE800040912D0350912E036D817E818F81988545
:10FE90000F946D0C20E030E040E05FE30F946109C7
:10FEA0000F94D30A0F94650A6093D9077093DA0709
:10FEB0008093DB079093DC0720912F033091300370
:10FEC000409131035091320369857A858B859C85F9
:10FED0000F946D0C20E030E040E05FE30F94610987
:10FEE0000F94D30A0F94650A6093DD077093DE07C1
:10FEF0008093DF079093E00720EF33E244E759E473
:10FF0000C301B2010F94C5098823C1F08091EA02B0
:10FF100083FD14C0E0919003F091910320E030E064
:10FF200046E153E462A973A984A995A90F94F90B3A
:10FF300018165CF18091C70787FD27C020EF33E2D8
:10FF400044E759E468A579A58AA59BA50F94C5093E
:10FF5000882361F088A599A5AAA5BBA5809303076E
:10FF600090930407A0930507B093060741E061E072
:10FF700081E00E94EFF2811106C088E297E10E94C1
:10FF80009C9F80E019C081E017C02091330330911D
:10FF900034034091350350913603C301B2010F94ED
:10FFA0006D0C0F94650A6093E1077093E2078093EC
:10FFB000E3079093E407C2CF64960FB6F894DEBFD0
:10FFC0000FBECDBFDF91CF911F910F91FF90EF90AA
:10FFD000DF90CF90BF90AF909F908F907F906F9069
:10FFE0005F904F9008954F925F926F927F928F92A1
:10FFF0009F92AF92BF92CF92DF92EF92FF920F93B8
:020000021000EC
:100000001F93CF93DF93CDB7DEB728970FB6F89441
:10001000DEBF0FBECDBF2B013C0129833A834B834A
:100020005C83ED82FE820F83188785017401209125
:100030009D0730919E0740919F075091A0070F9414
:100040006D0C4B015C012091A1073091A2074091FA
:10005000A3075091A40769817A818B819C810F94B9
:100060006D0C9B01AC01C501B4010F9461094B01FA
:100070005C012091A5073091A6074091A7075091F8
:10008000A8076D817E818F8198850F946D0C9B01EF
:10009000AC01C501B4010F946109F601608371835D
:1000A000828393832091A9073091AA074091AB07DF
:1000B0005091AC07C301B2010F946D0C4B015C0170
:1000C0002091AD073091AE074091AF075091B00736
:1000D00069817A818B819C810F946D0C9B01AC01AD
:1000E000C501B4010F9461094B015C012091B10776
:1000F0003091B2074091B3075091B4076D817E8172
:100100008F8198850F946D0C9B01AC01C501B401E2
:100110000F946109F8016083718382839383209136
:10012000B5073091B6074091B7075091B807C301A2
:10013000B2010F946D0C4B015C012091B907309115
:10014000BA074091BB075091BC0769817A818B81C6
:100150009C810F946D0C9B01AC01C501B4010F94FF
:1001600061094B015C012091BD073091BE074091B0
:10017000BF075091C0076D817E818F8198850F9454
:100180006D0C9B01AC01C501B4010F946109F7012D
:10019000608371838283938328960FB6F894DEBFC1
:1001A0000FBECDBFDF91CF911F910F91FF90EF90C8
:1001B000DF90CF90BF90AF909F908F907F906F9087
:1001C0005F904F9008953F924F925F926F927F920F
:1001D0008F929F92AF92BF92CF92DF92EF92FF9257
:1001E0000F931F93CF93DF9300D01F92CDB7DEB74D
:1001F000382E6091FD077091FE078091FF07909166
:1002000000080F94980A20914108309142084091CB
:100210004308509144080F946D0C2B013C016093EE
:10022000F1077093F2078093F3079093F4076091BE
:1002300001087091020880910308909104080F94BE
:10024000980A2091450830914608409147085091FE
:1002500048080F946D0C69837A838B839C83609329
:10026000F5077093F6078093F7079093F80760916E
:1002700005087091060880910708909108080F946E
:10028000980A2091490830914A0840914B085091B2
:100290004C080F946D0C6093F9077093FA078093E4
:1002A000FB079093FC072091C80725FF15C049EF75
:1002B000842E47E0942E55EFA52E57E0B52EE1EFA2
:1002C000CE2EE7E0DE2E7B018C0129813A814B8125
:1002D0005C81C301B20187DE2091F7063091F806F8
:1002E0004091F9065091FA066091F1077091F2077A
:1002F0008091F3079091F4070F9460092B013C0162
:100300006093F1077093F2078093F3079093F407DB
:100310002091F3063091F4064091F5065091F606CF
:100320006091F5077091F6078091F7079091F807B3
:100330000F9460096093F5077093F6078093F707B1
:100340009093F807332001F14092E5075092E607B9
:100350006092E7077092E8076093E9077093EA07F5
:100360008093EB079093EC078091F9079091FA073F
:10037000A091FB07B091FC078093ED079093EE07E7
:10038000A093EF07B093F0070F900F900F900F908E
:10039000DF91CF911F910F91FF90EF90DF90CF9061
:1003A000BF90AF909F908F907F906F905F904F9095
:1003B0003F9008954F925F926F927F928F929F929B
:1003C000AF92BF92CF92DF92EF92FF920F931F9363
:1003D000CF93DF932B013C0149015A01670178015A
:1003E0008091C70785FD53C020E030E048EC52EC17
:1003F000C701B6010F94F90B87FD1DC02DEC3CEC35
:100400004CE45DE360910B0770910C0780910D0740
:1004100090910E070F94610920E030E040EA50E42B
:100420000F9461099B01AC01C1E0C701B6010F94B3
:10043000C50918160CF4C0E0A3019201C301B20172
:100440000F946D0C6B017C01A5019401C501B401F1
:100450000F946D0C9B01AC01C701B6010F946109AB
:10046000D1E020917B0730917C0740917D0750912E
:100470007E070F94C50918160CF4D0E0CD2341F483
:1004800081E0A1DE80E997E10E94451E01C0C1E044
:100490008C2FDF91CF911F910F91FF90EF90DF9004
:1004A000CF90BF90AF909F908F907F906F905F9014
:1004B0004F9008952F923F924F925F926F927F924A
:1004C0008F929F92AF92BF92CF92DF92EF92FF9264
:1004D0000F931F93CF93DF93CDB7DEB760970FB61F
:1004E000F894DEBF0FBECDBF1C0180910E08F10154
:1004F0001081811169C013FF20C0628573858485D6
:1005000095850E945D742091C9073091CA0740917A
:10051000CB075091CC070F9460096093F10770935B
:10052000F2078093F3079093F4076093E5077093C5
:10053000E6078093E7079093E80714FF21C0F101D5
:1005400066857785808991890E945D742091CD07A9
:100550003091CE074091CF075091D0070F9460099A
:100560006093F5077093F6078093F7079093F80769
:100570006093E9077093EA078093EB079093EC0789
:1005800015FF8BC0F10162897389848995890E9466
:100590005D742091D1073091D2074091D3075091DB
:1005A000D4070F9460096093F9077093FA0780935A
:1005B000FB079093FC076093ED077093EE07809321
:1005C000EF079093F00769C013FF21C0F101628526
:1005D0007385848595850E945D742091E50730912F
:1005E000E6074091E7075091E8070F94610960938F
:1005F000E5077093E6078093E7079093E807609319
:10060000F1077093F2078093F3079093F40714FFB8
:1006100021C0F10166857785808991890E945D748A
:100620002091E9073091EA074091EB075091EC07E0
:100630000F9461096093E9077093EA078093EB07D1
:100640009093EC076093F5077093F6078093F70794
:100650009093F80715FF21C0F1016289738984899D
:1006600095890E945D742091ED073091EE074091CD
:10067000EF075091F0070F9461096093ED077093B5
:10068000EE078093EF079093F0076093F90770935C
:10069000FA078093FB079093FC078091C80740906E
:1006A000ED075090EE076090EF077090F00785FF20
:1006B0003BC02091F3063091F4064091F50650912D
:1006C000F6066091E9077091EA078091EB07909137
:1006D000EC070F9461096D877E878F87988B209137
:1006E000F7063091F8064091F9065091FA066091AC
:1006F000E5077091E6078091E7079091E8070F946E
:1007000061099E012F5F3F4F4901AE014B5F5F4F73
:100710005A01FE0139966F01830172012D853E85D4
:100720004F855889A3D930C02091F7063091F8063B
:100730004091F9065091FA066091E5077091E6073D
:100740008091E7079091E8070F94610969877A879C
:100750008B879C872091F3063091F4064091F50633
:100760005091F6066091E9077091EA078091EB07D6
:100770009091EC070F9461096D837E838F83988736
:1007800049825A826B827C82209127033091280310
:100790004091290350912A0369857A858B859C8530
:1007A0000F946D0C20E030E040E05FE30F946109AE
:1007B0000F94D30A0F94650A6093D5077093D607F8
:1007C0008093D7079093D80720912B0330912C0367
:1007D00040912D0350912E036D817E818F819885EC
:1007E0000F946D0C20E030E040E05FE30F9461096E
:1007F0000F94D30A0F94650A6093D9077093DA07B0
:100800008093DB079093DC0720912F033091300316
:10081000409131035091320369817A818B819C81AF
:100820000F946D0C20E030E040E05FE30F9461092D
:100830000F94D30A0F94650A6093DD077093DE0767
:100840008093DF079093E007F1010081118106FF9B
:1008500035C18091EA0283FD31C1F101C688D78894
:10086000E08CF18C8090330390903403A09035039A
:10087000B0903603A5019401C701B6010F946D0C29
:100880000E945D740F94650A2B013C0180910E0853
:10089000E0919003F0919103811104C080910D08C3
:1008A0008823B1F120E030E046E153E462A973A966
:1008B00084A995A90F94C50987FF08C08091C7072F
:1008C00087FD04C0412C512C320115C0C701B6016F
:1008D0009F772091E5023091E6024091E702509126
:1008E000E8020F946D0C20E030E04AE754E40F94E6
:1008F000F90B18163CF38091090890910A08A09111
:100900000B08B0910C08840D951DA61DB71DDEC007
:1009100020E030E046E153E462A973A984A995A9D7
:100920000F94C50987FF04C08091C70787FFD7C010
:100930008091090890910A08A0910B08B0910C08C9
:10094000A3019201281B390B4A0B5B0BCA01B901A9
:100950000F94980A9F772091E5023091E60240912A
:10096000E7025091E8020F946D0C6B017C0120E0CE
:1009700030E04AE754E4C501B4010F946D0C9B01CB
:10098000AC01C701B6010F94F90B18160CF4A7C0FF
:100990004092E1075092E2076092E3077092E40709
:1009A00010FF3DC08091510800910107109102078E
:1009B0008823C9F02FE737EB4AE85BE3F101628D4A
:1009C000738D848D958D0F946D0C6B017C01B80136
:1009D000882777FD8095982F0F94980A9B01AC018A
:1009E000C701B60112C0B801882777FD8095982FFE
:1009F0000F94980AF101228D338D448D558D0F94FB
:100A00006D0C2EE333EC4EE259E30F946D0C6093C2
:100A10000307709304078093050790930607E090FF
:100A2000ED07F090EE070091EF071091F00720918D
:100A3000E9073091EA074091EB075091EC0760918C
:100A4000E5077091E6078091E7079091E807B2DC2F
:100A5000811111C08091E1079091E207A091E30715
:100A6000B091E4078093090890930A08A0930B08BB
:100A7000B0930C080AC0F101808191819C01287318
:100A80003327232BC9F486FD02C080E031C040919A
:100A9000E1075091E2076091E3077091E4078091CC
:100AA000090890910A08A0910B08B0910C0848170A
:100AB00059076A077B0749F381E01AC0809109084A
:100AC00090910A08A0910B08B0910C088093E1075F
:100AD0009093E207A093E307B093E40761CF4092BD
:100AE000090850920A0860920B0870920C0850CFC7
:100AF00060960FB6F894DEBF0FBECDBFDF91CF91E9
:100B00001F910F91FF90EF90DF90CF90BF90AF902B
:100B10009F908F907F906F905F904F903F902F901D
:100B200008954F925F926F927F92AF92BF92CF9251
:100B3000DF92EF92FF920F931F93CF93DF93CDB786
:100B4000DEB728970FB6F894DEBF0FBECDBF69831E
:100B50007A838B839C8329013A01ED82FE820F8385
:100B6000188720EF33E244E759E40F94C50988233E
:100B700011F12091F7063091F8064091F906509155
:100B8000FA0669817A818B819C810F946109209199
:100B90002703309128034091290350912A030F9491
:100BA0006D0C0F94650A6093D5077093D6078093F8
:100BB000D7079093D80720EF33E244E759E4C30105
:100BC000B2010F94C509882301F12091F3063091F9
:100BD000F4064091F5065091F606C301B2010F9458
:100BE000610920912B0330912C0340912D035091EA
:100BF0002E030F946D0C0F94650A6093D9077093C0
:100C0000DA078093DB079093DC0720EF33E244E7B9
:100C100059E46D817E818F8198850F94C509882361
:100C2000C1F020912F033091300340913103509156
:100C300032036D817E818F8198850F946D0C0F94A6
:100C4000650A6093DD077093DE078093DF0790935A
:100C5000E00720EF33E244E759E4C601B5010F9401
:100C6000C5098823B1F020913303309134034091BA
:100C7000350350913603C601B5010F946D0C0F94E6
:100C8000650A6093E1077093E2078093E30790930E
:100C9000E40720EF33E244E759E46A8D7B8D8C8DC5
:100CA0009D8D0F94C509882361F08A8D9B8DAC8D35
:100CB000BD8D8093030790930407A0930507B0931D
:100CC000060740E061E081E00E94EFF2811106C07A
:100CD00082E597E10E949C9F80E003C080E073DA88
:100CE00081E028960FB6F894DEBF0FBECDBFDF912E
:100CF000CF911F910F91FF90EF90DF90CF90BF9019
:100D0000AF907F906F905F904F9008950E94371E34
:100D100080E059DA8091F1079091F207A091F307F2
:100D2000B091F4078093E4069093E506A093E6065D
:100D3000B093E7068091F5079091F607A091F70729
:100D4000B091F8078093E0069093E106A093E20645
:100D5000B093E3068091F9079091FA07A091FB0701
:100D6000B091FC078093DC069093DD06A093DE062D
:100D7000B093DF066091090870910A0880910B0812
:100D800090910C080F94980A20914D0830914E08CC
:100D900040914F08509150080F946D0C6093D80605
:100DA0007093D9068093DA069093DB06809103074F
:100DB00090910407A0910507B09106078093E10286
:100DC0009093E202A093E302B093E40208958F921D
:100DD0009F92AF92BF92CF92DF92EF92FF920F93CA
:100DE0001F93CF93DF93982EC62FD42FC22E20E0CF
:100DF00030E0A9016091E1027091E2028091E3028A
:100E00009091E4020F94C50987FDA7C0911005C019
:100E1000C11103C0E1E0ED2701C0E0E0CC2049F0C2
:100E2000A090D806B090D906C090DA06D090DB0624
:100E300008C0F0EFAF2EF3E2BF2EF4E7CF2EF9E4B7
:100E4000DF2EE11102C0DD23B9F05091DC064091A4
:100E5000DD063091DE062091DF06852F942FA32F2B
:100E6000B22F8093ED079093EE07A093EF07B09316
:100E7000F007E11107C004C050EF43E234E729E472
:100E8000CC23B9F0D091E006C091E1067091E20662
:100E90006091E3068D2F9C2FA72FB62F8093E90733
:100EA0009093EA07A093EB07B093EC07E11107C01A
:100EB00004C0D0EFC3E274E769E49920B1F08090F8
:100EC000E4069090E506F091E606E091E706C4019D
:100ED000AF2FBE2F8093E5079093E607A093E70717
:100EE000B093E807B82DA92D04C0B0EFA3E2F4E752
:100EF000E9E41F930F93FF92EF92E52EF42E032F58
:100F0000122F2D2F3C2F472F562F6B2F7A2F8F2FDD
:100F10009E2F0E94267E8091E1029091E202A09194
:100F2000E302B091E4028093030790930407A09337
:100F30000507B09306070F900F900F900F9080E079
:100F4000DF91CF911F910F91FF90EF90DF90CF90A5
:100F5000BF90AF909F908F9036C9DF91CF911F9136
:100F60000F91FF90EF90DF90CF90BF90AF909F9048
:100F70008F9008959091C80795FB222720F982173A
:100F800091F0882311F0906201C09F7D9093C80773
:100F9000882319F082E190E202C08CEF9FE10E9469
:100FA000A69F80E010C90895AF92BF92CF92DF92C2
:100FB000EF92FF920F931F93CF93E82E062FF42EFC
:100FC000C091C807C5FBCC27C0F980E0D3DF909162
:100FD000C70791609093C707EE2021F0002339F0F6
:100FE0001F2D06C0011103C011E01F2501C010E034
:100FF00040E06DE077E186E79AE00E9499AB86E7F2
:101000009AE00E94EDAE111102C0FF2019F00E947B
:10101000A57A1FC0EE2041F01092D5071092D60796
:101020001092D7071092D807002341F01092D907E9
:101030001092DA071092DB071092DC0740E060E0C4
:1010400081E00E94EFF2811104C085EE96E10E94DA
:101050009C9FE0900B07F0900C0700910D071091FA
:101060000E07809116038F93809115038F938091C3
:1010700014038F93809113038F93A0EFAA2EA3E202
:10108000BA2EA4E7CA2EA9E4DA2E20E030E0A901A6
:10109000CA01B9010E94267E81E095D81092DF0A2C
:1010A0008BED96E10E94451E0F900F900F900F90D0
:1010B0008C2FCF911F910F91FF90EF90DF90CF90E9
:1010C000BF90AF9057CF2F923F924F925F926F9207
:1010D0007F928F929F92AF92BF92CF92DF92EF92C8
:1010E000FF920F931F93CF93DF93CDB7DEB72B976C
:1010F0000FB6F894DEBF0FBECDBF6A874D83409117
:10110000F7065091F8066091F9067091FA06498346
:101110005A836B837C834090F3065090F406609072
:10112000F5067090F606882309F4AEC0222321F05C
:101130008FE390E20E941D96C090F907D090FA07C5
:10114000E090FB07F090FC0781EA93E00E94211DEC
:101150009B01AC01C701B6010F94F90B18161CF5E1
:10116000E09013031091140300911503F0901603FF
:1011700081EA93E00E94211DFF920F931F93EF924B
:1011800010EFA12E13E2B12E14E7C12E19E4D12ED7
:101190007B018C01A6019501C601B501C2DC0F904F
:1011A0000F900F900F9080E293E00E94211DDC01D0
:1011B000CB01B0588093F7069093F806A093F906F8
:1011C000B093FA0684E293E00E94211DDC01CB017A
:1011D000B0588093F3069093F406A093F506B0936D
:1011E000F60688E493E00E94211DE62E172F082FB3
:1011F000F92EA30192016091F3067091F40680919B
:10120000F5069091F6060F94600920912B0330911A
:101210002C0340912D0350912E030F946D0C0F94CD
:10122000650A2B013C0129813A814B815C816091E7
:10123000F7067091F8068091F9069091FA060F94DE
:101240006009209127033091280340912903509190
:101250002A030F946D0C0F94650A21E02F932F93AE
:10126000FF920F931F93EF92A12CB12C6501E12CFB
:10127000F12C8701A30192010E941FF80F900F909B
:101280000F900F900F900F900E94371E20E030E0DB
:1012900040E251E460912F0370913003809131035B
:1012A000909132030F946D0C0F94650A6E837F83C7
:1012B00088879987609105087091060880910708D2
:1012C0009091080869837A838B839C8380911908A5
:1012D00090911A08A0911B08B0911C0880935707A1
:1012E00090935807A0935907B0935A071B86412C37
:1012F000512C32017D81272E312C7B85872E99241C
:1013000087FC9094821493040CF01DC1C0902B07AD
:10131000D0902C07E0902D07F0902E0780911F07AA
:1013200090912007A0912107B0912207C81AD90AED
:10133000EA0AFB0ACC0CDD1CEE1CFF1C8FEF9FEFB2
:10134000DC018093470790934807A0934907B09327
:101350004A0780E293E00E94211D84E293E00E940C
:10136000211D8091C80780648093C8070E94FA23DA
:101370000E94FA230AE010E0959B38C08CE293E0CB
:101380000E94211DA7019601EE24FF248701E21A85
:10139000F30A040B150B31E03F933F939F938F9318
:1013A0007F936F93A12CB12C650120E030E0A9015F
:1013B00060E070E0CB010E941FF80F900F900F903B
:1013C0000F900F900F908091470790914807A09140
:1013D0004907B0914A07B7FF18C086ED9FE10E9408
:1013E000B09F812C912C30E82FEBFAC18EEC96E166
:1013F0000E948F9F64E670E080E090E00F942B04E1
:101400000150110909F0B8CFB9CF8091C8078F7B7F
:101410008093C807009157071091580720915907EA
:1014200030915A078091190890911A08A0911B08D1
:10143000B0911C08B901A801481B590B6A0B7B0B22
:10144000DB01CA014093470750934807609349075F
:1014500070934A0740911108509112086091130847
:1014600070911408480F591F6A1F7B1F4093110881
:101470005093120860931308709314084091150854
:10148000509116086091170870911808480F591F5D
:101490006A1F7B1F40931508509316086093170826
:1014A000709318080093190810931A0820931B08CA
:1014B00030931C0840910508509106086091070878
:1014C00070910808480F591F6A1F7B1F4093050839
:1014D00050930608609307087093080889819A81E1
:1014E000AB81BC81841B950BA60BB70B480E591E14
:1014F0006A1E7B1EC40101968215930504F58CE2D9
:1015000093E00E94211D1F9251E05F939F938F9360
:101510007F936F93A12CB12C6501EE80FF8008852D
:10152000198520E030E0A90160E070E0CB010E9465
:101530001FF80F900F900F900F900F900F906B85EA
:101540006F5F6B87DACEC301B2010F94980A2091C6
:10155000490830914A0840914B0850914C080F942B
:101560006D0C6B017C01AD816A2F70E080E090E032
:101570000F94960A9B01AC01C701B6010F94CC09E8
:101580006B017C0188E293E00E94211D9B01AC016C
:10159000C701B6010F9461094B018E839D8322E040
:1015A000AB01BC018EEA90E20E94CBA120E030E0CA
:1015B00040EA52E4B4018E819D810F946D0C20E0CD
:1015C00030E048EC54E40F946009AB01BC0122E028
:1015D00082E890E20E94CBA14091F1075091F2077E
:1015E0006091F3077091F40722E08BE494E20E948B
:1015F000CBA14091F5075091F6076091F7077091E4
:10160000F80722E087E494E20E948EA180E00E9425
:10161000E38088EC96E10E94451E8CE293E00E94F4
:10162000211D9B0140910508509106086091070813
:1016300070910808E980FA800B811C81E41AF50A90
:10164000060B170B1F9241E04F939F938F933F938D
:101650002F93A12CB12C650120E030E0A90160E0BE
:1016600070E0CB010E941FF80F900F900F900F9029
:101670000F900F90BA85BB2309F4B0C0C090F70655
:10168000D090F806E090F906F090FA062090F30664
:101690003090F4064090F5065090F6068EE390E206
:1016A0000E941D96609090037090910361147104E4
:1016B00009F444C0F30181819281A381B4819C012A
:1016C000AD0166277727CB01621B730B840B950B4B
:1016D0000F94980A209141083091420840914308A4
:1016E000509144080F946D0C6093F7067093F806C0
:1016F0008093F9069093FA06F30185819681A7817C
:10170000B0859C01AD0166277727CB01621B730B67
:10171000840B950B0F94980A209145083091460848
:1017200040914708509148080F946D0C6093F30660
:101730007093F4068093F5069093F60688E493E0A0
:101740000E94211D5B01182F092FA20191016091B8
:10175000F3067091F4068091F5069091F6060F94C9
:10176000600920912B0330912C0340912D0350915F
:101770002E030F946D0C0F94650A2B013C01A701F9
:1017800096016091F7067091F8068091F9069091A4
:10179000FA060F94600920912703309128034091A5
:1017A000290350912A030F946D0C0F94650A21E0D0
:1017B0002F932F930F931F93BF92AF92A12CB12C15
:1017C0006501E12CF12C8701A30192010E941FF811
:1017D0000F900F900F900F900F900F903E812D81E2
:1017E000B401832F922F2B960FB6F894DEBF0FBE55
:1017F000CDBFDF91CF911F910F91FF90EF90DF90C0
:10180000CF90BF90AF909F908F907F906F905F90A0
:101810004F903F902F90089540E050E060E87FE3C4
:101820004093BD075093BE076093BF077093C007F6
:101830004093AD075093AE076093AF077093B00726
:1018400040939D0750939E0760939F077093A00756
:101850001092B9071092BA071092BB071092BC07FA
:101860001092B5071092B6071092B7071092B807FA
:101870001092B1071092B2071092B3071092B407FA
:101880001092A9071092AA071092AB071092AC070A
:101890001092A5071092A6071092A7071092A8070A
:1018A0001092A1071092A2071092A3071092A4070A
:1018B000811104C087E290E20C94A69F089588E10C
:1018C0000FB6F89480936000109260000FBE809174
:1018D000C70780648093C70754985C9A389A399AEE
:1018E0003A9A80910A01826080930A0180910A01EC
:1018F000816080930A0180910A01846080930A01CB
:101900000F9A179A0E9A169A0D9A159A0A98129A81
:101910000998119A3F98479A9D98A59A809101013C
:10192000806280930101809102018F7D809302018A
:1019300080910101806480930101809102018F7B7D
:101940008093020180910101806180930101809167
:1019500002018F7E809302010E94AC210E94D62258
:1019600081E05ADF80E090E0A8E4B2E480930307CE
:1019700090930407A0930507B093060784E690E0D0
:101980009093020780930107909300078093FF06CE
:101990001092ED071092EE071092EF071092F007E9
:1019A0001092E9071092EA071092EB071092EC07E9
:1019B0001092E5071092E6071092E7071092E807E9
:1019C0001092900710928F071092821D1092831D23
:1019D0001092841D1092851D80E090E0A0EEB1E48D
:1019E0008093FB069093FC06A093FD06B093FE0641
:1019F0001092F3061092F4061092F5061092F60675
:101A00001092F7061092F8061092F9061092FA0654
:101A100088E893E1A0E0B0E08093990790939A075B
:101A2000A0939B07B0939C0781E08093E9021092FA
:101A3000ED061092EE061092EF061092F00610924C
:101A4000E9061092EA061092EB061092EC068093DB
:101A5000C80780E090E0AAE7B3E480931B07909367
:101A60001C07A0931D07B0931E0780931307909344
:101A70001407A0931507B093160780E090E0A6E640
:101A8000B3E480930B0790930C07A0930D07B093DA
:101A90000E0710921707109218071092190710924C
:101AA0001A0710920F071092100710921107109248
:101AB0001207109207071092080710920907109258
:101AC0000A0782EC95EFA1EBB2E48093770790933D
:101AD0007807A0937907B0937A071092E8061092DE
:101AE0005308109252080E9418CF40913A03509127
:101AF0003B0360913C0370913D038AE39BE00E94AD
:101B0000A0DD82EB94E20E948F9F86E79AE00E941C
:101B1000C4AB0E9498DA0E94724F0E9430D6109295
:101B2000FD071092FE071092FF0710920008109216
:101B3000F1071092F2071092F3071092F407109237
:101B400001081092020810920308109204081092E3
:101B5000F5071092F6071092F7071092F807109207
:101B600005081092060810920708109208081092B3
:101B7000F9071092FA071092FB071092FC071092D7
:101B8000090810920A0810920B0810920C08109283
:101B9000FD071092FE071092FF07109200080E94A6
:101BA000DB740E9414230E9422230E9478DA61E1F0
:101BB00078E08DEF97E00E940BED8AEF93E00F94B1
:101BC00037129091C607882311F0926001C09D7F63
:101BD0009093C607682F70E085EC93E00E9474A094
:101BE00088E197E10E94451E80E00E94F74F82E263
:101BF00099E00E949F9A2EE088E190E00FB6F89459
:101C0000A895809360000FBE2093600008954F92C6
